:020000040000FA
:0400000053EF48F082
:0200080008D01E
:0800180000D0E0CF02F101016C
:10002000D8CF01F1E8CF00F181509EB069EC39F0F2
:10003000F2B450EC39F0A1B265EC39F09EBA10EC94
:1000400039F0F2B23EEC39F0F0B044EC39F000C1D6
:0C005000E8FF01C1D8FF02C1E0FF100072
:10007000001210180606080A0A0C0606080A060AE4
:1000800006060808060E06060A0A08140C0A060ADE
:100090000806060610101010101010101010101086
:1000A0001010101010101010101010101010101050
:1000B000101010101014161416120C140E14141420
:1000C0000E180A0608080A060C0A08080808060698
:1000D000040A0C120A0A0A060A0E1408080612126A
:1000E000040E140806100E0C060608060606060680
:1000F000080804040A16161614080A080806060A50
:100100000808040A0C08060C0A141010101010102D
:1001100010101010101010101010101010101010DF
:1001200010101010101010101010140E0E0E0808E1
:10013000061414141414141414141414141414148D
:10014000141414141414141414141414141414146F
:100150001414141414141414141414140A0A0A0889
:100160000808080E0614100A100C060606060608F3
:10017000020E0E080808060606060A0A0408040EFF
:100180001412140E0A0E0C100E0A0A0A0E0C10009D
:1001C00000000019000241024102142314411423CB
:1001D000145F147D14B973020018000032020A1E65
:1001E0000A370A500A690A8214232041205F209BA3
:1001F000060037020E02280232021423640064193A
:10020000644B646400002823282328232823282300
:100210002823282328232823282328232823282386
:100220002823282328232823282328232823282376
:100230002823282328232823282328232823282366
:1002400028232823282300230041005F007D009BF2
:1002500000B900D700230041005F007D009B00B97A
:1002600000D7669600006CD86CD8640000000000CF
:10027000000000000000000000000000000000007E
:10028000000028021423147D557D557D557D557D34
:1002900000000A02000000001423144114020000B0
:1002A000145F0A020009557D0012001B0024002D76
:1002B0000036643264196432644B64646400641907
:1002C00014414141414164320A000A190A320A4B81
:1002D0006432557D6978693C4102149B2A483C028E
:1002E00034603478644BA07D000802270230557DCD
:1002F000144128232823282328232823282328239C
:100300002823282328232823282328232823282395
:100310002823282328232823282328232823282385
:100320002823282328232823282328232823282375
:1003300028230D02145F00020230000000000000BC
:1003400000230041005F007D009B00B900D700231F
:100350000041005F007D009B00B900D700230041F1
:10036000005F007D009B00B900D700230041005FC3
:10037000007D009B00B900D700230041005F007D95
:10038000009B00B900D700230041005F007D009B67
:1003900000B900D70A02557D020C6419640064009C
:1003A00064196400020C64641441021E147D1E0270
:1003B000142364196432644B646464006432000082
:1003C00014232802692369236923010141A8073006
:1003D0007887022700D80A080A10000018020023B4
:1003E0000041005F007D145F1441145F147D149B75
:0C03F000643264005A36145F147D149BC4
:100430004275696C64696E67204D4432204861736F
:10044000687D506C6561736520576169742E2E2E2E
:100450007D7D4865696E72696368735765696B6114
:100460006D70204F535443327D7D4D656E753F7DD9
:100470004D656E753A7D4C6F67626F6F6B7D47613E
:10048000732053657475707D5365742054696D6570
:100490007D7D5265736574204D656E757D7D5365F8
:1004A0007475707D457869747D7D576169742E2EF1
:1004B0007D7D4D443220486173683A7D44657361A7
:1004C000747D496E746572666163657D5374617293
:1004D000747D446174617D7D4865616465727D7D74
:1004E00050726F66696C657D446F6E652E7D4361E9
:1004F0006E63656C2052657365747D7D54696D65AE
:100500003A7D446174653A7D53657420486F757215
:10051000737D52657365742E2E2E7D7D4C6F6762E0
:100520006F6F6B7D437573746F6D2046756E63746A
:10053000696F6E7320497D7D5265736574204D65CA
:100540006E757D7D5365742054696D653A7D4D6F80
:1005500072657D7D4465636F706C616E7D7D476102
:10056000736C6973747D4D6F72657D7D45786974B8
:100570007D7D4E6F466C797D537461727420446941
:100580007665205B636D5D7D456E642044697665AC
:100590002020205B636D5D7D456E642044656C6149
:1005A000792020205B735D7D506F776572204F66E8
:1005B000662020205B735D7D5072652D6D656E75C4
:1005C000202020205B735D7D76656C6F6369747994
:1005D0005B6D2F6D696E5D7D57616B652D7570204C
:1005E000205B6D4261725D7D6D61782E5375726620
:1005F0002E5B6D4261725D7D474620646973706C4D
:10060000617920205B255D7D6D696E2E204F322043
:100610004469732E5B255D7D44697665206D656E4A
:10062000757320205B735D7D5361747572617465B1
:10063000207820205B255D7D44657361747572614F
:10064000746520785B255D7D4E6F466C7920526124
:1006500074696F205B255D7D474620616C61726D1A
:10066000203120205B255D7D434E5373686F7720DA
:10067000737572665B255D7D4465636F204F6666AA
:100680007365745B646D5D7D70704F32206C6F7745
:10069000205B634261725D7D70704F3220686967D4
:1006A000685B634261725D7D70704F322073686F6A
:1006B000775B634261725D7D73616D706C696E67BB
:1006C000207261746520207D44697669736F7220A1
:1006D00054656D702020207D44697669736F7220A7
:1006E0004465636F6461747D44697669736F7220D9
:1006F0004E6F74557365317D44697669736F7220EE
:1007000070704F322020207D44697669736F7220AB
:10071000446562756720207D44697669736F722035
:100720004E6F74557365327D434E5373686F7720F7
:10073000646976655B255D7D4C6F67626F6F6B20CA
:100740006F6666736574207D4C61737420446563C5
:100750006F2061745B6D5D7D456E642041706E6FCE
:1007600065205B6D696E5D7D53686F7720566261B1
:100770007474205B3D315D7D546869732070726FC5
:100780006772616D2069737D6469737472696275E3
:1007900074656420696E207468657D7D686F70651E
:1007A00020746861742069742077696C6C206265BC
:1007B0007D7D75736566756C2C2062757420574954
:1007C00054484F55547D414E592057415252414E45
:1007D00054593B20776974686F75747D6576656ED2
:1007E0002074686520696D706C6965647D7D7761D2
:1007F0007272616E7479206F667D4D455243484137
:100800004E544142494C495459206F727D7D4649AE
:10081000544E45535320464F5220417D504152542F
:100820004943554C415220505552504F53452E7D0F
:100830005365652074686520474E552047656E6591
:1008400072616C7D5075626C6963204C6963656E82
:10085000736520666F727D7D6D6F7265206465744F
:1008600061696C733A7D7777772E6865696E726916
:100870006368737765696B616D702E64657D44652F
:10088000636F73746F707D7D6D2F6D696E7D4E6FBC
:100890002053746F707D4465636F73756D7D44691B
:1008A000766574696D657D7D44657074687D4669A3
:1008B000727374204761733F7D7D44656661756C1A
:1008C000743A7D7D4D696E757465737D4D6F6E7480
:1008D0006820207D446179202020207D5965617247
:1008E0002020207D536574207D7D47617323207D0A
:1008F0005965737D43757272656E743A7D7D53657B
:10090000747570204D656E753A7D437573746F6DA7
:100910002046756E6374696F6E73497D4465636FBD
:10092000747970653A7D5A482D4C3136204F437D9D
:100930004761756765202020207D47617567657D6B
:100940005A482D4C31362043437D416374697665A6
:10095000204761733F207D7D476173205365747527
:1009600070202D204761736C6973747D44657074C9
:1009700068202B7D4465707468202D7D4261636B17
:100980007D7D43435220536574506F696E74204DD2
:10099000656E757D43435220536574506F696E7464
:1009A000204D656E757D5350237D42617474657270
:1009B0007920496E666F7D7D42617474657279201D
:1009C000496E666F726D6174696F6E7D4379636C99
:1009D00065733A7D41706E6F657D4C617374204321
:1009E0006F6D706C6574653A7D7D4C6F776573745F
:1009F0002056626174743A7D4C6F77657374206120
:100A0000743A7D7D546D696E3A7D546D61783A7D9E
:100A1000536574204761737D4F32202B7D7D4F32AB
:100A2000202D7D7D4865202B7D7D4865202D7D7D99
:100A3000457869747D7D44656C6574657D7D44652C
:100A40006275673A7D7D4F4E207D4F46467D4465F9
:100A50006C2E20616C6C7D7D556E6578706563745D
:100A600065642072657365742066726F6D7D44697C
:100A700076656D6F64652120506C656173652068D3
:100A8000656C707D616E64207265706F7274207425
:100A90006865204465627567207D496E666F726D7A
:100AA0006174696F6E2062656C6F77217D7D426134
:100AB000696C6F75747D41706E6F65202020207D9C
:100AC00044657363656E747D537572666163657D9D
:100AD000517569743F7D4D6F72657D7D436F6E66A4
:100AE00069726D3A7D7D4D656E7520323A7D436148
:100AF0006E63656C7D7D4F4B217D53746F707761A4
:100B0000742E7D7D3A2E2E2E2E2E2E2E2E2E3A7DBA
:100B10002870704F323A7D7D42617229207D4E6F80
:100B20007420757365642121217D4C31362D474633
:100B3000204F437D437573746F6D2046756E6374EB
:100B4000696F6E7349497D7D4746204C6F77202041
:100B5000202020205B255D7D47462048696768206E
:100B6000202020205B255D7D436F6C6F7223204227
:100B7000617474657279207D436F6C6F72232053AA
:100B800074616E646172647D436F6C6F7223204484
:100B90006976656D61736B7D436F6C6F722320574F
:100BA00061726E696E67737D53686F7720736563DA
:100BB000732E205B3D315D7D4469766520636C6FEB
:100BC000636B205B3D315D7D6E6F74207573656472
:100BD000202020202020207D4176722E2044657028
:100BE0007468205B3D315D7D426C696E6B204761AE
:100BF0007320205B3D315D7D446570746857617280
:100C00006E5B6D4261725D7D434E53207761726E03
:100C1000696E67205B255D7D4746207761726E694E
:100C20006E6720205B255D7D70704F32207761728A
:100C30006E5B634261725D7D56656C2E7761726E8C
:100C40005B6D2F6D696E5D7D54696D65206F6666A5
:100C5000736574205B735D7D6E6F7420757365645E
:100C6000202020202020207D6E6F74207573656405
:100C7000202020202020207D6E6F742075736564F5
:100C8000202020202020207D6E6F742075736564E5
:100C9000202020202020207D6E6F742075736564D5
:100CA000202020202020207D6E6F742075736564C5
:100CB000202020202020207D6E6F742075736564B5
:100CC000202020202020207D6E6F742075736564A5
:100CD000202020202020207D6E6F74207573656495
:100CE000202020202020207D6E6F74207573656485
:100CF000202020202020207D6E6F74207573656475
:100D0000202020202020207D6E6F74207573656464
:100D1000202020202020207D6E6F74207573656454
:100D2000202020202020207D6E6F74207573656444
:100D3000202020202020207D6E6F74207573656434
:100D4000202020202020207D437573746F6D204665
:100D5000756E6374696F6E732049497D53686F7750
:100D6000204C6963656E73657D7D53696D2E2052DD
:100D70006573756C74733A7D4E4F542055534544DA
:100D800021212121217D70704F32202B7D7D7070BB
:100D90004F32202D7D7D44696C2E7D7D4465636FCF
:100DA000747970653A205A482D4C3136204F437D76
:100DB000466F72204F70656E204369726375697467
:100DC0002020207D4469766572732E2053757070E3
:100DD0006F7274732035207D5472696D6978204775
:100DE000617365732E2020202020207D436F6E6666
:100DF000696775726520796F757220676173207DF0
:100E0000696E204761737365747570206D656E75CA
:100E10002E20207D436865636B20434631312026B8
:100E2000204346313220217D4465636F74797065BB
:100E30003A204761756765202020207D44697665EA
:100E400074696D652077696C6C20626520696E7DC0
:100E50004D696E757465733A5365636F6E64732E76
:100E60002020207D4F535443322077696C6C206ED4
:100E70006F7420202020207D636F6D707574652055
:100E80004465636F2C204E6F466C797D74696D6587
:100E900020616E642044657361742E2D2020207DB6
:100EA00074696D6520617420616C6C2120202020A4
:100EB0002020207D4465636F747970653A5A482D0F
:100EC0004C3136204343207D466F72202853656D98
:100ED000692D29436C6F73656420207D43697263BB
:100EE0007569742072656272656174686572737D7C
:100EF000436F6E666967757265207468652033207C
:100F00002020207D536574506F696E747320696E64
:100F100020434352202D207D5365747570206D65EC
:100F20006E752E2035206261696C2D7D6F7574732E
:100F30002061726520617661696C61626C652E7DED
:100F40004465636F747970653A2041706E6F6520F7
:100F50002020207D4F535443322077696C6C2064ED
:100F60006973706C6179207D656163682064657365
:100F700063656E742073657061722D7D6174656C3C
:100F80007920696E204D696E3A5365632E20207D6D
:100F900057696C6C2074656D706F72616C6C792030
:100FA0007365747D73616D706C65726174652074B6
:100FB0006F2031207365637D4E6F204465636F2021
:100FC00063616C63756C6174696F6E7D4465636F9A
:100FD000747970653A204C31362D4746204F437D59
:100FE0004465636F6D7072657373696F6E206361C2
:100FF0006C2D207D63756C6174696F6E73207769E9
:10100000746820746865207D47462D4D6574686F4F
:1010100064202847465F6C6F2F47467D5F686929CB
:101020002E20436865636B20434633322026207DA3
:101030004346333321204F70656E204369726375D8
:101040006974207D776974682044656570205374E5
:101050006F70732E2020207D4465636F74797065F6
:101060003A204C31362D47462043437D4465636F1B
:101070006D7072657373696F6E2063616C2D207D76
:1010800063756C6174696F6E73207769746820741E
:101090006865207D47462D4D6574686F642028473C
:1010A000465F6C6F2F47467D5F6869292E20436835
:1010B00065636B20434633322026207D434633331D
:1010C00021436C6F73656420436972637569747D35
:1010D0007769746820446565702053746F70732E4F
:1010E0002020207D4465636F6D6F646520636861B7
:1010F0006E6765642120207D4C31362D47462043A4
:10110000437D4E6F7420666F756E647D53657450B9
:101110006F696E747D7D4E6F204465636F7D47728D
:10112000617068737D7D446973706C61797D4E6F09
:10113000206465636F7D536561726368206D6F64C1
:10114000756C657D457869747D7D52657365742025
:1011500043462C4761732026204465636F7D4469B4
:101160007361626C65206D6F64756C657D7D53691C
:101170006D756C61746F727D4F5354432053696D6C
:10118000756C61746F727D7D5374617274204469F3
:1011900076657D7D2B20316D7D7D2D20316D7D7DB2
:1011A0002B31306D7D7D2D31306D7D7D45786974BD
:1011B0007D7D6E6F74207573657D787D4461746587
:1011C00020666F726D61743A7D7D53657475702011
:1011D0004D656E7520323A7D4D4D444459597D7DA3
:1011E00044444D4D59597D7D59594D4D44447D7D63
:1011F0004F535443207D4261696C7D7D416972206B
:101200007D7D41697220207D43616C6962726174E9
:10121000657D4D61782044657074687D6E6F747D66
:10122000666F756E64217D7D6D563A7D4E657720C3
:101230004346206164646564217D4E657720437573
:1012400073746F6D46756E6374696F6E737D7765C9
:1012500072652061646465642120436865636B7D09
:101260004346204920616E64204346204949204D71
:10127000656E757D666F722044657461696C73215B
:101280007D7D53616C696E6974793A7D426F7474C7
:101290006F6D2054696D653A7D7D4D61782E2044D7
:1012A000657074683A7D43616C63756C6174652028
:1012B0004465636F7D7D53686F77204465636F700D
:1012C0006C616E7D4C656164205469737D7D4C65F5
:1012D0006164205469737D7D53746F7077617463AA
:1012E000687D5265736574204C6F67626F6F6B7DAC
:1012F0005265626F6F74204F5354437D526573651E
:1013000074204465636F646174617D7D2B8B01D8AB
:101310001200268D05D8269D12002B8B01D81200B5
:101320000B6F800EA66EF86A010EF76EBC0EF66E9D
:101330000BC14BF1000E2BBB010E4C6FD8904B37FD
:101340004C37020E4B27000E4C234B51F6264C51C6
:10135000F722090026ADF5CF7DF0090026ADF5CFC7
:101360007CF0000EE8CF7EF00D6B0E6BF76AF86A2A
:10137000700EF66E01D02B9B0900F5500D27000E64
:101380000E230B2FF9D72BBBF6D7F86A300E0D259D
:10139000F66E040E0E21F76E26AD20EE60F0090009
:1013A0007D0EF56201D00AD0F5CFDEFF09007D0E7B
:1013B000F56201D003D0F5CFDEFFF1D726AD4EECBC
:1013C0000CF0120031C14BF132C14CF13C0E4D6FAB
:1013D0004E6B4FD847C132F14BC131F11200D8905A
:1013E00045334433462FFBD71200D8904A33493354
:1013F00048334733462FF9D712004851FF08486F4A
:101400004751D890FF08476F12001E975351515D06
:101410004F6F54515259506FD8A812001E874FC1B8
:1014200053F150C154F1516952695351515D4F6F9D
:1014300054515259506F1200496B4A6B4B514D0336
:10144000F350476FF450486F4B514E03F350482709
:10145000F45049234C514D03F3504827F45049238D
:10146000D8B04A2B4C514E03F3504927F4504A232D
:101470001200476B486B4D514E11D8B4FF0C010E52
:10148000466F4EBF05D0462BD8904D374E37F9D713
:10149000D890473748374D514B5F4E51D8A04E2911
:1014A0004C5FD8B005D04D514B274E514C2301D045
:1014B00047814607D8B41200D8904E334D33E8D751
:1014C000200E466F4A514C6F49514B6F4851526F35
:1014D0004751516F4A6B496B486B476B546B536B69
:1014E000D890513752374B374C37533754374E51CA
:1014F000545DD8A47EEF0AF04D51535DD8A088EF1B
:101500000AF04D51535FD8A054074E51545FD88014
:101510004737483749374A37462F70EF0AF01200ED
:10152000D89074337333752FFBD71200D89079336A
:10153000783377337633752FF9D712007751FF0858
:10154000776F7651D890FF08766F120029978251F5
:10155000805D7E6F835181597F6FD8A812002987E3
:101560007EC182F17FC183F1806981698251805D92
:101570007E6F835181597F6F1200786B796B7A513E
:101580007C03F350766FF450776F7A517D03F350FC
:101590007727F45078237B517C03F3507727F4505E
:1015A0007823D8B0792B7B517D03F3507827F45002
:1015B000792312000A6FE6EF0AF000000000000035
:1015C000000000000000000000000000000000001B
:1015D000000000000000000000000000000000000B
:1015E00000000000000000000000000000000000FB
:1015F00000000000000000000000000000000000EB
:10160000000000000A2FDDEF0AF01200096F12EF50
:101610000BF00000000000000000000000000000CF
:1016200000000000000000000000000000000000BA
:1016300000000000000000000000000000000000AA
:10164000000000000000000000000000000000009A
:101650000000000000000000000000000000630E19
:10166000DAEC0AF0092F09EF0BF01200630E31617A
:10167000316F31C133F1346B1E950A0E396F356B02
:1016800067D8010E396F356B1E8562D8120031C1E3
:1016900033F1346B1E85F1D731C133F1346B1E95B4
:1016A000640E396F356B54D8E8D7249F366F1E8B84
:1016B000362B362F1E9B228B362B362F229B31C189
:1016C00033F132C134F11E95100E396F270E356F8C
:1016D0001EAD3ED8E80E396F030E356F22BB07D022
:1016E00024BF03D01E85362D1E9522B91E851EAD42
:1016F0002FD81E9D640E396F356B26B924D022BBBE
:1017000009D024BF03D01E85362D1E9522B91E8513
:1017100022BB1E851DD80A0E396F356B22BB09D03E
:1017200024BF03D01E85362D1E9522B91E8522BBEF
:101730001E8528B708D00CD8010E396F356B1E8571
:1017400023A506D823952699376B372B22991200AB
:10175000386B3551345DD8A00ED004E13951335D7A
:10176000D8A009D03551345F3951335FD8A0340740
:10177000382B1E85EED7372F1200372B300E382529
:101780001EB504D01EBF04D0200E01D0248FDE6E03
:10179000362F12002E0EDE6E22891200A96E2DD079
:1017A000A96E27D02A91010EAA6E690E03D0259149
:1017B000AA6A640EAD6E228F040EA96E9D9A9E9A3F
:1017C000818646D8AECFA8FF818825BF0FD015D817
:1017D0008198A8CFADFF36D8A93EF3D781969E9ABF
:1017E0009D8AAA6A259F229FBEEF48F0FF0EAD6E2C
:1017F000F5D7A69EA69CA6801200A69EA69CA684AF
:10180000F29E550EA76EAA0EA76EA682F28EA6B203
:10181000FED7A6941200948C948E240EAC6E900E7B
:10182000AB6E080EB86EB06A220EAF6EAE6A9E6ADC
:101830009D8A1200AC6AAB6A9D9A949C949E829C8D
:10184000829E1200ABAE12000000ACA2FBD71200C9
:101850009E9A259F426B436B9EBA120000000000C7
:10186000000000009EBA120000000000000000000E
:101870009EBA120000000000000000009EBA120094
:1018800000000000000000009EBA1200432FE4D7C1
:10189000422FE1D7AB98AB88258F1200DE6A7BC060
:1018A000F7F17AC0F6F134EC5AF00101F7C17BF0A0
:1018B000F6C17AF01200106F10C17DF0210E2DD903
:1018C000D8901035000ED8B0010E2CD9D890103514
:1018D00029D912000F6F0FC17CF0200E1ED9000E07
:1018E00021D90F511FD91200220E17D984807AC036
:1018F00083FF809480847BC083FF80948084210E4A
:101900000CD9D8901035000ED8B0010E0BD9D89054
:101910001037102907D9200E00D9000E03D90F5116
:1019200001D9220EFAD884807AC083FF8094808403
:101930007BC083FF809480841200220EEED88480C6
:101940007AC083FF809480847BC083FF80948084EE
:101950001200836A80968194809A84948094849201
:101960001200F1514EEC0EF0F2C11BF11B51B2DF2F
:10197000F4515BEC0CF0E1DF1B2B1B51F363F6D74A
:101980001B51A8DFF4515BEC0CF0D7DFF2C11BF167
:101990001B51A0DFF5515BEC0CF0CFDF1B2B1B5173
:1019A000F363F6D71B5196DFF5515BEC0CF0C5DF06
:1019B000F4C11BF11B517FDFF2518CDF95DF1B2B34
:1019C0001B51F563F7D7F4C11BF11B5174DFF351C1
:1019D00081DF8ADF1B2B1B51F563F7D755EC18F01D
:1019E0001200F1514EEC0EF0350E97D8F4C11BF1F8
:1019F000D8901B35000ED8B0010E94D8D8901B3566
:101A000091D8360E8AD8F5C11BF1D8901B35000E3F
:101A1000D8B0010E87D8D8901B3584D8370E7DD822
:101A2000F2C11BF11B517ED8F3C11BF11B517AD8B7
:101A3000200E73D8000E76D8F2C11BF11B5172D85C
:101A4000210E6BD8F4C11BF1D8901B35000ED8B015
:101A5000010E68D8D8901B3565D8220E5ED8F2C129
:101A60001BF1F3C11CF11B511C5F1C2BF4C11BF1BA
:101A7000F5C11DF11B511D5F1D2B84801DC11BF184
:101A80007AC083FF809480847BC083FF80948084AD
:101A90007AC083FF809480847BC083FF809480849D
:101AA0001B2FEED71C2FEAD7000E37D855EC18F0B5
:101AB0001200350E32D8000E35D8000E33D8360E4F
:101AC0002CD8010E2FD83F0E2DD8370E26D8000E59
:101AD00029D8EF0E27D8200E20D8000E23D8000ECC
:101AE00021D8210E1AD8000E1DD8000E1BD8220EA8
:101AF00014D88480836A0A0E1D6F1E0E1C6F1B6B28
:101B000080948084809480841B2FFAD71C2FF7D771
:101B10001D2FF3D7000E01D812008490836E80949D
:101B2000808412008480836E80948084120080966A
:101B3000200E06EC0BF081840000809A0000848265
:101B4000FA0E06EC0BF0848400008492020EDAECAC
:101B50000AF084820A0E06EC0BF0240EDEDF020E81
:101B6000DCDF000EDFDF000EDDDF030ED6DF000E50
:101B7000D9DF300ED7DF180ED0DF000ED3DF280EEE
:101B8000D1DFF80ECADF000ECDDF0F0ECBDFF90E6E
:101B9000C4DF000EC7DF0F0EC5DF100EBEDF000E64
:101BA000C1DF000EBFDF0CD884DF8086200E06EC7C
:101BB0000BF0050EB2DF000EB5DF010EB3DF120031
:101BC000700EABDF1F0EAEDF000EACDF710EA5DFB7
:101BD000230EA8DF800EA6DF720E9FDF2A0EA2DF83
:101BE000800EA0DF730E99DF150E9CDF110E9ADFB9
:101BF000740E93DF1C0E96DF110E94DF750E8DDFD1
:101C00001B0E90DF150E8EDF760E87DF1A0E8ADF31
:101C1000150E88DF770E81DF1C0E84DF180E82DF41
:101C2000780E7BDF210E7EDF150E7CDF1200700E3A
:101C300074DF140E77DF000E75DF710E6EDF170E86
:101C400071DF000E6FDF720E68DF150E6BDF800E26
:101C500069DF730E62DF150E65DF110E63DF740E30
:101C60005CDF140E5FDF0B0E5DDF750E56DF1B0EA3
:101C700059DF150E57DF760E50DF130E53DF0E0EB1
:101C800051DF770E4ADF1C0E4DDF180E4BDF780E4A
:101C900044DF150E47DF0E0E45DF12002D6F2DC1FC
:101CA0002EF1030E2E17000E2E4F500E2E4FA00EAB
:101CB0002E4FF80E2F6F2DC12EF11C0E2E172E4316
:101CC0002E43000E2E4F040E2E4F080E2E4F0C0EDC
:101CD0002E4F100E2E4F140E2E4F200E2E4F3F0E55
:101CE000306F30332F3330332F3330332F332DC118
:101CF0002EF12D6B30332D3330332D3330332D33E4
:101D0000E00E2E172E432E432E432E432E43000E5D
:101D10002E4F040E2E4F080E2E4F0C0E2E4F100E6F
:101D20002E4F140E2E4F200E2E4F3F0E306F30339D
:101D30002D3330332D3330332D3330332D33303397
:101D40002D332DC17AF02FC17BF01200E26F1F0EF0
:101D5000E26505D0010EAA6E200EE25F01D0AA6AEC
:101D6000E251040DF350820FA96EF9EC0BF0A8506C
:101D7000AA6A1200E26F1F0EE26505D0010EAA6E7C
:101D8000200EE25F01D0AA6AE251040DF350820FE7
:101D9000A96EF9EC0BF0A8CF31F1A92AF9EC0BF000
:101DA000A8CF32F1AA6A12009A0EE16F298D03D0F2
:101DB000240EE16F299D1E8F59EC0DF0010EB96FB5
:101DC000209920971F99A96BA46B219D219FE6EC78
:101DD00029F0010EE8CF7FF029AD04D0BA0E90ECC7
:101DE00009F003D01B0E90EC09F0000EE8CF7FF055
:101DF00055EC18F0010E29AD000EAA6EB76B2091BC
:101E00002093140EE8CF7DF0230EE8CF7CF020EE77
:101E100060F0A9C131F1000E29BD200E312731C17A
:101E2000DAF1376B372B366B47EC0BF03A0EDE6E80
:101E3000200EDE6E4EEC0CF0E151A92590EC09F07D
:101E40001F0EDA5DD8B415D0260EDA5DD8B411D0E5
:101E5000270EDA5DD8B40DD0280EDA5DD8B409D0DB
:101E6000290EDA5DD8B405D02A0EDA5DD8B401D0D7
:101E700003D0010EDA6F01D0DA6B140EE8CF7DF0DB
:101E8000410EE8CF7CF020EE60F02B0EDE6E2F0EC0
:101E9000DE6E2D0EDE6E3A0EDE6E200EDE6E2B0E28
:101EA00021BD2D0EDE6E4EEC0CF0140EE8CF7DF051
:101EB0005F0EE8CF7CF020EE60F0310EDE6E2F0E6C
:101EC000DE6E310EDE6E300EDE6E3A0EDE6E200EEF
:101ED000DE6E310EDE6E300E21BFDE6E200EDE6E47
:101EE0004EEC0CF0140EE8CF7DF07D0EE8CF7CF0C8
:101EF00020EE60F0590E89EC09F0A451800FA96E14
:101F0000F9EC0BF0A8CF31F1A451810FA96EF9ECD7
:101F10000BF0A8CF32F1329F376B372B366B36512F
:101F200055EC0BF02C0EDE6E310EA8AE380EDA67D3
:101F3000310EDE6E350EA8BEDE6E420EDE6E200E57
:101F4000DE6E200EDE6E200EDE6E4EEC0CF0140EF9
:101F5000E8CF7DF09B0EE8CF7CF020EE60F0610EC4
:101F600089EC09F0A451820FA96EF9EC0BF0A8CF0F
:101F700031F1A451830FA96EF9EC0BF0A8CF32F127
:101F8000376B372B366B365155EC0BF0200EDE6E6F
:101F9000200EDE6E200EDE6E4EEC0CF00B0E90EC82
:101FA00009F024EC11F0FCEC1BF006EC30F020B34F
:101FB0000FD020B11AD01FB3BEEF48F01FB125ECEF
:101FC0003CF01FB108EC42F01F911FB91CD0EDD7B7
:101FD000B92B070EB96302D0010EB96FB76BFCECD9
:101FE0001BF024EC11F02093E0D7AA6A010E29BD62
:101FF000AA6EB94F0FD0B94F17D0B94F19D0B94FFA
:102000001BD0B94F39D0020E29AD010EB96FAA6AA3
:10201000C0EF11F0A92BA9BBA96BA951040DF3CFF7
:10202000A4F1010EB96FE4D6217D020EB96FE0D69E
:10203000217F030EB96FDCD6A451800FA96EF9EC95
:102040000BF0A8CF31F1A451810FA96EF9EC0BF080
:10205000A8CF32F1329FA451820FA96E31C1A8FFDF
:10206000FDEC0BF0A451830FA96E32C1A8FFFDEC6B
:102070000BF0040EB96FBCD6A451820FA96EF9EC17
:102080000BF0A8CF31F1A451830FA96EF9EC0BF03E
:10209000A8CF32F1A451810FA96EF9EC0BF0A8CFB3
:1020A000A5F1010EDA6305D031673169312B326B4E
:1020B00016D021AD0BD0010E21BF0A0E315F000EEC
:1020C000A5BF325B7F0E32BF326F09D0010E21BF38
:1020D0000A0E3127000EA5BF322332BF326BA45146
:1020E000820FA96E31C1A8FFFDEC0BF0A451830F44
:1020F000A96E32C1A8FFFDEC0BF0050EB96F78D6C2
:10210000E26F1F0EE26505D0010EAA6E200EE25F9F
:1021100001D0AA6AE251040DF350800FA96EF9ECC8
:102120000BF0A8CF31F1A92AF9EC0BF0A8CF32F1CE
:10213000AA6A1200CE4F14D0CE4F19D01200CE4F43
:102140000FD0CE4F14D0CE4F19D0CE4F1ED0CE4F81
:1021500023D0CE4F28D0CE4F2FD0CE4F34D0120028
:102160000B0E3DD8EAEC10F0020ECE6F12000C0EF2
:1021700049D8EAEC10F0030ECE6F1200110E2FD8E2
:10218000EAEC10F0040ECE6F1200120E3BD8EAEC0F
:1021900010F0050ECE6F1200130E34D8EAEC10F0DA
:1021A000060ECE6F1200060ECE6F1D0E3ED8EAEC64
:1021B00010F0070ECE6F1200200E24D8EAEC10F0BB
:1021C000080ECE6F1200210E1DD8EAEC10F0010EA1
:1021D000CE6F1200316F3167120050EF27F0386F69
:1021E000BAEC0EF031C151F132C152F1385180ECEC
:1021F00010F031C153F132C154F105EC0AF01EA7C1
:10220000FF0C000C386FBAEC0EF031C153F132C143
:1022100054F1385180EC10F031C151F132C152F11A
:1022200005EC0AF01EA7FF0C000C386FBAEC0EF09C
:1022300031C153F132C154F1CEC151F1526B05ECB1
:102240000AF01EA7FF0C000C2397239912002A976F
:102250008196010EB96F1E9F59EC0DF0B76B1F9957
:10226000209120931F8F20878CEC1CF0FCEC1BF03E
:102270002397239955EC11F020B124D01FAFBEEF66
:1022800048F01FB125EC3CF01FB108EC42F01FB143
:102290005BEC3BF01FB189EC46F01F911FB9BEEF1C
:1022A00048F01FB3BEEF48F0E5D723A908D020833C
:1022B000B92B060EB96518D0010EB96F15D023B72A
:1022C00020811200B94FE4EF2CF0B94F9DEF33F0AD
:1022D000B94F27EF13F0B94FBDEF11F0B94F7AEFB7
:1022E00011F0B94FBEEF48F0B76B20B7FCEC1BF014
:1022F00023991200010EB96F1E9F59EC0DF0B76BB8
:102300001F99209120931F8F2087E0EC1CF0FCEC9C
:102310001BF02397239955EC11F0050EB96304D0F7
:10232000060EB96FFCEC1BF020B115D01FAF8FD794
:102330001FB125EC3CF01FB108EC42F01FB15BEC83
:102340003BF01FB189EC46F01F911FB980D71FB336
:10235000BEEF48F0E0D7B94FCDEF14F0B94F5DEFC5
:1023600031F0B94F7FEF32F0B94FC9EF49F0B94FB3
:10237000C9EF49F0050EB96F6ED72A97010EB96FF4
:102380001E9F59EC0DF0AAEC1CF0B76B1F99209121
:1023900020931F8F20870AEC12F0B6EC12F0FCECB1
:1023A0001BF02397239955EC11F020B117D01FAFE4
:1023B000BEEF48F01FB125EC3CF01FB108EC42F035
:1023C0001FB15BEC3BF01FB189EC46F01F911FB9C8
:1023D000BEEF48F01FB3BEEF48F0E5D7B94FD8EFD6
:1023E0000EF0B94FD4EF0EF0B94FACD0B94F03D0C7
:1023F000B94F5CD036D02A87220ED0EC0BF0A82A39
:10240000060EA86201D0A86AFDEC0BF0040EB96FAD
:102410002399BBD7220ED0EC0BF0A86604D0650E32
:1024200090EC09F01200A82E04D0660E90EC09F092
:102430001200A82E04D0680E90EC09F01200A82E0D
:1024400004D08A0E90EC09F01200A82E04D0980E49
:1024500090EC09F01200A82E1200EC0E90EC09F09E
:1024600012002AA7BEEF48F059EC0DF0E6EC29F077
:10247000010EE8CF7FF0EB0E90EC09F0000EE8CFF4
:102480007FF0220ED0EC0BF0070EA802F350C10F24
:10249000B96F070E386FB95190EC09F0B92B382F8E
:1024A000FAD71E0E72EC49F0BEEF48F0010EB96F7C
:1024B0001E9F59EC0DF0C8EC1CF0B76B1F992091D2
:1024C00020931F8F208718EC13F0F2EC12F0FCEC35
:1024D0001BF02397239955EC11F0040EB96304D037
:1024E000060EB96FFCEC1BF020B117D01FAFBEEF8A
:1024F00048F01FB125EC3CF01FB108EC42F01FB1D1
:102500005BEC3BF01FB189EC46F01F911FB9BDEFAA
:1025100011F01FB3BEEF48F0DED7B94F54D0B94F1A
:1025200074D0B94F07D0B94F28D7B94F26D7050E69
:10253000B96F26D752EC49F06DEC49F0030EB96F34
:102540002399B6D71A0ED0EC0BF0A82A630EA86414
:102550000AD0690EA86007D01A0ECEEC0BF0030E5D
:10256000B96F239912D7640EA86EF6D71A0ED0EC65
:102570000BF0630EA86421D8690EA8601ED85F0E08
:10258000E8CF7CF0530EE8CF7DF0000EE8CF7EF070
:1025900020EE60F0A8CF31F1326B1E8F030E55ECA8
:1025A0000BF01E9F6B0EDE6E670EDE6E2F0EDE6E64
:1025B0006C0EDE6E4EEC0CF01200640EA86E1A0E5D
:1025C000CEEC0BF012005B0ED0EC0BF0A82A020E42
:1025D000A86401D0A86A5B0ECEEC0BF0010EB96FB7
:1025E00023996BD75B0ED0EC0BF0A86604D0030EDA
:1025F0008DEC09F01200A82E04D0040E8DEC09F029
:102600001200050E8DEC09F01200270ED0EC0BF035
:10261000A82A010EA86401D0A86A270ECEEC0BF000
:102620002985010EA8622995020EB96F239945D715
:10263000270ED0EC0BF0A86603D0830E90EC09F0C7
:10264000A806A866F6D6820E90EC09F01200010EDC
:10265000B96F59EC0DF0FBEC1CF0B76B1F99209192
:1026600020931F8F2087FBEC1CF0FCEC1BF02397C2
:10267000239955EC11F020B116D01FAFE8D51FB14A
:1026800025EC3CF01FB108EC42F01FB15BEC3BF0D5
:102690001FB189EC46F01F911FB927EF11F01FB34E
:1026A000BEEF48F0E6D7B94F08D0B94F3AD0B94F8E
:1026B00016D0B94F05D0B94F20D0030EB96FCBD586
:1026C0006AEC20F0B96FB96701D0F7D7A9EC0CF02C
:1026D000000E9B6E7E0ED36EFF0000EF00F06AECE2
:1026E00020F0B96FB96701D0E8D759EC0DF0190E99
:1026F00090EC09F0A6EC14F0E0D76AEC20F0B96F8A
:10270000B96701D0DAD759EC0DF0190E90EC09F049
:102710008CC100F58DC101F520EC80F00101BEEF08
:1027200048F06AEC20F0B96FB96701D0C6D759EC10
:102730000DF0190E90EC09F08CC100F58DC101F57A
:1027400020EC80F00101AA6A030EA96E326B150E0F
:10275000E5D8150EE3D8150EE1D8150EDFD8150E05
:10276000DDD8150EDBD8010EA86E210ECEEC0BF0D5
:10277000A86A220ECEEC0BF0A86A230ECEEC0BF06A
:10278000000EA86A270ECEEC0BF0A86A5A0ECEEC0B
:102790000BF0A86A5B0ECEEC0BF0640E1A0ECEECBA
:1027A0000BF01F0EA86E1B0ECEEC0BF0A86A1C0ED1
:1027B000CEEC0BF0A86A1D0ECEEC0BF0A86A1E0E34
:1027C000CEEC0BF0A86A1F0ECEEC0BF0A86A200E20
:1027D000CEEC0BF0640EA86E240ECEEC0BF0250EA2
:1027E000CEEC0BF0260ECEEC0BF0010ECB6FCC6BCB
:1027F0007F0EA96E326B640E91D81E0E8FD8F00E2C
:102800008DD8780E8BD8050E89D8070E87D8040E80
:10281000326F328F880E82D8040E326F328F4C0E98
:102820007DD8140E7BD8140E79D81E0E77D86E0E74
:1028300075D85A0E73D83C0E71D8640E6FD80A0E34
:102840006DD80A0E6BD8130E69D8A00E67D8960EF5
:1028500065D80A0E63D8060E61D8060E5FD8000E42
:102860005DD8000E5BD8000E59D8000E57D8140E54
:1028700055D8326B328F000E51D8030E4FD80A0E46
:102880004DD8000E4BD8010EAA6E7F0EA96E326B8A
:102890001E0E44D85A0E42D8C70E40D8FF0E3ED85E
:1028A0003E0E3CD8E00E3AD8000E38D8000E36D88E
:1028B000000E34D8000E32D8000E30D8320E326FEF
:1028C000328FC80E2BD8650E29D8650E27D8A10ED9
:1028D00025D80F0E23D82A0E21D8000E1FD8000E9F
:1028E0001DD8000E1BD8000E19D8000E17D8000EE8
:1028F00015D8000E13D8000E11D8000E0FD8000EF8
:102900000DD8000E0BD8000E09D8000E07D8000E07
:1029100005D8000E03D8AA6ABEEF48F0316FA92A85
:1029200031C1A8FFFDEC0BF0A92A32C1A8FFFDECD4
:102930000BF0A92A31C1A8FFFDEC0BF0A92A329FA8
:1029400032C1A8FFFDEC0BF0326B1200BC6BBD6B0B
:10295000020E356F366B400E396F22933A693A5149
:1029600002EC2CF0392FFAD7C584B7EC2CF0070E07
:1029700006EC0BF0362FEFD7352FECD72293BC6B3C
:10298000BD6BFD0EF6EC2BF0FD0EF6EC2BF0FE0E03
:10299000F6EC2BF0BC6BBD6B120059EC0DF02095E2
:1029A00020992097B76B209120931F992191219313
:1029B0002195BA6BE6EC29F0010EE8CF7FF01D0EF1
:1029C00090EC09F0000EE8CF7FF0160E90EC09F0C5
:1029D000170E90EC09F007EC15F0180E90EC09F0CA
:1029E0002397239923B7CCEC15F023B998EC15F075
:1029F00020B942D01FB125EC3CF01FB108EC42F0E9
:102A00001F911FB991D01FB3BEEF48F0EBD7460E10
:102A1000E8CF7DF0410EE8CF7CF020EE60F005C1FC
:102A200031F1376B372B366B47EC0BF03A0EDE6E1D
:102A300004C131F1376B372B366B47EC0BF0200EAE
:102A4000DE6E200EDE6E4EEC0CF0460EE8CF7DF012
:102A50005F0EE8CF7CF020EE60F007C1EEF106C11A
:102A6000EFF108C1F0F1D4EC22F0200EDE6E200E62
:102A7000DE6E4EEC0CF0120007C131F1314F1F0E2B
:102A8000314F1C0E314F1F0E314F1E0E314F1F0E96
:102A9000314F1E0E314F1F0E314F1F0E314F1E0E84
:102AA000314F1F0E314F1E0E314F1F0E066502D0E3
:102AB000010E066F200EE8CF7DF09B0EE8CF7CF074
:102AC000080E386F4AEC1BF0050E0A6F036B1F915E
:102AD0001FA1FED71F9125EC15F0460EE8CF7DF023
:102AE000410EE8CF7CF020EE60F005C131F1376B8C
:102AF000372B366B47EC0BF03A0EDE6E04C131F12A
:102B0000376B372B366B47EC0BF03A0EDE6E03C19A
:102B100031F1376B372B366B47EC0BF0200EDE6E46
:102B20004EEC0CF00A2FD4D7010EB96F7CEF11F0E8
:102B300021B12089BA2BBAC1BBF1BB4F2085BB4F55
:102B40002185BB4F2183BB4F2181200EE8CF7DF033
:102B50009B0EE8CF7CF020EE60F05E0E89EC09F071
:102B6000BAC1BBF1BB2F04D05A0E89EC09F00FD0CB
:102B7000BB2F04D05B0E89EC09F009D0BB2F04D029
:102B80005C0E89EC09F003D05D0E89EC09F04EEC87
:102B90000CF024EC11F012002399036B21B120D02A
:102BA00021B310D021B515D020B506D0052B170EB6
:102BB00005651CD0056B1AD0042B3B0E046516D09E
:102BC000046B14D0062B1F0E066510D0010E066F85
:102BD0000DD0072B0C0E076509D0010E076F06D02C
:102BE000082B140E086502D00A0E086F07EC15F0CA
:102BF00024EC11F012007B6B080E7A6F6BC17CF134
:102C00006CC17DF1BDEC0AF0100E7627270E7723FC
:102C100071C180F172C181F176C182F177C183F116
:102C2000A6EC0AF07EC184F17FC185F129B71ED0E0
:102C3000229584C17AF185C17BF184C17CF185C183
:102C40007DF1BDEC0AF0110E756F96EC0AF084C1AF
:102C500080F185C181F176C182F177C183F1A6EC63
:102C60000AF07EC186F17FC187F117D0228584C129
:102C70007AF185C17BF184C17CF185C17DF1BDEC28
:102C80000AF00F0E756F96EC0AF084517627855185
:102C9000772376C186F177C187F169C180F16AC176
:102CA00081F1FA0E826F836BA6EC0AF07EC17AF195
:102CB0007FC17BF184C17CF185C17DF1BDEC0AF05F
:102CC00076C173F177C174F10C0E756F90EC0AF058
:102CD00073C176F174C177F129A70DD063517627BE
:102CE00064517723100E7627270E772376C188F15B
:102CF00077C189F10FD063C180F164C181F176C1E0
:102D000082F177C183F1A6EC0AF07EC176F17FC132
:102D100077F1E8D765C167F166C168F1C80E67272A
:102D2000000E682367C17AF168C17BF184C17CF130
:102D300085C17DF1BDEC0AF076C173F177C174F104
:102D40000D0E756F90EC0AF073C18AF174C18BF1AE
:102D500061C173F162C174F1010E756F90EC0AF0FC
:102D600073518A2774518B23B80E8A270B0E8B233D
:102D70006FC180F170C181F188C182F189C183F195
:102D8000A6EC0AF07EC17AF17FC17BF18AC17CF1A9
:102D90008BC17DF1BDEC0AF00C0E756F96EC0AF05C
:102DA00029B79EEC0AF0E80E7627030E772376C14A
:102DB0008CF177C18DF124AD04D0C5C18CF1C6C1B1
:102DC0008DF16DC167F16EC168F1640E6727000E69
:102DD000682367C17AF168C17BF186C17CF187C144
:102DE0007DF1BDEC0AF00B0E756F96EC0AF0239D99
:102DF00022B509D0C80E7627000E772376C196F14A
:102E000077C197F11200C80E806F816B76C182F195
:102E100077C183F1A6EC0AF029B7238D7EC196F124
:102E20007FC197F11200C7D8A00E3C6F0C0E576FF0
:102E3000FBD81200D6D856C170F155C16FF11200FF
:102E4000BAD8900EF2D7CDD856C172F155C171F1F2
:102E50001200B1D80D0E576F540E3C6FE5D8C1D893
:102E600056C15AF155C159F10D0E576F580E3C6FAE
:102E7000DBD8B7D856C15CF155C15BF10D0E576F69
:102E8000640E3C6FD1D8ADD856C15EF155C15DF12D
:102E90000D0E576F680E3C6FC7D8A3D856C160F1AE
:102EA00055C15FF15AC162F1D8906233D890623354
:102EB000D890623359C161F1D8805AA1D89061335A
:102EC000D8805AA3D8906133D8805AA5D89061335E
:102ED0005BC163F1D8805CA1D8906333D8805CA3D8
:102EE000D8906333D8805CA5D8906333D8805CA732
:102EF000D8906333D8805CA9D8906333D8805CAB1A
:102F0000D89063335CC164F1D88059A1D890643300
:102F1000D88059A3D8906433D88059A5D890643309
:102F2000D8906433D8906433D89064335EC165F12F
:102F3000D8805DAFD8906537D8805DADD8906537C3
:102F4000666B5EBF66835EBD668160C169F1D880D5
:102F50005FAFD89069376A6B60BF6A815DC16BF102
:102F60006B9D5BB16B8D6B9F5BB36B8F6C6B5BB55C
:102F70006C815BB76C835BB96C855BBB6C876E6B7C
:102F80005FC16DF16D9F229F120080820000808ED4
:102F9000000000000000000000000000809E120001
:102FA00080920000808E0000000000000000000001
:102FB0000000809E1200E9DFF3DFE7DFF1DFE5DFED
:102FC000EFDFE3DFEDDFE1DFEBDFDFDFE9DFDDDFD9
:102FD000E7DFDBDFE5DFE4DFE3DFE2DFE1DFE0DFE8
:102FE0001200080E576F10D83CC156F1080E576FEB
:102FF0000BD83CC155F1808E00000000000000009D
:1030000000000000809E1200808E00000000000082
:10301000000000000000809E80A8D89080B8D88072
:103020003C37572FF1D71200809E8082030E575FE6
:10303000808E000000000000000000000000809E64
:10304000000000000000000000000000808E000072
:1030500000000000000000000000809E0000000052
:103060000000000000000000808E00000000000052
:10307000000000000000809E3CAF80923CBF808238
:10308000D8903C37808E0000000000000000000057
:103090000000809E572FF0D71200240EA6EC0EF0F1
:1030A00007D0250EA6EC0EF003D0230EA6EC0EF0F2
:1030B0002D6F000E2D6301D018D0040E2D6301D0AA
:1030C00014D0080E2D6301D010D0C00E2D6301D096
:1030D0000CD0C40E2D6301D008D0C80E2D6301D0D2
:1030E00004D02D514EEC0EF01200FF0E4EEC0EF0FF
:1030F0001200D96FD94F08D0D94F2DD0D94F39D020
:10310000D94F45D0D94F59D032C134F131C133F103
:103110008FC132F18EC131F1BEEC2BF031C151F1D2
:1031200032C152F12B0EBAEC0EF031C153F132C163
:1031300054F105EC0AF01EA707D055EC18F034C185
:1031400032F133C131F1120051EC18F034C132F1D7
:1031500033C131F1120065C531F12C0EA6EC0EF031
:10316000315DD8B003D055EC18F0120051EC18F0D6
:10317000120032C531F12D0EA6EC0EF0315DD8B043
:1031800003D055EC18F0120051EC18F0120047C1B2
:1031900051F148C152F12E0EA6EC0EF0640DF3CFA2
:1031A00053F1F4CF54F105EC0AF01EA703D055EC0F
:1031B00018F0120051EC18F012001EA708D044C1FC
:1031C00031F12F0EA6EC0EF0315DD8B003D055ECE6
:1031D00018F0120051EC18F01200D96FD7C1D8F1D5
:1031E000D6C1D7F1D5C1D6F1D4C1D5F1D3C1D4F16F
:1031F000D9C1D3F129A51200C80EE8CF7CF0640E26
:10320000E8CF7DF0000EE8CF7EF0000EE8CF7FF033
:1032100055EC18F020EE60F0D351DE6ED451DE6E26
:10322000D551DE6ED651DE6ED751DE6ED851DE6ED0
:10323000200EDE6E4EEC0CF01200819697EC0DF035
:1032400059EC0DF055EC18F0000EE8CF7FF0850E2C
:1032500090EC09F0860E90EC09F0870E90EC09F0E6
:10326000880E90EC09F0640EE8CF7CF00A0EE8CFEF
:103270007DF0000EE8CF7EF0000EE8CF7FF055EC39
:1032800018F020EE60F0D351DE6ED451DE6ED551D1
:10329000DE6ED651DE6ED751DE6ED851DE6E2E0E4A
:1032A000DE6E200EDE6E1EC131F1376B372B366BB2
:1032B0004CEC0BF0200EDE6E1FC131F1376B372B5B
:1032C000366B4CEC0BF04EEC0CF07D0EE8CF7CF046
:1032D0000A0EE8CF7DF0000EE8CF7EF0000EE8CFBA
:1032E0007FF055EC18F020EE60F020C131F1376B23
:1032F000372B366B4CEC0BF0200EDE6E21C131F11A
:10330000376B372B366B4CEC0BF0200EDE6E22C188
:1033100031F1376B372B366B4CEC0BF0200EDE6E39
:1033200023C131F1376B372B366B4CEC0BF0200E91
:10333000DE6E24C131F1376B372B366B4CEC0BF062
:103340004EEC0CF0960EE8CF7CF00A0EE8CF7DF044
:10335000000EE8CF7EF0000EE8CF7FF055EC18F0BD
:1033600020EE60F025C131F1376B372B366B4CEC1A
:103370000BF0200EDE6E26C131F1376B372B366B2A
:103380004CEC0BF0200EDE6E27C131F1376B372B82
:10339000366B4CEC0BF0200EDE6E28C131F1376B32
:1033A000372B366B4CEC0BF0200EDE6E29C131F161
:1033B000376B372B366B4CEC0BF04EEC0CF023A735
:1033C000FED7819812004DEC18F00B0E8DEC09F031
:1033D000560E90EC09F0570E90EC09F055EC18F0F1
:1033E0001200000EE8CFF1F13C0EE8CFF2F1EF0E43
:1033F000E8CFF3F15A0EE8CFF4F19F0EE8CFF5F1E4
:10340000F1EC0CF065EC1DF0D2EC1DF01200E9DFE0
:103410004DEC18F0540E90EC09F055EC18F0080E35
:10342000386F910EE8CF7CF0000EE8CF7DF04AECCB
:103430001BF012002AB512007A0EEDEC18F0B90E4E
:10344000E8CF7CF0770EE8CF7DF0010EE8CF7EF07C
:10345000000EE8CF7FF055EC18F020EE60F022C5AA
:1034600031F1376B372B366B4CEC0BF0270EDE6EE1
:103470004EEC0CF0000EE8CF7EF01200B2DF4DEC07
:1034800018F0550E90EC09F055EC18F012002AB522
:1034900012001FBF31D0790EEDEC18F04DEC18F092
:1034A000520E90EC09F055EC18F0760EE8CF7CF057
:1034B0005E0EE8CF7DF0010EE8CF7EF0000EE8CF83
:1034C0007FF055EC18F020EE60F02BC531F1376B32
:1034D000372B366B36EC0BF06D0EDE6E24C531F1FA
:1034E000376B372B366B36EC0BF0270EDE6E4EEC5F
:1034F0000CF0000EE8CF7EF02AB51200780EEDEC4D
:1035000018F0B90EE8CF7CF0770EE8CF7DF0010E11
:10351000E8CF7EF0000EE8CF7FF055EC18F020EEFB
:1035200060F031C531F1C70E3161316F1E9F376BCD
:10353000372B366B4CEC0BF0270EDE6E4EEC0CF09E
:1035400032C531F1080EA6EC0EF0316101D067D71B
:10355000770EEDEC18F0910EE8CF7CF0000EE8CF7E
:103560007DF0000EE8CF7EF0030E79EC18F020EE2F
:1035700060F0470EDE6E460EDE6E3A0EDE6E32C52F
:1035800031F1376B372B366B4CEC0BF0250EDE6EC2
:10359000200EDE6E4EEC0CF055EC18F01200410ED1
:1035A000E8CF7CF0690EE8CF7DF0000EE8CF7EF02A
:1035B00055EC18F020EE60F0E8C131F11E8F376B4A
:1035C000372B366B4CEC0BF01E9F6D0EDE6E690ECA
:1035D000DE6E6E0EDE6E200EDE6E4EEC0CF05F0EBA
:1035E000E8CF7CF0640EE8CF7DF0000EE8CF7EF0EF
:1035F00055EC18F020EE60F0E9C131F11E8F376B09
:10360000372B366B4CEC0BF01E9F6D0EDE6E200ED2
:10361000DE6E4EEC0CF012002AB51200760EEDECC8
:1036200018F05A0EE8CF7CF0000EE8CF7DF0000EC7
:10363000E8CF7EF0050E79EC18F020EE60F02D0E4C
:103640001EB72B0EDE6E44C131F1376B372B366B54
:1036500036EC0BF0530E89EC09F04EEC0CF055EC07
:1036600018F02A891200080E386F5A0EE8CF7CF045
:10367000000EE8CF7DF02A990DD0060E386F020EAD
:10368000E8CF7CF0730EE8CF7DF004D0010EE8CFD8
:103690007EF003D0000EE8CF7EF020EE60F0200E2A
:1036A000DE6E382FFCD74EEC0CF0000EE8CF7EF02B
:1036B0001200270EA6EC0EF0316F010E31631200DE
:1036C0001FBF1200020EE8CF7CF0400EE8CF7DF065
:1036D000000EE8CF7EF0000EE8CF7FF055EC18F03A
:1036E00020EE60F005C131F1376B372B366B47ECBC
:1036F0000BF03A0EDE6E04C131F1376B372B366BAF
:1037000047EC0BF04EEC0CF01200630EEDEC18F0F1
:10371000320EE8CF7CF0010EE8CF7DF0000EE8CF4E
:103720007EF0000EE8CF7FF055EC18F020EE60F050
:1037300019C131F1316705D01AC131F1316701D0BA
:1037400039D02CAF34D0B62F01D034D02C8F060E08
:10375000B66125D819C131F11AC132F1E2EC09F094
:10376000325131C132F1316F490EDE6E6E0EDE6EB6
:10377000740EDE6E3A0EDE6E376B372B366B47EC0F
:103780000BF03A0EDE6E32C131F1376B372B366BF0
:1037900047EC0BF0200EDE6E4EEC0CF012002C9F6E
:1037A000050EB66F12002C8F050EB66F1200B62FE5
:1037B00001D0CCD72C9F060EB661F5DF05C131F1E3
:1037C000376B372B366B47EC0BF03A0EDE6E04C1CD
:1037D00031F1376B372B366B47EC0BF03A0EDE6E60
:1037E00003C131F1376B372B366B47EC0BF0200EF2
:1037F000DE6E4EEC0CF01200230EE8CF7CF0000ED3
:10380000E8CF7DF0000EE8CF7EF0000EE8CF7FF02D
:1038100055EC18F020EE60F0B80EDE6E4EEC0CF0B9
:10382000410EE8CF7CF0000EE8CF7DF0000EE8CF2F
:103830007EF0000EE8CF7FF020EE60F0B80EDE6E76
:103840004EEC0CF05F0EE8CF7CF0000EE8CF7DF080
:10385000000EE8CF7EF0000EE8CF7FF020EE60F0A3
:10386000B80EDE6E4EEC0CF07D0EE8CF7CF0000E54
:10387000E8CF7DF0000EE8CF7EF0000EE8CF7FF0BD
:1038800020EE60F0B80EDE6E4EEC0CF09B0EE8CF32
:103890007CF0000EE8CF7DF0000EE8CF7EF0000E49
:1038A000E8CF7FF055EC18F020EE60F0B80EDE6E39
:1038B0004EEC0CF0B90EE8CF7CF0000EE8CF7DF0B6
:1038C000000EE8CF7EF0000EE8CF7FF020EE60F033
:1038D000B80EDE6E4EEC0CF0B9C138F1384F230E45
:1038E000384F410E384F5F0E384F7D0E384F9B0ECC
:1038F000384FB90EE8CF7CF0000EE8CF7DF0000E17
:10390000E8CF7EF0000EE8CF7FF020EE60F0B70E3B
:10391000DE6E4EEC0CF01200E6EC29F0010EE8CF62
:103920007FF0050E90EC09F0000EE8CF7FF0060E58
:1039300090EC09F0070E90EC09F0090E90EC09F0FC
:103940000A0E90EC09F08E0E90EC09F00B0E90EC44
:1039500009F01200E6EC29F0010EE8CF7FF0620ECC
:1039600090EC09F0000EE8CF7FF0630E90EC09F0C8
:10397000990E90EC09F0140E8DEC09F0640E90ECA9
:1039800009F08E0E90EC09F00B0E90EC09F012008D
:10399000E6EC29F0010EE8CF7FF0020E8DEC09F085
:1039A000000EE8CF7FF0010E8DEC09F0810E90EC57
:1039B00009F0BB0E90EC09F00B0E90EC09F0120030
:1039C000E6EC29F0010EE8CF7FF0900E90EC09F0C4
:1039D000000EE8CF7FF0080E90EC09F06E0E90EC30
:1039E00009F0710E90EC09F0F70E90EC09F00B0E57
:1039F00090EC09F01200E6EC29F0010EE8CF7FF020
:103A00001C0E90EC09F0000EE8CF7FF0150E90EC44
:103A100009F0F50E90EC09F01C0E8DEC09F01D0E6E
:103A20008DEC09F01E0E8DEC09F00B0E90EC09F0F8
:103A30001200E6EC29F0010EE8CF7FF0F80E90ECD2
:103A400009F0000EE8CF7FF0F90E90EC09F0150EAA
:103A50008DEC09F0160E8DEC09F0170E8DEC09F0C7
:103A6000180E8DEC09F00B0E90EC09F01200650EAB
:103A7000EDEC18F096C198F197C199F1640EE8CF7A
:103A80007CF0010EE8CF7DF0000EE8CF7EF0000E56
:103A9000E8CF7FF055EC18F020EE60F02D0E23BD3E
:103AA000DE6E96C131F197C132F1030E376F1E8F72
:103AB000020E55EC0BF01E9FB00EDE6E430EDE6E56
:103AC000200EDE6E4EEC0CF012002AB51200750EC0
:103AD000EDEC18F096C198F197C199F1D80EE8CFA6
:103AE0007CF0410EE8CF7DF0000EE8CF7EF0000EB6
:103AF000E8CF7FF055EC18F020EE60F02D0E23BDDE
:103B0000DE6E96C131F197C132F1030E376F1E8F11
:103B1000020E55EC0BF01E9FB00EDE6E200EDE6E18
:103B20004EEC0CF01200740EEDEC18F0780EE8CFAD
:103B30007CF0000EE8CF7DF0000EE8CF7EF0040EA2
:103B400079EC18F020EE60F0700EDE6E700EDE6E16
:103B50004F0EDE6E320EDE6E3A0EDE6E47C131F172
:103B600048C132F12887010E55EC0BF02897200E42
:103B7000DE6E4EEC0CF055EC18F012000A0E386FA9
:103B8000780EE8CF7CF0000EE8CF7DF04AEC1BF019
:103B90001200C00EE8CF7CF0410EE8CF7DF0050E9C
:103BA000386F78D529BB12002AB51200000EE8CF75
:103BB0007FF0F0EC1DF02BAD12002A0EA6EC0EF0FB
:103BC000316F010E316312002C772CA71200010E09
:103BD000E8CF7FF0F0EC1DF0000EE8CF7FF0120090
:103BE000730EEDEC18F0C00EE8CF7CF0410EE8CF7C
:103BF0007DF0000EE8CF7EF055EC18F0640E10C595
:103C000031F1D880315511C531F1D8803157090EC5
:103C1000A6EC0EF011C532F1316501D005D0326746
:103C200003D0050E386F36D5150E31630ED03267CE
:103C30000CD020EE60F0080E86EC09F0200E2BBDB3
:103C40002A0EDE6E4EEC0CF0120020EE60F01E8F9D
:103C5000376B372B366B4CEC0BF02F0EDE6E11C52D
:103C600031F1376B372B366B4CEC0BF0200E2BBD44
:103C70002A0EDE6E1E9F4EEC0CF01200550EE8CFA1
:103C80007DF0000EE8CF7EF0000EE8CF7FF0AA6A4C
:103C9000220ED0EC0BF0A86620D07D0EE8CF7CF091
:103CA00055EC18F020EE60F04F0EDE6E4EEC0CF08E
:103CB000550EE8CF7DF0000EE8CF7EF0000EE8CF85
:103CC0007FF0960EE8CF7CF055EC18F020EE60F017
:103CD000430EDE6E4EEC0CF01200A806A86601D072
:103CE0001200A806A86629D07D0EE8CF7CF055EC1E
:103CF00018F020EE60F0430EDE6E550EE8CF7DF03A
:103D0000000EE8CF7EF0000EE8CF7FF04EEC0CF016
:103D1000960EE8CF7CF055EC18F020EE60F0430EE4
:103D2000DE6E550EE8CF7DF0000EE8CF7EF0000E7F
:103D3000E8CF7FF04EEC0CF01200A806A86601D088
:103D40001200A806A86629D07D0EE8CF7CF020EEF0
:103D500060F0470EDE6E550EE8CF7DF0000EE8CF26
:103D60007EF0000EE8CF7FF055EC18F04EEC0CF032
:103D7000960EE8CF7CF020EE60F0460EDE6E550E1B
:103D8000E8CF7DF0000EE8CF7EF0000EE8CF7FF0A8
:103D900055EC18F04EEC0CF012007D0EE8CF7CF0E4
:103DA00020EE60F0470EDE6E550EE8CF7DF0000E7F
:103DB000E8CF7EF0000EE8CF7FF055EC18F04EEC27
:103DC0000CF0960EE8CF7CF020EE60F0460EDE6E32
:103DD000550EE8CF7DF0000EE8CF7EF0000EE8CF64
:103DE0007FF055EC18F04EEC0CF01200000EE8CF0E
:103DF000F1F1190EE8CFF2F1780EE8CFF3F1520E9F
:103E0000E8CFF4F19F0EE8CFF5F1F1EC0CF028B11A
:103E10005ED06D0EEDEC18F05A0EE8CF7DF0000E7E
:103E2000E8CF7EF01E8F020E0A6F000E096F326B14
:103E3000322B040E0A2720EE60F0470EDE6E32C1F0
:103E400031F1376B372B366B4CEC0BF03A0EDE6EE4
:103E5000200EDE6E0AC1A9FFF9EC0BF0A8CF31F1FC
:103E6000376B372B366B4CEC0BF02F0EDE6EA92A1E
:103E7000F9EC0BF0A8CF31F1376B372B366B4CECEC
:103E80000BF01B0ED0EC0BF032C131F1A832312F08
:103E9000FDD7D8B004D04A0E4EEC0EF002D055EC4F
:103EA00018F0210ED0EC0BF0A850326301D009D0ED
:103EB000190E09275A0EE8CF7DF009C17CF04EECAF
:103EC0000CF055EC18F0050E3263B2D712005A0E02
:103ED000E8CF7DF0000EE8CF7EF01E8F230E0A6F34
:103EE000000E096FE46B0A2BE42B190E09275A0EFA
:103EF000E8CF7DF009C17CF020EE60F0530EDE6E5D
:103F0000500EDE6EE4C131F1376B372B366B4CEC63
:103F10000BF03A0EDE6E200EDE6E0AC1A9FFF9EC40
:103F20000BF0A8CF31F1326B030E55EC0BF04EECD9
:103F30000CF0030EE463D7D7210ED0EC0BF0A8CF22
:103F4000D0F1D005040DF350070FA96EF9EC0BF07A
:103F5000A8CF32F1D005040DF350060FA96EF9EC8D
:103F60000BF0A8CF31F15A0EE8CF7DF0640EE8CF08
:103F70007CF020EE60F0440EDE6E690EDE6E6C0E9C
:103F8000DE6E3A0EDE6E376B372B366B4CEC0BF079
:103F90002F0EDE6E32C131F1376B372B366B4CECA6
:103FA0000BF04EEC0CF01E9F1200710EEDEC18F0B1
:103FB00029BB120027BF120028A123D0870EE8CF0B
:103FC0007CF05A0EE8CF7DF0000EE8CF7EF0000EB8
:103FD000E8CF7FF055EC18F020EE60F0240ED0EC26
:103FE0000BF0A8CF31F1326B030E55EC0BF0420E03
:103FF000DE6E610EDE6E720EDE6E1E9F4EEC0CF0FB
:1040000057D0820EE8CF7CF0640EE8CF7DF0010E31
:10401000E8CF7EF0000EE8CF7FF055EC18F0210ECF
:10402000D0EC0BF0A8CFD0F1D005040DF350070F62
:10403000A96EF9EC0BF0A8CF11F5D005040DF350E3
:10404000060FA96EF9EC0BF0A8CFCFF111C50AF15C
:10405000D880640E0A55D880A856A8CF10F5640EF3
:1040600010C531F1D880315511C531F1D8803157A3
:1040700011C532F1150E316306D0326704D0090E36
:104080008DEC09F015D020EE60F01E8F376B372BCA
:10409000366B4CEC0BF02F0EDE6E11C531F1376B29
:1040A000372B366B4CEC0BF01E9F4EEC0CF000D017
:1040B000000EE8CFF1F17A0EE8CFF2F1AF0EE8CFC3
:1040C000F3F1520EE8CFF4F19F0EE8CFF5F1B1EC29
:1040D0000CF01200000EE8CFF1F1440EE8CFF2F13F
:1040E000920EE8CFF3F1220EE8CFF4F1650EE8CF9F
:1040F000F5F1F1EC0CF0230EA6EC0EF0E8CFF1F1A7
:10410000460EE8CFF2F1900EE8CFF3F1230EE8CFA0
:10411000F4F1640EE8CFF5F1B1EC0CF08F0E90ECF9
:1041200009F0910E90EC09F0920E90EC09F0010E5E
:10413000B96F000EE8CFF1F1600EE8CFF2F18F0E0B
:10414000E8CFF3F1270EE8CFF4F1330EE8CFF5F125
:10415000F1EC0CF0B9C138F1600E384F600E384FF9
:10416000780EE8CF7CF0270EE8CF7DF0000EE8CF88
:104170007EF0000EE8CF7FF055EC18F020EE60F0F6
:10418000B70EDE6E4EEC0CF01F9920912093239910
:104190002397B76B640E06EC0BF006EC30F020B3FF
:1041A00015D020B10ED01FB125EC3CF01FB108ECAA
:1041B00042F01F911FB903D01FB301D0EED7000CFE
:1041C000010CB94FFCD7B94FFBD7F9D7B92B030E68
:1041D000B96302D0010EB96FACD7720EEDEC18F0D6
:1041E0008FC132F18EC131F1BEEC2BF0270E32615E
:1041F00071D02ABB91EC21F02A9B20EE60F0030ED7
:10420000526FE80E516F32C154F131C153F1532B4B
:10421000000E542305EC0AF01EA780D8180EE8CF34
:104220007CF0000EE8CF7DF0020EE8CF7EF0000EAD
:10423000E8CF7FF0010E79EC18F0000E526F630E9C
:10424000516F32C154F131C153F105EC0AF01EA790
:104250000AD01E8F2887376B372B366B365155ECBB
:104260000BF01E9F02D0300EDE6E4EEC0CF0289745
:10427000010EE8CF7EF0320EE8CF7CF0280EE8CFBA
:104280007DF0010E79EC18F08FC132F18EC131F161
:10429000BEEC2BF020EE60F02E0EDE6E000E526FA4
:1042A000090E516F32C154F131C153F105EC0AF0DE
:1042B0001EA707D0040E376F2385000E55EC0BF0B8
:1042C00002D0300EDE6E4EEC0CF02395000EE8CFDF
:1042D0007EF012002AAB91EC21F020EE60F0180E77
:1042E000E8CF7CF0000EE8CF7DF0020EE8CF7EF044
:1042F000000EE8CF7FF0010E79EC18F028871E8FB2
:10430000376B372B366B365155EC0BF01E9F4EEC4E
:104310000CF02897000EE8CF7EF01200200EDE6E23
:104320001200000EE8CFF1F1180EE8CFF2F15A0EAC
:10433000E8CFF3F1000EE8CFF4F15A0EE8CFF5F133
:10434000F1EC0CF02A8B1200680EEDEC18F0960ED2
:10435000E8CF7CF0010EE8CF7DF0000EE8CF7EF0D4
:10436000000EE8CF7FF055EC18F020EE60F00E0E56
:1043700089EC09F0200EDE6E20C531F121C532F145
:10438000E2EC09F01E8F315132C131F1326F376BDF
:10439000372B366B4CEC0BF03A0EDE6E32C131F13E
:1043A000376B372B366B47EC0BF01E9F4EEC0CF047
:1043B0001200670EEDEC18F07D0EE8CF7CF0010ED8
:1043C000E8CF7DF0000EE8CF7EF0000EE8CF7FF062
:1043D00055EC18F020EE60F0230E89EC09F0200E69
:1043E000DE6ECBC131F1CCC132F1E2EC09F01E8FAF
:1043F000315132C131F1326F376B372B366B4CECA8
:104400000BF03A0EDE6E32C131F1310731BF316B44
:10441000376B372B366B47EC0BF01E9F4EEC0CF0D6
:1044200012001FBD1200620EEDEC18F0190EE8CF5D
:104430007CF0010EE8CF7DF0000EE8CF7EF0000E9C
:10444000E8CF7FF055EC18F020EE60F08CC131F130
:104450008DC132F11E8F376B372B366B365155ECD1
:104460000BF01E9F6D0EDE6E620EDE6E610EDE6E56
:10447000720EDE6E200EDE6E4EEC0CF01200660E3A
:10448000EDEC18F01F0EA6EC0EF0316F010E31634B
:1044900023D0AF0EE8CF7CF0010EE8CF7DF0000E08
:1044A000E8CF7EF0000EE8CF7FF055EC18F020EE5C
:1044B00060F0C1C131F1C2C132F1010E376F238505
:1044C0001E8F020E55EC0BF01E9F560EDE6E200E58
:1044D000DE6E4EEC0CF01200230EA6EC0EF0E8CFD0
:1044E000F1F1AE0EE8CFF2F1C20EE8CFF3F1010E1A
:1044F000E8CFF4F1200EE8CFF5F1B1EC0CF0040EAA
:10450000516F100E526FC1C153F1C2C154F105EC8D
:104510000AF01EB746D0AC0E536F0D0E546FC1C1DA
:1045200051F1C2C152F105EC0AF01EB737D04FC1AC
:104530004BF150C14CF1140E4D6F4E6B39EC0AF03B
:1045400047C10AF10A2B030E0A650A6F230EA6EC77
:104550000EF0E8CFF1F1B50EE8CFF2F1BB0EE8CFE7
:10456000F3F1200EE8CFF4F1220EE8CFF5F1F1ECF3
:104570000CF0220EA6EC0EF0E8CFF1F1B00EE8CF71
:10458000F2F1C00EE8CFF3F1020EE8CFF4F10AC168
:10459000F5F1F1EC0CF055EC18F01200010E0A6F79
:1045A000D5D71E0E0A6FD2D75B0ED0EC0BF0A866E3
:1045B0000ED0EEC131F11E8F376B372B366B47ECC7
:1045C0000BF01E9F2F0EDE6EEFC131F112D05B0E8D
:1045D000D0EC0BF0A82E1FD0EFC131F11E8F376B3E
:1045E000372B366B47EC0BF01E9F2F0EDE6EEEC1A5
:1045F00031F11E8F376B372B366B47EC0BF01E9F5C
:104600002F0EDE6EF0C131F11E8F376B372B366BFC
:1046100047EC0BF01200F0C131F11E8F376B372BD6
:10462000366B47EC0BF01E9F2F0EDE6EEEC131F1A4
:104630001E8F376B372B366B47EC0BF01E9F2F0E00
:10464000DE6EEFC131F11E8F376B372B366B47ECC7
:104650000BF012005B0ED0EC0BF0A86615D0EEC18B
:1046600031F11E8F376B372B366B47EC0BF01E9FEB
:104670002F0EDE6EEFC131F11E8F376B372B366B8D
:1046800047EC0BF01E9F12005B0ED0EC0BF0A82E37
:10469000E6D7EFC131F11E8F376B372B366B47EC06
:1046A0000BF01E9F2F0EDE6EEEC131F11E8F376BA9
:1046B000372B366B47EC0BF01E9F1200640EEDECAF
:1046C00018F04B0EE8CF7CF0010EE8CF7DF0000E25
:1046D000E8CF7EF0000EE8CF7FF055EC18F020EE2A
:1046E00060F007C1EEF106C1EFF108C1F0F1D4ECC2
:1046F00022F04EEC0CF01200000EE8CFF1F1000EAB
:10470000E8CFF2F11A0EE8CFF3F1410EE8CFF4F161
:10471000640EE8CFF5F1F1EC0CF012002AB51200AE
:10472000700EEDEC18F0B80EE8CF7CF0000EE8CF7C
:104730007DF0010EE8CF7EF0000EE8CF7FF055EC63
:1047400018F020EE60F090C131F191C132F1BEEC71
:104750002BF01E8F2385030E55EC0BF01E9F1E9D24
:104760004EEC0CF0000EE8CF7EF012001FBF1200DE
:10477000410EEDEC18F027BF92D029BB90D0260E49
:10478000A6EC0EF0316F010E316301D088D0A4C1C8
:1047900031F1A5C132F11E9F20EE60F0376B372B4F
:1047A000366B1E8D365155EC0BF0140EE8CF7CF0B5
:1047B000780EE8CF7DF0010EE8CF7EF055EC18F0D2
:1047C0004EEC0CF0000EE8CF7EF012001FBF12007E
:1047D0004DEC18F08C0E90EC09F055EC18F0550EDD
:1047E000E8CF7CF05A0EE8CF7DF0010EE8CF7EF0E6
:1047F00055EC18F0DFC131F11E9F20EE60F0376BF1
:10480000372B366B4CEC0BF03A0EDE6EE0C131F11B
:10481000376B372B366B47EC0BF04EEC0CF0000E81
:10482000E8CF7EF01200000EE8CFF1F13C0EE8CFA9
:10483000F2F1770EE8CFF3F15A0EE8CFF4F19F0EC4
:10484000E8CFF5F1F1EC0CF012004DEC18F08B0E06
:1048500090EC09F055EC18F0910EE8CF7CF05A0E70
:10486000E8CF7DF0010EE8CF7EF055EC18F0DAC10C
:1048700031F120EE60F0376B372B366B4CEC0BF0E0
:104880003A0EDE6EDBC131F1376B372B366B47ECFE
:104890000BF04EEC0CF0000EE8CF7EF01200A4C13D
:1048A00031F1A5C132F11E9F1E8D20EE60F0376BF5
:1048B000372B366B1E8D365155EC0BF03A0EDE6EF3
:1048C000A6C131F1376B372B366B47EC0BF0140E6A
:1048D000E8CF7CF05A0EE8CF7DF0010EE8CF7EF0F5
:1048E00055EC18F04EEC0CF01E9D000EE8CF7EF05B
:1048F0001200000EE8CFF1F1360EE8CFF2F1660EAD
:10490000E8CFF3F13E0EE8CFF4F19F0EE8CFF5F1DA
:10491000F1EC0CF012001FBF1200560EEDEC18F077
:104920004DEC18F01B0E8DEC09F055EC18F0500E04
:10493000E8CF7CF06E0EE8CF7DF0000EE8CF7EF081
:1049400055EC18F020EE60F017C131F118C132F1CA
:10495000020E315F000E325BE2EC09F031C10AF168
:1049600032C131F1326B000E1E9F1E8D376B372B1B
:10497000366B1E8D365155EC0BF03A0EDE6E0AC1C9
:1049800031F1376B372B366B47EC0BF01E9F4EEC3B
:104990000CF0550EEDEC18F0500EE8CF7CF03E0E0A
:1049A000E8CF7DF0000EE8CF7EF055EC18F020EE59
:1049B00060F092C131F193C132F1BEEC2BF01E8F49
:1049C0002385030E55EC0BF01E9F6D0EDE6E200E40
:1049D000DE6E4EEC0CF01200610EEDEC18F0000EE5
:1049E000E8CF7CF0010EE8CF7DF0000EE8CF7EF03E
:1049F000000EE8CF7FF055EC18F020EE60F0060EC8
:104A000086EC09F0AA6AA96AF9EC0BF0A8CF31F19B
:104A1000A92AF9EC0BF0A8CF32F11E8F376B372B98
:104A2000366B365155EC0BF0200EDE6E560EDE6EF8
:104A3000010E316F1E8F376B372B366B4CEC0BF042
:104A40002E0EDE6E470E316F1E8F376B372B366B97
:104A500047EC0BF01E9F4EEC0CF012006F0EEDECCD
:104A600018F07CEC23F01F0E90EC09F028B107D071
:104A7000200E90EC09F07A0E90EC09F006D0EE0EC4
:104A800090EC09F0890E90EC09F0210E90EC09F001
:104A9000220E90EC09F012006F0EEDEC18F0F00E03
:104AA00090EC09F0F10E90EC09F0190E8DEC09F084
:104AB000930E90EC09F0F40E90EC09F01200640EE5
:104AC000E8CF7DF0000EE8CF7CF0000EE8CF7EF05E
:104AD00055EC18F020EE60F0530EDE6E650EDE6EC3
:104AE0006C0EDE6E180ED0EC0BF0A8CF31F11E9FCD
:104AF000376B372B366B36EC0BF02F0EDE6E190E44
:104B0000D0EC0BF0A8CF31F1376B372B366B36EC8E
:104B10000BF04EEC0CF07B0E90EC09F07C0E90EC60
:104B200009F07D0E90EC09F07E0E90EC09F0120079
:104B3000FE0E90EC09F0FA0E90EC09F0FB0E90ECF2
:104B400009F0FC0E90EC09F0FD0E90EC09F012005B
:104B5000230EA6EC0EF0E8CFF1F17C2B7CC0F2F135
:104B60007CC0F3F1120EF3277A0EE8CFF4F131276F
:104B700031078A0E3161316F31C1F5F1F1EC0CF082
:104B8000000EE8CFF1F17CC0F2F17CC0F3F1120E1F
:104B9000F32731C1F4F1F42B8B0EE8CFF5F1F1ECF2
:104BA0000CF01200000EE8CFF1F132C1F2F17D0EEF
:104BB000E8CFF3F1640EE8CFF4F19F0EE8CFF5F102
:104BC000F1EC0CF012006E0EEDEC18F02BC531F18B
:104BD000316706D0B6EC26F0EF0E90EC09F012002B
:104BE000E469E70EE56F190EE527E42BFCEC25F0F0
:104BF000050EE463F8D712001E8F640EE8CF7DF037
:104C0000E5C17CF0E5C132F115EE2BF0E451E3CFC4
:104C100031F13151D8B4D2EF25F020EE60F0376B8E
:104C2000372B366B4CEC0BF06D0EDE6E4EEC0CF051
:104C30008C0EE8CF7DF0E5C17CF015EE24F0E45158
:104C4000E3CF31F120EE60F0376B372B366B47EC5A
:104C50000BF0270EDE6E4EEC0CF0A8EC25F01200E7
:104C60006D0EEDEC18F0640EE8CF7DF0000EE8CF8D
:104C70007EF01E8F020E0A6FE70E096F326B322B29
:104C8000040E0A27190E0927640EE8CF7DF009C12A
:104C90007CF020EE60F0470EDE6E32C131F1376BF2
:104CA000372B366B4CEC0BF03A0EDE6E0AC1A9FFC7
:104CB000F9EC0BF0A8CF31F1376B372B366B4CEC9E
:104CC0000BF02F0EDE6EA92AF9EC0BF0A8CF31F114
:104CD000376B372B366B4CEC0BF01B0ED0EC0BF01C
:104CE00032C131F1A832312FFDD74A0ED8A04EEC97
:104CF0000EF04EEC0CF055EC18F0050E3263BFD7F9
:104D00001200640EE8CF7DF0000EE8CF7EF01E8F1B
:104D1000230E0A6FE70E096FE46B0A2BE42B190EC2
:104D2000092709C17CF0640EE8CF7DF020EE60F029
:104D3000530EDE6E500EDE6EE4C131F1376B372B51
:104D4000366B4CEC0BF03A0EDE6E0AC1A9FFF9ECA3
:104D50000BF0A8CF31F1326B030E55EC0BF04EEC9B
:104D60000CF0030EE463D9D71E9F1200000EE8CFAB
:104D7000F1F1000EE8CFF2F1B90EE8CFF3F1520EE7
:104D8000E8CFF4F19F0EE8CFF5F1F1EC0CF0120052
:104D90006C0EEDEC18F0000EE8CF7CF0550EE8CF6D
:104DA0007DF0000EE8CF7EF0000EE8CF7FF055ECEE
:104DB00018F020EE60F0B80EDE6E4EEC0CF0190E1E
:104DC000E8CF7CF0550EE8CF7DF0000EE8CF7EF006
:104DD000000EE8CF7FF055EC18F020EE60F0B80E32
:104DE000DE6E4EEC0CF0320EE8CF7CF0550EE8CFC4
:104DF0007DF0000EE8CF7EF0000EE8CF7FF055EC9E
:104E000018F020EE60F0B80EDE6E4EEC0CF04B0E9B
:104E1000E8CF7CF0550EE8CF7DF0000EE8CF7EF0B5
:104E2000000EE8CF7FF055EC18F020EE60F0B80EE1
:104E3000DE6E4EEC0CF0640EE8CF7CF0550EE8CF41
:104E40007DF0000EE8CF7EF0000EE8CF7FF055EC4D
:104E500018F020EE60F0B80EDE6E4EEC0CF0B9C12A
:104E600038F1000E384F000E384F190E384F320E01
:104E7000384F4B0E384F640EE8CF7CF0550EE8CF1C
:104E80007DF0000EE8CF7EF0000EE8CF7FF055EC0D
:104E900018F020EE60F0B70EDE6E4EEC0CF0120053
:104EA000000EE8CFF1F1380EE8CFF2F1580EE8CF5E
:104EB000F3F1450EE8CFF4F1730EE8CFF5F1F1EC24
:104EC0000CF0230EA6EC0EF0E8CFF1F13A0EE8CF8D
:104ED000F2F1560EE8CFF3F1460EE8CFF4F1720E80
:104EE000E8CFF5F1B1EC0CF03C0EE8CF7CF0470ECA
:104EF000E8CF7DF0000EE8CF7EF0010EE8CF7FF026
:104F000051EC18F020EE60F0430EDE6E460EDE6EC1
:104F100038C131F1376B372B366B4CEC0BF0210E6F
:104F2000DE6E4EEC0CF0000EE8CF7FF055EC18F082
:104F30001200680EEDEC18F0690EEDEC18F0000EA2
:104F4000E8CFF1F1190EE8CFF2F1780EE8CFF3F1E6
:104F5000520EE8CFF4F19F0EE8CFF5F1F1EC0CF032
:104F6000230EA6EC0EF0E8CFF1F1190EE8CFF2F126
:104F7000780EE8CFF3F1520EE8CFF4F19F0EE8CFB0
:104F8000F5F1B1EC0CF025EE33F0100E0A6F096B61
:104F9000230EA6EC0EF0E8CFF1F11C0E0925E8CFA8
:104FA000F2F11C0E0925E8CFF3F1092B092B640E51
:104FB000E8CFF4F1DECFF5F1D890F533D890F533A2
:104FC000640EF5279D0EF561F56FF1EC0CF00A2FDC
:104FD000DFD725EE43F0100E0A6F096B230EA6EC07
:104FE0000EF0E8CFF1F1560E0925E8CFF2F1560E9A
:104FF0000925E8CFF3F1092B092B640EE8CFF4F172
:10500000DECFF5F1D890F533D890F533640EF5275F
:105010009D0EF561F56FF1EC0CF00A2FDFD7540E01
:10502000E8CF7DF0200EE8CF7CF055EC18F020EEB4
:1050300060F04E0EDE6E320EDE6E4EEC0CF0540E54
:10504000E8CF7DF05A0EE8CF7CF055EC18F020EE5A
:1050500060F0480EDE6E650EDE6E4EEC0CF063C541
:105060000AF120EE60F015EE33F00A2BE6CF31F1B5
:105070000A2FFCD7376B372B366B4CEC0BF0250E19
:10508000DE6E200EDE6E540EE8CF7DF03E0EE8CFD1
:105090007CF0000EE8CF7EF055EC18F04EEC0CF0F2
:1050A0001E9F230EA6EC0EF0E8CFF1F1490EE8CFDB
:1050B000F2F14A0EE8CFF3F1790EE8CFF4F19D0E4C
:1050C000E8CFF5F1B1EC0CF0230EA6EC0EF0E8CF32
:1050D000F1F13D0EE8CFF2F1540EE8CFF3F1790E85
:1050E000E8CFF4F17A0EE8CFF5F1F1EC0CF0230EF5
:1050F000A6EC0EF0E8CFF1F1410EE8CFF2F1500E40
:10510000E8CFF3F1820EE8CFF4F1830EE8CFF5F1AA
:10511000F1EC0CF0230EA6EC0EF0E8CFF1F1410E0D
:10512000E8CFF2F1500EE8CFF3F18B0EE8CFF4F1B7
:105130008C0EE8CFF5F1F1EC0CF0230EA6EC0EF09E
:10514000E8CFF1F1410EE8CFF2F1500EE8CFF3F1E4
:10515000940EE8CFF4F1950EE8CFF5F1F1EC0CF0F8
:10516000230EA6EC0EF0E8CFF1F13D0EE8CFF2F100
:10517000540EE8CFF3F19D0EE8CFF4F19E0EE8CF88
:10518000F5F1F1EC0CF01200E6EC29F0010EE8CF9D
:105190007FF0030E90EC09F0000EE8CF7FF0440E94
:1051A00090EC09F0450E90EC09F0460E90EC09F0F9
:1051B000470E90EC09F0480E90EC09F0490E90EC87
:1051C00009F04A0E90EC09F01200E6EC29F0010E0D
:1051D000E8CF7FF0030E90EC09F0000EE8CF7FF0EF
:1051E0004B0E90EC09F04C0E90EC09F04D0E90EC4B
:1051F00009F04E0E90EC09F04F0E90EC09F0500EB5
:1052000090EC09F0510E90EC09F01200E6EC29F058
:10521000010EE8CF7FF00F0E8DEC09F0000EE8CF05
:105220007FF0100E8DEC09F0110E8DEC09F0120ECE
:105230008DEC09F0130E8DEC09F012002AB5120066
:105240006A0EEDEC18F0A80EE8CF7CF0410EE8CF26
:105250007DF0000EE8CF7EF0000EE8CF7FF020EE6C
:1052600060F018C531F1316708D055EC18F0070E21
:1052700086EC09F04EEC0CF012008CC14BF18DC1A4
:105280004CF10A0E4D6F4E6B39EC0AF048674769D6
:1052900058C1E8FF476103D047C118F52FD08CC132
:1052A0004BF18DC14CF10A0E4D6F4E6B39EC0AF08B
:1052B00047C14BF148C14CF1CFC14DF14E6B1CECD5
:1052C0000AF047C153F148C154F158C1E8FF640DD9
:1052D000F3CF51F1F4CF52F105EC0AF01EA70CD038
:1052E00047C14BF148C14CF1640E4D6F4E6B39EC28
:1052F0000AF047C118F502D058C118F5040E79EC30
:1053000018F018C531F1326B1E8F030E55EC0BF0FF
:105310001E9F4EEC0CF055EC18F0120030EC80F0B3
:1053200001011A0E8DEC09F020EE60F0230EDE6E06
:1053300063C531F163C50AF11E8F376B372B366BAE
:105340004CEC0BF0200EDE6E280EDE6E100E0A61A5
:1053500005D04E0EDE6E320EDE6E04D0480EDE6ECE
:10536000650EDE6E290EDE6E200EDE6E640EE8CF58
:105370007DF0190EE8CF7CF0000EE8CF7EF055EC02
:1053800018F04EEC0CF020EE60F015EE33F00A2B26
:10539000E6CF31F10A2FFCD7376B372B366B4CEC4D
:1053A0000BF0250EDE6E200EDE6E640EE8CF7DF073
:1053B000320EE8CF7CF0000EE8CF7EF055EC18F00E
:1053C0004EEC0CF01E9F1200000E03D0230EA6EC34
:1053D0000EF0E8CFF1F1000EE8CFF2F11A0EE8CFAF
:1053E000F3F1000EE8CFF4F19F0EE8CFF5F1F1EC08
:1053F0000CF012002AB5120027BF120029BB1200C0
:105400002AB912006B0EEDEC18F05A0EE8CF7CF0C2
:10541000000EE8CF7DF0000EE8CF7EF0020E79ECB2
:1054200018F020EE60F0430EDE6E4E0EDE6E530E70
:10543000DE6E3A0EDE6E65C531F11E8F376B372B8F
:10544000366B4CEC0BF01E9F250EDE6E4EEC0CF016
:10545000120065C531F10F0EA6EC0EF0315DD8A03B
:105460001200570EEDEC18F0AF0EE8CF7CF02D0EC9
:10547000E8CF7DF0000EE8CF7EF0000EE8CF7FF0A1
:10548000020E79EC18F020EE60F0430EDE6E4E0E48
:10549000DE6E530EDE6E3A0EDE6E65C531F11E8F86
:1054A000376B372B366B4CEC0BF01E9F250EDE6EE8
:1054B0004EEC0CF01200400ED0EC0BF0010EA86286
:1054C00029D0C80EE8CF7CF0000EE8CF7DF0000EAA
:1054D000E8CF7EF0000EE8CF7FF04DEC18F020EE24
:1054E00060F0400E316F180E326F312B85EC2AF0D0
:1054F0007D0EA86201D004D0A8CFDEFF322FF5D7F1
:105500004EEC0CF055EC18F0120031C1A9FFF9EC8B
:105510000BF01200180E386FC80EE8CF7CF0000EAA
:10552000E8CF7DF04AEC1BF01200000EE8CFF1F15D
:10553000000EE8CFF2F1EF0EE8CFF3F1520EE8CF14
:10554000F4F19F0EE8CFF5F1F1EC0CF012004FC230
:105550000AF14EC209F1095303E0B4EC2AF012003B
:10556000F20E90EC09F01200090EE46FE70EE56F01
:1055700012EE50F0190EE527C1EC2AF0E42FFAD70D
:1055800012001E8F640EE8CF7DF0E5C17CF0E5C10E
:1055900032F1E6CF31F1315120EE60F0376B372B2D
:1055A000366B4CEC0BF06D0EDE6E4EEC0CF08C0E90
:1055B000E8CF7DF0E5C17CF0E6CF31F120EE60F080
:1055C000376B372B366B47EC0BF0270EDE6E4EEC4D
:1055D0000CF0120028B164D06D0EEDEC18F0000E46
:1055E000E8CF7DF0000EE8CF7EF01E8F020E0A6F2E
:1055F0000A0E096F326B322B040E0A2720EE60F080
:10560000470EDE6E32C131F1376B372B366B4CEC07
:105610000BF03A0EDE6E0AC1A9FFF9EC0BF0A8CF31
:1056200031F1376B372B366B4CEC0BF02F0EDE6EF7
:10563000A92AF9EC0BF0A8CF31F1376B372B366B79
:105640004CEC0BF0200EDE6E32511B0FD0EC0BF049
:10565000A8CF31F1376B372B366B36EC0BF06D0E74
:10566000DE6E1B0ED0EC0BF032C131F1A832312FBF
:10567000FDD7D8B004D04A0E4EEC0EF002D055EC57
:1056800018F0190E0927000EE8CF7DF009C17CF053
:105690004EEC0CF055EC18F0050E3263ACD712004E
:1056A000000EE8CF7DF0000EE8CF7EF01E8F230EB7
:1056B0000A6F0A0E096FE46B0A2BE42B190E0927F7
:1056C000000EE8CF7DF009C17CF020EE60F0530EB3
:1056D000DE6E500EDE6EE4C131F1376B372B366B68
:1056E0004CEC0BF03A0EDE6E200EDE6E0AC1A9FF06
:1056F000F9EC0BF0A8CF31F1326B030E55EC0BF047
:105700004EEC0CF0030EE463D7D7210ED0EC0BF077
:10571000A8CFD0F1D005040DF350070FA96EF9EC16
:105720000BF0A8CF32F1D005040DF350060FA96E8F
:10573000F9EC0BF0A8CF31F1000EE8CF7DF06E0E42
:10574000E8CF7CF020EE60F0440EDE6E690EDE6E77
:105750006C0EDE6E3A0EDE6E376B372B366B4CEC12
:105760000BF02F0EDE6E32C131F1376B372B366BFB
:105770004CEC0BF04EEC0CF01E9F120024BD1200FE
:105780001A0ED0EC0BF0A8CF0AF1690E0A611200D4
:10579000630E0A65120031C14BF132C14CF1640E47
:1057A0004D6F4E6B1CEC0AF00AC14DF14E6B60EC74
:1057B0000AF047C131F148C132F112003A6F010ECF
:1057C000BC27000EBD23BDAF02D0BC6BBD6B3A2F12
:1057D000F6D712003A6F010EBC5F000EBD5BBDAF85
:1057E00002D07F0EBD6F3A2FF6D712009CD8010E63
:1057F000BC27000EBD232291BDAF1200BC6BBD6B58
:105800002281120022B31CD822A30BD82283000EBF
:10581000BC2BBD232291BDAF1200BC6BBD6B22819E
:1058200012003A6FC580A3D8A60EC96EA0D894D82E
:10583000BDC1C9FF9CD890D8BCC1C9FF98D88CD82D
:105840003AC1C9FF94D888D812003A6B3B6B219FAC
:10585000219DC5848CD8C5808AD8A60EC96E87D8EC
:10586000C5BCF7D73BC1C9FF82D876D83AC1C9FFBA
:105870007ED872D8C5827BD8A70EC96E78D86CD86E
:10588000C58675D821BD05D0218DFD0EC962219D2B
:1058900011D021BF05D0218FFD0EC96209D00AD0D9
:1058A000FE0EC96205D03AC1BCF13BC1BDF10DD0BD
:1058B000219F219D010E3A27000E3B233BBF03D0C1
:1058C000C58855D8DDD7BC6BBD6BC58450D8219F2A
:1058D000219D1200C5844BD8C58049D8A60EC96E3B
:1058E00046D8C5BCF7D7BDC1C9FF41D835D8BCC162
:1058F000C9FF3DD831D8C5823AD8A70EC96E37D86E
:105900002BD8C58634D8C950C58431D81200E2DFFF
:10591000010EBC27000EBD232291BDAF1200BC6B4F
:10592000BD6B228112003A6FC58021D8A60EC96EC8
:105930001ED812D8BDC1C9FF1AD80ED8BCC1C9FF24
:1059400016D80AD83AC1C9FF12D806D8C5840FD8CC
:10595000060E06EC0BF01200C5BC01D812004D0E6D
:10596000EDEC18F081880BD89E96C36B1200C32F04
:1059700001D0F5D79EA6FBD7C36B9E961200C66AD0
:105980004E0EEDEC18F0C56AC76A9496948882961C
:10599000090EC36F8286000082B804D08296829678
:1059A000C32FF8D79486C66A0A0E06EC0BF0000ED9
:1059B000C76E280EC66E000EC56E080EC86E8198A2
:1059C0004F0EEDEC18F012002495289559EC0DF0CF
:1059D000249324972499BB6BBA6BC06B010EE8CF5C
:1059E0007FF00C0E90EC09F0000EE8CF7FF0A46B76
:1059F000A56BBFEC2CF025EC2CF0386B396B050E49
:105A0000B96F010EE8CF7FF00C0E90EC09F0000E9C
:105A1000E8CF7FF0219D219F010EA427000EA52332
:105A2000A5BF27D0010EEAEC2BF06AEC2CF021BDCB
:105A300005D0218DFA0EC962219D10D021BF05D05D
:105A4000218FFA0EC96207D809D0BCC1BEF1BDC111
:105A5000BFF1C02B13D0219F219D1200010E3827CA
:105A6000000E392339BF01D0D7D724A927EF11F071
:105A70002CD0C051D8B4F9D7248327D0030EDEEC44
:105A80002BF024A704D0A651C063BAD264D024B3AB
:105A90001CD0D1DA050EB96316D0C0C1ABF1BEC1BE
:105AA000A9F1BFC1AAF1A4C190F1A5C191F138C17A
:105AB000EDF139C1A7F1030EA927000EAA23030EA9
:105AC000905F000E915BB92F9BD224A97DD7E6ECA5
:105AD00029F0010EE8CF7FF01A0E90EC09F0000ECD
:105AE000E8CF7FF00B0E90EC09F01F9920912093E6
:105AF000209723992397B76B010E24B5AC51B96F4A
:105B000024952499FCEC1BF006EC30F020B383D2F2
:105B100020B10ED01FB125EC3CF01FB108EC42F0D3
:105B20001F911FB927EF11F01FB3BEEF48F0ECD75C
:105B30002091060EB96302D027EF11F0B9C1ACF184
:105B40002485BA51050DF350B925A66F59EC0DF017
:105B50002487C06B43D724973DEC1BF0000EE8CFA1
:105B60007CF0000EE8CF7DF020EE60F0230EDE6EBC
:105B70001C0EBAEC0EF0316703D0326701D016D09C
:105B8000010E3127000E322331C151F132C152F1E1
:105B9000A6C153F1546B05EC0AF04FC131F150C16D
:105BA00032F11E8F0A0E55EC0BF007D0A6C131F171
:105BB000376B372B366B47EC0BF0200EDE6E87EC25
:105BC0002CF0C9CF31F187EC2CF0C9CF31F1200E88
:105BD000DEEC2BF06AEC2CF0C9CFA8F1200EEAEC39
:105BE0002BF031C1EEF187EC2CF0C9CFEFF187EC4F
:105BF0002CF0C9CFF0F1D4EC22F0200EDE6E87EC51
:105C00002CF0C9CF31F1376B372B366B47EC0BF0EB
:105C10003A0EDE6E87EC2CF0C9CF31F1376B372BA3
:105C2000366B47EC0BF04EEC0CF0190EE8CF7CF025
:105C3000050EE8CF7DF020EE60F087EC2CF0C9CFA8
:105C400031F187EC2CF0C9CF32F131C14BF132C1C7
:105C50004CF1A40E4D6F4E6B39EC0AF047C1C5F103
:105C600048C1C6F1C52B000EC6231E8F030E55EC8E
:105C70000BF06D0EDE6E200EDE6E87EC2CF0C9CFC1
:105C800031F187EC2CF0C9CF32F131C14BF132C187
:105C90004CF13C0E4D6F4E6B1CEC0AF01E8F376BB7
:105CA000372B366B365155EC0BF0270EDE6E87EC3A
:105CB0002CF0C9CF31F131514727000E482347C19D
:105CC0004BF148C14CF19F0E4D6F4E6B39EC0AF011
:105CD00047C14BF148C14CF1A8514D6F4E6B39ECA7
:105CE0000AF047C1C7F148C1C8F1C72B000EC8234D
:105CF0001E8F376B372B366B47EC0BF0220EDE6EA8
:105D0000200EDE6E87EC2CF0C9CF31F187EC2CF041
:105D1000C9CF32F1030E376F1E8F020E55EC0BF018
:105D2000B00EDE6E430EDE6E4EEC0CF0320EE8CF9F
:105D30007CF0050EE8CF7DF020EE60F087EC2CF0D3
:105D4000C9CF31F187EC2CF0C9CF32F11E8F376B00
:105D5000372B366B365155EC0BF06D0EDE6E620E46
:105D6000DE6E610EDE6E720EDE6E200EDE6E440E94
:105D7000DE6E650EDE6E730EDE6E610EDE6E740E0E
:105D8000DE6E200EDE6E87EC2CF0C9CF31F187EC91
:105D90002CF0C9CF32F1E2EC09F01E8F315132C143
:105DA00031F1326F376B372B366B4CEC0BF03A0E10
:105DB000DE6E32C131F1376B372B366B47EC0BF0AF
:105DC0001E9F4EEC0CF087EC2CF087EC2CF087EC4F
:105DD0002CF087EC2CF087EC2CF087EC2CF087EC87
:105DE0002CF087EC2CF087EC2CF087EC2CF087EC77
:105DF0002CF087EC2CF087EC2CF087EC2CF087EC67
:105E00002CF087EC2CF087EC2CF087EC2CF087EC56
:105E10002CF0C9CFB0F1B099B09BB09DB09FB02B22
:105E2000B0C1E8F187EC2CF0C9CFB1F1B199B19BC9
:105E3000B19DB19FB1C1E9F187EC2CF0C9CFB2F1AE
:105E400087EC2CF0C9CFB3F187EC2CF0C9CFB4F1BB
:105E500087EC2CF0C9CFB5F187EC2CF087EC2CF057
:105E6000010EE8CFF1F14B0EE8CFF2F1EF0EE8CFE3
:105E7000F3F1000EE8CFF4F19F0EE8CFF5F1F1EC6D
:105E80000CF087EC2CF0B76B87EC2CF09E0E376F84
:105E9000219F050EB86F4B0EDA6FB8295BEC0CF042
:105EA000C7C1C9F1C8C1CAF1CA2BC96701D0C92B82
:105EB00064D821BF26D0C5C14DF1C6C14EF131C154
:105EC0004BF132C14CF139EC0AF04B0E4727D8B0F8
:105ED000DAC147F19AEC2FF047C1DAF147516AEC89
:105EE0000CF0B82BB8515BEC0CF055EC18F074ECDE
:105EF0000CF0C94F02D041D8FCD7CA2FFAD7372FA0
:105F0000CFD71F992091209323992397B76B06EC45
:105F100030F020B152D020B350D01FB125EC3CF06E
:105F20001FB108EC42F01F911FB947D01FB3BEEF5D
:105F300048F0EDD74751DA6301D012004751DA65D6
:105F40000ED0DAC148F1480748516AEC0CF055EC24
:105F500018F09DEC0CF047514863F5D7120047C18B
:105F600048F1480748516AEC0CF055EC18F09DECEC
:105F70000CF0DA514863F5D7120087EC2CF0C9CF4A
:105F800031F187EC2CF0C9CF32F187EC2CF0C9CF7E
:105F9000B7F1279BB7BF278BB79FFD0E316305D0A5
:105FA000FD0E326302D0218F1200B76701D01200BC
:105FB00087EC2CF0B72FFCD712001F99B76BA9C143
:105FC000BCF1AAC1BDF190C1A4F191C1A5F1ABC1D1
:105FD000C0F1EDC138F1A7C139F1C0072493BA0768
:105FE000BB6B050EB96FBA2B59EC0DF00AD524B373
:105FF000E5EF2CF0BB6B050EB96FBA2B59EC0DF029
:10600000BEC1BCF1BFC1BDF101EF2DF023B92083AA
:1060100023B720811200B92B070EB96301D0E7D74F
:10602000BB29B96302D0060EB96FB76BFCEC1BF04D
:106030002399209369D52489BB2B28B50CD0E6EC95
:1060400029F0010EE8CF7FF01A0E90EC09F0000E57
:10605000E8CF7FF02885140EE8CF7DF0BA51050D0A
:10606000F350C05D1E0DF350050FE8CF7CF020EE1D
:1060700060F0C0C131F1376B372B366B47EC0BF05A
:10608000200EDE6E87EC2CF0C9CF31F10D0E31659C
:1060900004D087EC2CF0C9CF31F131C1EEF187EC9F
:1060A0002CF0C9CFEFF187EC2CF0C9CFF0F12AEC3E
:1060B00023F087EC2CF087EC2CF0200EDE6E87ECC2
:1060C0002CF0C9CF31F187EC2CF0C9CF32F11E8F03
:1060D0002385030E55EC0BF06D0EDE6E200EDE6E8A
:1060E00087EC2CF0C9CF31F187EC2CF0C9CF32F11D
:1060F0001E8F376B372B366B365155EC0BF0270E56
:10610000DE6E4EEC0CF012002C939D9A8186DBEC37
:106110004AF06B0EAD6E22EC0CF081969D8AA5EFD5
:106120003AF027959D9A818620EC80F0010130ECB1
:1061300080F0010118EC80F00101010ECB6FCC6BF7
:10614000680EAD6E22EC0CF01F8581969D8AA5EF3E
:106150003AF027939D9A8186AA6AA3D881969D8A50
:10616000A5EF3AF0299F9D9A8186010EAA6E99D8D3
:10617000AA6A81969D8AA5EF3AF0269F9D9A81860C
:1061800022EC0CF0010EAD6E22EC0CF0470EAD6E61
:1061900029EE4AF0100E386F22EC0CF0DECFADFF86
:1061A000382FFAD781969D8AA5EF3AF0249B9D9AC5
:1061B000818659EC0DF0E6EC29F0010EE8CF7FF076
:1061C0000F0E90EC09F0000EE8CF7FF0050E426F45
:1061D000AA0EAD6E22EC0CF0422FFAD7550EAD6E22
:1061E000100E90EC09F025EC2CF0010EBC27000EEF
:1061F000BD23110E90EC09F054D822EC0CF0C1C173
:10620000ADFF22EC0CF0C2C1ADFF22EC0CF0010E90
:10621000AD6E22EC0CF0470EAD6E120E90EC09F054
:10622000426B436BC580B7EC2CF0A60EC96EB7EC81
:106230002CF0C5BCF7D7BDC1C9FFB7EC2CF0ACEC56
:106240002CF0BCC1C9FFB7EC2CF0ACEC2CF0C58233
:10625000B7EC2CF0A70EC96EB7EC2CF0ACEC2CF020
:10626000130E90EC09F022EC0CF0C586B7EC2CF084
:10627000C9CFADFF010E4227000E432343BF04D018
:10628000C588B7EC2CF0EFD7C584B7EC2CF0140E12
:1062900090EC09F0FA0E06EC0BF081969D8A30EF37
:1062A0003AF0426BA96AF9EC0BF0A8CFADFFA92A2E
:1062B00022EC0CF0422FF7D71200010EB96F209993
:1062C00020971F99A96B219D219F59EC0DF0E6ECB9
:1062D00029F0010EE8CF7FF06F0E90EC09F0000E70
:1062E000E8CF7FF0B76B20912093140EE8CF7DF0BC
:1062F000230EE8CF7CF020EE60F0700E89EC09F000
:10630000A9C131F1312B1E8F376B372B366B36EC31
:106310000BF0200EDE6E280EDE6EC00E89EC09F04A
:10632000200EDE6E210ED0EC0BF0A8CFD0F1D00500
:10633000040DF350060FA96EF9EC0BF0A8CF31F164
:106340001E8F376B372B366B36EC0BF02F0EDE6E55
:10635000D005040DF350070FA96EF9EC0BF0A8CF90
:1063600031F11E8F376B372B366B36EC0BF0290E65
:10637000DE6E4EEC0CF0140EE8CF7DF0410EE8CF4F
:106380007CF020EE60F0610E89EC09F0A951240F39
:10639000A96EF9EC0BF0A8CF31F1326B1E8F030E12
:1063A00055EC0BF01E9F420EDE6E610EDE6E720E1D
:1063B000DE6E200EDE6E4EEC0CF0140EE8CF7DF09B
:1063C0005F0EE8CF7CF020EE60F0BE0E89EC09F0A5
:1063D0004EEC0CF0140EE8CF7DF07D0EE8CF7CF093
:1063E00020EE60F0BF0E89EC09F04EEC0CF0140EBC
:1063F000E8CF7DF09B0EE8CF7CF020EE60F0590EE8
:1064000089EC09F0310EDE6E2E0EDE6E300EDE6E81
:10641000300EDE6E4EEC0CF00B0E90EC09F024EC1E
:1064200011F0FCEC1BF006EC30F020B30FD020B1E3
:106430001ED01FB3BEEF48F01FB125EC3CF01FB1DA
:1064400008EC42F01F911FB91CD0EDD7B92B020EFA
:10645000B96301D0B92B070EB96302D0010EB96F31
:10646000B76BFCEC1BF024EC11F02093DCD7B94F98
:106470003ED0B94F0AD0B94F08D0B94F1AD0B94F52
:106480002CD0020EB96F7CEF11F0A951240FA96E28
:10649000F9EC0BF0A8CF31F1312BFB0E316302D0B8
:1064A000FA0E316F31C1A8FFFDEC0BF0030EB96F8E
:1064B00019D7A951240FA96EF9EC0BF0A8CF31F12F
:1064C0003107FF0E316302D0000E316F31C1A8FFDA
:1064D000FDEC0BF0040EB96F05D7A951240FA96E7E
:1064E000640EA86EFDEC0BF0050EB96FFBD6A92B60
:1064F000030EA96301D0A96B010EB96FF3D659EC55
:106500000DF0E6EC29F0010EE8CF7FF0720E90EC72
:1065100009F0000EE8CF7FF0230EE8CF7CF0000EEC
:10652000E8CF7DF0000EE8CF7EF020EE60F0730E35
:1065300089EC09F0320ED0EC0BF0A8CF31F1330E1C
:10654000D0EC0BF0A8CF32F11E8F376B372B366BA8
:10655000365155EC0BF0200EDE6E280EDE6E340E3A
:10656000D0EC0BF0A8CF31F1350ED0EC0BF0A8CF6A
:1065700032F11E8F376B372B366B365155EC0BF0E3
:10658000290EDE6E4EEC0CF0410EE8CF7CF020EED2
:1065900060F0750E89EC09F02F0ED0EC0BF0A8CF4F
:1065A000EEF1300ED0EC0BF0A8CFEFF1310ED0ECC5
:1065B0000BF0A8CFF0F1D4EC22F04EEC0CF05F0E13
:1065C000E8CF7CF020EE60F0760E89EC09F0280E22
:1065D000D0EC0BF0A8CF31F1290ED0EC0BF0A8CF06
:1065E00032F1010E376F1E8F020E55EC0BF01E9F1D
:1065F000560EDE6E4EEC0CF07D0EE8CF7CF020EEF9
:1066000060F0770E89EC09F02A0ED0EC0BF0A8CFE1
:10661000EEF12B0ED0EC0BF0A8CFEFF12C0ED0EC5E
:106620000BF0A8CFF0F1D4EC22F04EEC0CF09B0E66
:10663000E8CF7CF020EE60F0780E89EC09F0360EA1
:10664000D0EC0BF0A8CF31F1370ED0EC0BF0A8CF87
:1066500032F1030E376F1E8F020E55EC0BF01E9FAA
:10666000B00EDE6E200EDE6E280EDE6E380ED0EC22
:106670000BF0A8CFEEF1390ED0EC0BF0A8CFEFF174
:106680003A0ED0EC0BF0A8CFF0F1D4EC22F0290EAA
:10669000DE6E200EDE6E4EEC0CF0B90EE8CF7CF014
:1066A00020EE60F0790E89EC09F03B0ED0EC0BF097
:1066B000A8CF31F13C0ED0EC0BF0A8CF32F1030E95
:1066C000376F1E8F020E55EC0BF01E9FB00EDE6E64
:1066D000200EDE6E280EDE6E3D0ED0EC0BF0A8CF45
:1066E000EEF13E0ED0EC0BF0A8CFEFF13F0ED0EC68
:1066F0000BF0A8CFF0F1D4EC22F0290EDE6E200EC4
:10670000DE6E4EEC0CF081A0FED7239723992091EA
:1067100006EC30F020B10DD01FB3BEEF48F01FB132
:1067200025EC3CF01FB108EC42F01F911FB901D0DD
:10673000EFD7030EB96F7CEF11F0010EB96F59EC72
:106740000DF033EC38F0B76B1F9920912093E6ECF5
:1067500029F0010EE8CF7FF06A0E90EC09F0000EF0
:10676000E8CF7FF0A96BA46B050E096F020E0A6FCC
:10677000140EE8CF7DF0040E0A271E0E09270951DA
:10678000E8CF7CF020EE60F0470EDE6EA9C131F15B
:10679000312B1E8F376B372B366B36EC0BF03A0EE6
:1067A000DE6EEBEC37F04EEC0CF0280EE8CF7DF00F
:1067B0000951E8CF7CF020EE60F0210EA96EF9ECD3
:1067C0000BF0A804A96302D02A0EDE6EEBEC37F0C2
:1067D0004EEC0CF0300EE8CF7DF00951E8CF7CF0A4
:1067E00020EE60F00AC1A9FFA92AF9EC0BF0A8CFAE
:1067F00031F13153000E31651AD0E4EC37F00AC1A3
:10680000A9FFF9EC0BF0A8CF31F1376B372B366BC2
:106810004CEC0BF02F0EDE6EA92AF9EC0BF0A8CF92
:1068200031F1376B372B366B4CEC0BF03FD00AC194
:10683000A9FFF9EC0BF0A8CF31F13153150E3165FA
:1068400017D0640E316108D0DDEC37F0376B372B91
:10685000366B4CEC0BF02AD04F0EDE6E320EDE6E35
:10686000200EDE6E376B372B366B4CEC0BF01ED0E8
:10687000316349EC34F0410EDE6E490EDE6E520E8D
:10688000DE6E200EDE6E376B372B366B4CEC0BF06A
:106890000DD0450EDE6E520EDE6E520EDE6E200EF6
:1068A000DE6E376B372B366B4CEC0BF0EBEC37F0C6
:1068B0004EEC0CF0690EE8CF7DF00951E8CF7CF08A
:1068C00020EE60F0200EDE6E690EDE6E6E0EDE6E65
:1068D000200EDE6EA9511C0FA96EF9EC0BF0A8CFAB
:1068E00031F1376B372B366B4CEC0BF06D0EDE6EE7
:1068F000EBEC37F04EEC0CF055EC18F0A92B050E34
:10690000A963B8EF33F00B0E90EC09F024EC11F012
:10691000FCEC1BF006EC30F020B30FD020B11ED001
:106920001FB3BEEF48F01FB125EC3CF01FB108ECDF
:1069300042F01F911FB90ED0EDD7B92B070EB963E6
:1069400002D0010EB96FB76BFCEC1BF024EC11F018
:106950002093E0D7020EB96F2BEF11F0B94F09D099
:10696000B94F0CD0B94F0FD0B94F12D0B94F15D085
:10697000F1D7000EA96F000EA46F14D0010EA96FFD
:10698000040EA46F0FD0020EA96F080EA46F0AD0D8
:10699000030EA96F0C0EA46F05D0040EA96F100E84
:1069A000A46F00D0010EB96F2893209920971F99EA
:1069B000219D59EC0DF01E0E90EC09F00B0E90ECA1
:1069C00009F0B76B209120934ADA410EE8CF7CF0B2
:1069D000140EE8CF7DF020EE60F04F0EDE6E320E2A
:1069E000DE6E3A0EDE6E200EDE6EA451060FA96E2C
:1069F000F9EC0BF0A8CF31F1376B372B366B4CEC41
:106A00000BF0250EDE6E200EDE6E280EDE6E4D0EB5
:106A1000DE6E4F0EDE6E440EDE6E3A0EDE6E120E2F
:106A2000A6EC0EF00A0DF3CF4BF1F4CF4CF1A451CC
:106A3000060FA96EF9EC0BF0A8CF4DF14E6B39ECB7
:106A40000AF00A0E475F47C131F1000E485B48C1AA
:106A500032F1376B372B366B365155EC0BF06D0E30
:106A6000DE6E290EDE6E200EDE6E200EDE6E4EEC29
:106A70000CF05F0EE8CF7CF020EE60F0480EDE6E8A
:106A8000650EDE6E3A0EDE6E200EDE6EA451070F2E
:106A9000A96EF9EC0BF0A8CF31F1376B372B366BC1
:106AA0004CEC0BF0250EDE6E200EDE6E200EDE6E40
:106AB0004EEC0CF07D0EE8CF7CF020EE60F02B0E5B
:106AC000DE6E2F0EDE6E2D0EDE6E3A0EDE6E200EA8
:106AD000DE6E2B0E21BD2D0EDE6E4EEC0CF09B0EED
:106AE000E8CF7CF020EE60F0590E89EC09F0A4515B
:106AF000040FA96EF9EC0BF0A8CF31F1376B372BEF
:106B0000366B4CEC0BF02F0EDE6EA451050FA96E08
:106B1000F9EC0BF0A8CF31F1376B372B366B4CEC1F
:106B20000BF0200EDE6E200EDE6E4EEC0CF024EC30
:106B300011F0FCEC1BF006EC30F020B30FD020B1CC
:106B40001AD01FB3BEEF48F01FB125EC3CF01FB1C7
:106B500008EC42F01F911FB918D0EDD7B92B070EE2
:106B6000B96302D0010EB96FB76BFCEC1BF024ECDB
:106B700011F02093E0D7B94F90D0B94F11D0B94F51
:106B800043D0B94F06D0B94F69D0A9C1B9F1B92BDB
:106B9000D6D5217D040EB96F14D7010EB96F09D770
:106BA000A451060FA96EF9EC0BF0A8CF31F121BD6D
:106BB00007D0312B650E316310D0040E316F0DD02C
:106BC0003107030E316309D0A451070FA96EF9EC08
:106BD0000BF0640E316FA850315FA451070FA96EFE
:106BE000F9EC0BF0A8503125326F650E326302D0FC
:106BF000040E316FA451060FA96E31C1A8FFFDEC40
:106C00000BF0020EB96FDDD6A451070FA96EF9EC97
:106C10000BF0A8CF31F121BD06D0312B5C0E3163D2
:106C200007D0316B05D03107FF0E316301D0316BD6
:106C3000A451060FA96EF9EC0BF0A8503125326F64
:106C4000650E326301D03107A451070FA96E31C11F
:106C5000A8FFFDEC0BF0030EB96FB3D6A451040FDF
:106C6000A96EF9EC0BF0A8CF31F1A451050FA96E74
:106C7000F9EC0BF0A8CF32F1A451060FA96E31C187
:106C8000A8FFFDEC0BF0A451070FA96E32C1A8FFBD
:106C9000FDEC0BF0050EB96F94D659EC0DF0010E1A
:106CA000B96F6D0E90EC09F00B0E90EC09F0B76B1C
:106CB00020912093D4D8A4D9410EE8CF7CF0140EB3
:106CC000E8CF7DF020EE60F0690E89EC09F01B0E34
:106CD000D0EC0BF0A9C131F1312BA832312FFDD707
:106CE000D8A004D0600E89EC09F006D0200EDE6E2C
:106CF000200EDE6E200EDE6E4EEC0CF05F0EE8CF46
:106D00007CF0140EE8CF7DF020EE60F0580E89EC98
:106D100009F0200EDE6E210EA96EF9EC0BF0A8042E
:106D2000A96304D0600E89EC09F006D0200EDE6E57
:106D3000200EDE6E200EDE6E4EEC0CF07D0EE8CFE7
:106D40007CF0140EE8CF7DF020EE60F06B0E89EC45
:106D500009F04EEC0CF09B0EE8CF7CF0140EE8CF5F
:106D60007DF020EE60F06C0E89EC09F04EEC0CF03A
:106D700024EC11F0FCEC1BF006EC30F020B30FD04B
:106D800020B11AD01FB3BEEF48F01FB125EC3CF084
:106D90001FB108EC42F01F911FB9F7D6EDD7B92B00
:106DA000070EB96302D0010EB96FB76BFCEC1BF094
:106DB00024EC11F02093E0D7B94FEFD6B94F11D0A2
:106DC000B94F05D0B94F23D0B94F35D0DED6A9C1C0
:106DD000A8FFA82A210EA96EFDEC0BF0030EB96FD7
:106DE00066D71B0ED0EC0BF0A9C131F1312B314F1E
:106DF000A870314FA872314FA874314FA876314F27
:106E0000A8781B0ECEEC0BF0020EB96F50D7A9512B
:106E10001C0FA96EF9EC0BF0A8CF31F1312B640EE9
:106E2000316302D0630E316F31C1A8FFFDEC0BF06E
:106E3000040EB96F3CD7A9511C0FA96EF9EC0BF0E9
:106E4000A8CF31F13107FF0E316302D0000E316F50
:106E500031C1A8FFFDEC0BF0050EB96F28D7E6ECA9
:106E600029F0010EE8CF7FF0020EE8CF7CF0000E93
:106E7000E8CF7DF020EE60F05F0E89EC09F0A9C14B
:106E800031F1312B1E8F376B372B366B36EC0BF015
:106E90003A0EDE6E200EDE6E4EEC0CF0020EE8CFE7
:106EA0007CF0320EE8CF7DF020EE60F0A451070FA9
:106EB000A96EF9EC0BF0A8CF31F13153000E31651A
:106EC0001DD0E4EC37F0A451060FA96EF9EC0BF0DD
:106ED000A8CF31F1376B372B366B4CEC0BF02F0E04
:106EE000DE6EA451070FA96EF9EC0BF0A8CF31F1BB
:106EF000376B372B366B4CEC0BF041D0A451060F9F
:106F0000A96EF9EC0BF0A8CF31F13153150E3163B6
:106F1000316517D0640E316108D0DDEC37F0376B86
:106F2000372B366B4CEC0BF02AD04F0EDE6E320E48
:106F3000DE6E200EDE6E376B372B366B4CEC0BF0B3
:106F40001ED031630ED0410EDE6E490EDE6E520E43
:106F5000DE6E200EDE6E376B372B366B4CEC0BF093
:106F60000ED0450EDE6E520EDE6E520EDE6E200E1E
:106F7000DE6E376B372B366B4CEC0BF000D0200EEF
:106F8000DE6E690EDE6E6E0EDE6E200EDE6EA951B6
:106F90001C0FA96EF9EC0BF0A8CF31F1376B372B32
:106FA000366B4CEC0BF06D0EDE6E200EDE6E4EEC92
:106FB0000CF0000EE8CF7FF012004E0EDE6E580E81
:106FC000DE6E200EDE6E1200540EDE6E580EDE6E89
:106FD000200EDE6E12001B0ED0EC0BF0A9C131F1B9
:106FE000312BA832312FFDD7D8A006D0230EA6EC26
:106FF0000EF04EEC0EF012004A0E4EEC0EF01200A7
:10700000A451060FA96EF9EC0BF0A8CF32F1A951EB
:107010001C0FA96EF9EC0BF0A8CF31F10A0E312745
:1070200032513103F3CF4BF1F4CF4CF10A0E4D6FD7
:107030004E6B39EC0AF047C131F148C132F1370EDD
:10704000E8CF7DF0230EE8CF7CF020EE60F0950EC7
:1070500089EC09F0030E55EC0BF0960E89EC09F063
:107060004EEC0CF01200AA6AA86A760ECEEC0BF079
:10707000770ECEEC0BF0780ECEEC0BF0790ECEEC5A
:107080000BF07A0ECEEC0BF0150EA86E600ECEEC67
:107090000BF0640ECEEC0BF0680ECEEC0BF06C0E29
:1070A000CEEC0BF0700ECEEC0BF0A86A610ECEECBD
:1070B0000BF0650ECEEC0BF0690ECEEC0BF06D0E06
:1070C000CEEC0BF0710ECEEC0BF0030EA96EAA6A9B
:1070D00020EE60F0A92AF9EC0BF0A8CFDEFF170E26
:1070E000A962F8D71C0ED0EC0BF0A8CFDEFF1D0E66
:1070F000D0EC0BF0A8CFDEFF1E0ED0EC0BF0A8CF2B
:10710000DEFF1F0ED0EC0BF0A8CFDEFF200ED0EC80
:107110000BF0A8CFDEFF1B0ED0EC0BF0A8CFDEFFEC
:1071200020EE74F0050EEA6FE86BDE50E827EA2FD8
:10713000FCD7E86701D012002091630EEB6F2DD8C9
:10714000050EEC6F3ED8E8C1A8FF7A0ECEEC0BF02E
:1071500024D8040EEC6F35D8E8C1A8FF790ECEEC28
:107160000BF01BD8030EEC6F2CD8E8C1A8FF780EEB
:10717000CEEC0BF012D8020EEC6F23D8E8C1A8FFBA
:10718000770ECEEC0BF009D8010EEC6F1AD8E8C1DF
:10719000A8FF760ECEEC0BF01200E96BE86BEA6B01
:1071A00020EE74F0DE50EB6505D0E86103D0E86FA7
:1071B000E9C1EAF1E92B050EE963F4D7E8C1EBF187
:1071C000120020EE60F0EA51040DF350D926000EB3
:1071D000DA22EAC1EDF1ED2B79C0E9F11B0ED0EC1A
:1071E0000BF0E933ED2FFDD7D8A0E86BEC51040D7F
:1071F000F3CFA9FF5A0EA926DECFA8FFFDEC0BF0B6
:10720000A92ADECFA8FFFDEC0BF0A92ADECFA8FF4C
:10721000FDEC0BF0A92ADECFA8FFFDEC0BF012006D
:1072200024BD1FD0AECF42F1600E425F424F248B8F
:10723000424F238B424F248D424F2581424F268F50
:10724000424F0000424F2783424F2785424F2A81F9
:10725000424F298F424F2C83AE509E9AAB98AB88F9
:1072600012002BB7F9D78186AE6601D0AE2AAE5098
:10727000640DF3CFC5F1F4CFC6F1EED7F292D5BECF
:1072800009D02387D58E1200F090D5BE03D0238974
:10729000D58E1200F294D56AD76AD66AD58E1200BE
:1072A000F294D59ED76AD66A1200F19C2991000EFD
:1072B000D56ED58E1200F18C1200F19A2993000E32
:1072C000D56ED58E1200F18A1200A192B19ECA9499
:1072D00012009E908198080ECF60402B080ECF5E62
:1072E000402B0F0E406502D0D6EC39F01FA901D01B
:1072F000120022BF1200412B010E41630AD0229DD1
:107300003E6B3F6B9A6B9B6B23EC17F013EC17F003
:107310001200020E41630FD01AEC17F020EC17F0A8
:10732000FBEC15F08C513E278D513F2396519A2747
:1073300097519B231200030E416301D0E5D7040E41
:10734000416301D0E9D7050E416301D0DDD7060EB8
:10735000416301D0E1D7070E416301D0D5D7DCDF0F
:10736000416B020E3D6FD8903F333E33D8909B3334
:107370009A333D2FF8D73FC18DF13EC18CF19BC1AF
:1073800097F19AC196F1228D24AD04D0E80E9E6F3C
:10739000030E9F6F1E979E518C5D8E6F9F518D596E
:1073A0008F6FD8A812008E6B8F6B1200406B1F81FD
:1073B000D8941FA31CD0A72BA805A76502D0A76B44
:1073C0002187172BD8B4182B21A911D0A62B3B0E3F
:1073D000A66505D0A66B1F87A42BD8B4A52B29AB17
:1073E00006D0DB2B3B0EDB6502D0DB6BDA2B032BED
:1073F0003B0E03651200036B1F85042B3B0E0465D7
:107400001200046B052B170E05651200056B062B89
:10741000F8C103F107C175F1754F1F0E754F1C0EB2
:10742000754F1F0E754F1E0E754F1F0E754F1E0E9A
:10743000754F1F0E754F1F0E754F1E0E754F1F0E89
:10744000754F1E0E754F1F0E06651200010E066F5A
:10745000072B0C0E07651200010E076F082B120098
:107460000DEC49F0316B31C118F5E0EC0DF0BFECDB
:107470002CF00BEC0CF097EC0DF0ECEC24F085EC20
:107480001BF05EEC23F0A2C100F5A3C101F5A2C17F
:1074900002F5A3C103F527BF12D029BB10D029ECF8
:1074A0002AF0A4EC21F0D9EC21F02CA59CEC27F0DB
:1074B0002CB5F6EC1EF0D5EC1FF03EEC1EF027AF1D
:1074C00003D0670E90EC09F029AB03D0740E90EC5A
:1074D00009F0B76BB86B1F9D1F9F229D946B956B36
:1074E000986B996B050EB66F81968198249D2B97AA
:1074F000000EE8CF7CF0000EE8CF7DF0000EE8CF64
:107500007EF0000EE8CF7FF055EC18F0239723991A
:10751000D5EC1FF05BEC2AF0010ECE6F470EEDECC0
:1075200018F00C0EA6EC0EF00A6F0AC113F50B0E44
:10753000A6EC0EF00A6F0AC112F530EC80F00101E2
:10754000480EEDEC18F024EC11F01FA119D028A181
:1075500001D000D085EC1BF05BEC3BF025EC3CF05F
:1075600089EC46F03FEC22F0E1EC3BF031EC3BF0F3
:107570009FEC10F03EEC1EF02BB14DEC46F01F914D
:10758000FEEC3BF022BD11EC22F022BD37EC1DF0E9
:1075900022BD08EC42F0229D1FB5F4EC3AF01FBF6B
:1075A00027EF11F01FB331EF3CF01FB992EF45F018
:1075B00024BBD6EF30F023BBFFEF47F025B1D7EF68
:1075C0000BF02AB1D2EF0BF026BFBDEF30F027B39E
:1075D000A9EF30F027B591EF30F029BFB2EF30F0CE
:1075E0002CB384EF30F0B1D75EEC23F034EC3BF0F9
:1075F000A8EC47F05BEC2AF021EC3BF027BF10D061
:1076000029BB0ED029EC2AF0D9EC21F0A4EC21F012
:107610001FBD06D02CA59CEC27F02CB5F6EC1EF077
:1076200014EC3BF01F9512002681010ECB5F000E7B
:10763000CC5BCB671200CC67120026918196CB2BD6
:10764000120020C531F121C532F1316705D0326712
:1076500003D0196B1A6B1200010E1927000E1A23A2
:10766000120026B1817612008188490EEDEC18F0E7
:107670009EC102F59FC103F50A6B0AC111F54F0EB9
:107680000A6F0AC110F58CC100F58DC101F50B0E12
:10769000A6EC0EF00A6F0AC112F50C0EA6EC0EF065
:1076A0000A6F0AC113F540EC80F001014A0EEDECBF
:1076B00018F08198120094928282239182A42381EF
:1076C000829294820A0EDAEC0AF0239382A4238336
:1076D0009492829223B171D023B364D0948228A96A
:1076E00044D0289F2899320ED0EC0BF0A8CF38F167
:1076F000330ED0EC0BF0A8CF39F1D890010E38271B
:10770000000E392338C1A8FF320ECEEC0BF039C180
:10771000A8FF330ECEEC0BF0340ED0EC0BF0A8CF5C
:1077200038F1350ED0EC0BF0A8CF39F1D890010E1E
:107730003827000E392338C1A8FF340ECEEC0BF0E9
:1077400039C1A8FF350ECEEC0BF007C1A8FF2F0EF4
:10775000CEEC0BF006C1A8FF300ECEEC0BF008C14A
:10776000A8FF310ECEEC0BF0120028AF1200289FBC
:10777000320ED0EC0BF0A8CF38F1330ED0EC0BF07A
:10778000A8CF39F1D890010E3827000E392338C11F
:10779000A8FF320ECEEC0BF039C1A8FF330ECEECB1
:1077A0000BF012008188640E06EC0BF08198640ED9
:1077B00006EC0BF08188288912008188288F28998F
:1077C00012001FAD1200B82B040EA6EC0EF0B86527
:1077D00012001F9DE4EC29F027BF08D029BB06D07A
:1077E0002CA59CEC27F02CB5F6EC1EF011EC22F049
:1077F000ECEC24F0B86B23972399120023B718D030
:1078000023B907D0D59EF294D76AD66AF292F09047
:1078100012002399E6EC29F0010EE8CF7FF0040E68
:1078200090EC09F0000EE8CF7FF01F8DB76B1200CF
:1078300023971FAD02D01F8F12002C752CA59CEC36
:1078400027F02CB5F6EC1EF01200B72B030EA6ECB9
:107850000EF0050FD8B0FF0EE806B76512001F89BD
:10786000120053EC42F0520EEDEC18F059EC0DF012
:10787000E3EC19F0D2EC1DF065EC1DF029BB1F877D
:1078800027BF04D029BB02D007EC1AF01FA145D0B6
:107890001FAD59EC1BF027BF09D029BB17D028B169
:1078A00018D027EC3FF00CEC3DF01BD01FADB6EC30
:1078B00023F096EC41F02BB38BEC24F023BF04D0E3
:1078C000238F2EEC42F00DD0239F0BD0BDEC3CF06B
:1078D00008D01EEC29F00CEC3DF02BB529EC3FF064
:1078E00000D096EC41F022B73FEC22F01FBDB3EC84
:1078F0003CF01FBF48EC45F0EDEC3CF02BB14DECFB
:1079000046F02BB38BEC24F01F91260EA6EC0EF064
:10791000316F010E316301D0258325A30BD01FBD2C
:1079200008D0B6EC23F028B11EEC29F026B527ECE0
:107930003FF025931FAFFCEC42F01FBF40EC43F03B
:107940001FA38CD322BDBBEC41F0229D1FB5DAEC06
:1079500041F021B70BEC3EF01FBF04D024BD02D094
:107960000300000093D7B82B040EA6EC0EF0B86508
:1079700012001F9D7CEC23F0120025EC24F021B9AD
:107980000DD0E6EC23F0E02B3C0EE06302D0E06B80
:10799000DF2B259721B912002587120025A7120099
:1079A0000BD813EC24F0DE6BE06BDF6BDB6BDA6B78
:1079B000906B916B25971200DCC151F1DDC152F142
:1079C00090C153F191C154F105EC0AF01EA71200C9
:1079D00090C1DCF191C1DDF11200819832C531F125
:1079E0000E0EA6EC0EF0316107EC3DF026BB81884F
:1079F0001FC531F1312D120066C531F10E0EA6EC16
:107A00000EF0316107EC3DF026BB818812008188C1
:107A1000020EAF6F278B120023BFAED0238F2EEC48
:107A200042F0F2EC3EF08CC14BF18DC14CF10A0EEC
:107A30004D6F4E6B39EC0AF047C14BF148C14CF128
:107A4000CFC14DF14E6B1CEC0AF047C14BF148C160
:107A50004CF1640E4D6F4E6B39EC0AF047C107F5DF
:107A600028B118C507F528EC80F0010165C531F192
:107A70001B0EA6EC0EF0315DD8B0FAEC29F082ECCA
:107A80003FF024A16AD0610ED0EC0BF0A8CF0FF527
:107A9000600ED0EC0BF00FC50AF1D880640E0A55C9
:107AA000A856A8CF0EF5650ED0EC0BF0A8CF0DF5BB
:107AB000640ED0EC0BF00DC50AF1D880640E0A55A7
:107AC000A856A8CF0CF5690ED0EC0BF0A8CF0BF59B
:107AD000680ED0EC0BF00BC50AF1D880640E0A5585
:107AE000A856A8CF0AF56D0ED0EC0BF0A8CF09F57B
:107AF0006C0ED0EC0BF009C50AF1D880640E0A5563
:107B0000A856A8CF08F5710ED0EC0BF0A8CF1DF544
:107B1000700ED0EC0BF01DC50AF1D880640E0A552A
:107B2000A856A8CF1CF5760ED0EC0BF0A8CF6AF5BE
:107B3000770ED0EC0BF0A8CF69F5780ED0EC0BF0F7
:107B4000A8CF68F5790ED0EC0BF0A8CF67F57A0EC8
:107B5000D0EC0BF0A8CF1BF51200460EEDEC18F0A0
:107B6000316B31C16AF531C169F531C168F531C197
:107B700067F531C11BF51200239F27BF120029BBF7
:107B80001200420EEDEC18F0E1EC3DF0000EE8CFF3
:107B90004CF200EC80F00101430EEDEC18F023C52F
:107BA000CDF1CD6712002BC50AF10A6729D024B1A7
:107BB00007EC1AF02491A96B22C5AAF11AEC1AF06D
:107BC00012008CC100F58DC101F50B0EA6EC0EF074
:107BD0000A6F0AC112F50C0EA6EC0EF00A6F0AC16C
:107BE00013F5100EA6EC0EF00A6F0AC117F51D0E64
:107BF000A6EC0EF00A6F0AC11EF50DEC49F012005A
:107C000024A13EEC1AF024812BC5A9F124C5AAF1C8
:107C100047EC1AF0120021972583819824BD1200A9
:107C200021BB08D0218BBCC1BEF1BDC1BFF12F0E5D
:107C3000DEEC2BF08E51F6EC2BF08F51F6EC2BF0A6
:107C4000AD6BB02D02D0020EAD27B12D02D0020EC9
:107C5000AD27B22D02D0020EAD27B32D02D0030EF8
:107C6000AD27B42D02D0090EAD27B52D02D0000EE0
:107C7000AD2727AB11D0010EAD27AE6BAF51AE27AC
:107C8000AF6B27A703D0020EAD27AE8927A903D07B
:107C9000010EAD27AE8BAD8FAD51F6EC2BF027ABBF
:107CA00016D0AE51F6EC2BF027A70CD0180ED0EC66
:107CB0000BF0A850F6EC2BF0190ED0EC0BF0A850FE
:107CC000F6EC2BF027A903D0D051F6EC2BF0279B34
:107CD00027972799B02F01D07AD8B12F01D06CD82F
:107CE000B22F01D05ED8B32F01D04DD8B42F01D020
:107CF00018D8B52F01D010D8B0BFB06BB1BFB16BE1
:107D0000B2BFB26BB3BFB36BB4BFB46BB5BFB56B2F
:107D1000440EEDEC18F012001A0EA6EC0EF0B56F42
:107D2000120031C9B4F1B451F6EC2BF030C9B4F102
:107D3000B451F6EC2BF033C9B4F1B451F6EC2BF09E
:107D400032C9B4F1B451F6EC2BF035C9B4F1B451E9
:107D5000F6EC2BF034C9B4F1B451F6EC2BF037C982
:107D6000B4F1B451F6EC2BF036C9B4F1B451F6ECE1
:107D70002BF038C9B4F1B451F6EC2BF0190EA6EC87
:107D80000EF0B46F1200000EF6EC2BF0000EF6ECC5
:107D90002BF0000EF6EC2BF0180EA6EC0EF0B36FE5
:107DA0001200000EF6EC2BF0000EF6EC2BF0170E86
:107DB000A6EC0EF0B26F1200A951F6EC2BF0AA510E
:107DC000F6EC2BF0160EA6EC0EF0B16F12009651E9
:107DD000F6EC2BF09751F6EC2BF0150EA6EC0EF00E
:107DE000B06F12001FA32DD08CC151F18DC152F183
:107DF00094C153F195C154F18CC194F18DC195F1A9
:107E000005EC0AF04FC14BF150C14CF1270E4D6FFC
:107E10004E6B1CEC0AF047C144F148C145F1070E16
:107E2000466FEFEC09F0630E446501D0446F050E18
:107E3000A6EC0EF0445DD8A004D0208B0CEC1BF017
:107E4000120020AB1200209B33EC1BF0120028B173
:107E500012008CC14BF18DC14CF10A0E4D6F4E6B6F
:107E600039EC0AF047C14BF148C14CF1CFC14DF19B
:107E70004E6B1CEC0AF047C153F148C154F1130E8C
:107E8000A6EC0EF0640DF3CF51F1F4CF52F105ECF6
:107E90000AF026951EB72685269B47C153F148C197
:107EA00054F1120EA6EC0EF0640DF3CF51F1F4CFA5
:107EB00052F105EC0AF01EA704D0268B050EAF6F19
:107EC000278B47C153F148C154F1110EA6EC0EF0B7
:107ED000640DF3CF51F1F4CF52F105EC0AF01EB767
:107EE00005D0268B2685040EAF6F278B26B506D0CE
:107EF00026A307D0BEEC1DF0269303D093EC1DF013
:107F0000268312002B9D8EC14BF18FC14CF1640E64
:107F10004D6F4E6B39EC0AF01B0ED0EC0BF0A8A0A5
:107F200011D0010ED06301D00DD01C0ED0EC0BF09F
:107F3000030EA86407D04751A86404D0030EA85CC0
:107F400047612B8D1B0ED0EC0BF0A8A211D0020EB6
:107F5000D06301D00DD01D0ED0EC0BF0030EA86441
:107F600007D04751A86404D0030EA85C47612B8D4D
:107F70001B0ED0EC0BF0A8A411D0030ED06301D0DF
:107F80000DD01E0ED0EC0BF0030EA86407D04751A5
:107F9000A86404D0030EA85C47612B8D1B0ED0ECA7
:107FA0000BF0A8A610D0040ED06301D00CD01F0E89
:107FB000D0EC0BF0A86407D04751A86404D0030E9E
:107FC000A85C47612B8D1B0ED0EC0BF0A8A810D03D
:107FD000050ED06301D00CD0200ED0EC0BF0A864BD
:107FE00007D04751A86404D0030EA85C47612B8DCD
:107FF000D2EC1DF0120020C54BF121C54CF14B67AE
:1080000007D04C6705D0010ECB6FCC6B26911200C8
:108010004BC104F54CC105F50D0EA6EC0EF04D6FED
:108020004DC106F54B0EEDEC18F01CEC80F0010193
:108030004C0EEDEC18F004C54BF105C54CF14B6747
:1080400007D04C6705D0010ECB6FCC6B2691120088
:108050004BC1CBF14CC1CCF1268112001FA78BEF95
:1080600041F024BD8BEF41F029BBA6DCA2C100F595
:10807000A3C101F50C0EA6EC0EF00A6F0AC113F5B0
:10808000470EEDEC18F030EC80F00101B4DF480E43
:10809000EDEC18F0FD0EF6EC2BF0FD0EF6EC2BF0EF
:1080A000FE0EF6EC2BF0BEC1BCF1BFC1BDF1FA0E65
:1080B000F6EC2BF0FA0EF6EC2BF0200EF6EC2BF093
:1080C0000751F6EC2BF00651F6EC2BF00851F6ECCC
:1080D0002BF00551F6EC2BF00451F6EC2BF029AB0C
:1080E00011D0DCC131F1DDC132F1BEEC2BF031C178
:1080F000DCF132C1DDF1DC51F6EC2BF0DD51F6ECB8
:108100002BF010D090C131F191C132F1BEEC2BF0C7
:1081100031C190F132C191F19051F6EC2BF09151B7
:10812000F6EC2BF0A451F6EC2BF0A551F6EC2BF06D
:10813000A651F6EC2BF0AB51F6EC2BF0AC51F6EC73
:108140002BF0A251F6EC2BF0A351F6EC2BF020C54E
:1081500031F121C532F13151F6EC2BF03251F6EC10
:108160002BF0060ED0EC0BF0A850F6EC2BF0070E1F
:10817000D0EC0BF0A850F6EC2BF00A0ED0EC0BF084
:10818000A850F6EC2BF00B0ED0EC0BF0A850F6EC50
:108190002BF00E0ED0EC0BF0A850F6EC2BF00F0EDF
:1081A000D0EC0BF0A850F6EC2BF0120ED0EC0BF04C
:1081B000A850F6EC2BF0130ED0EC0BF0A850F6EC18
:1081C0002BF0160ED0EC0BF0A850F6EC2BF0170E9F
:1081D000D0EC0BF0A850F6EC2BF0180ED0EC0BF016
:1081E000A850F6EC2BF0190ED0EC0BF0A850F6ECE2
:1081F0002BF0210ED0EC0BF0A850F6EC2BF0010E7A
:10820000F6EC2BF0470EF6EC2BF0C151F6EC2BF010
:10821000C251F6EC2BF0140EA6EC0EF029BB010EA9
:10822000F6EC2BF0020E386F383B150EA6EC0EF074
:108230003825F6EC2BF0020E386F383B160EA6EC04
:108240000EF03825F6EC2BF0020E386F383B170E87
:10825000A6EC0EF03825F6EC2BF0030E386F383B09
:10826000180EA6EC0EF03825F6EC2BF0090E386F40
:10827000383B190EA6EC0EF03825F6EC2BF0000E6C
:10828000386F383B1A0EA6EC0EF03825F6EC2BF0C2
:108290001A0ED0EC0BF0A850F6EC2BF0000EF6EC1A
:1082A0002BF0FB0EF6EC2BF0FB0EF6EC2BF0020E97
:1082B000D0EC0BF0A8CF38F1030ED0EC0BF0A8CF28
:1082C00039F1D890010E3827000E392338C1A8FFA4
:1082D000020ECEEC0BF039C1A8FF030ECEEC0BF072
:1082E0001C0EBAEC0EF0316703D0326701D012D009
:1082F000010E3127000E3223700E820FA96E31C19C
:10830000A8FFFDEC0BF0700E830FA96E32C1A8FF21
:10831000FDEC0BF08196249D2CB1E6EC4AF060EC6C
:1083200080F00101196B1A6B30EF3AF01FA71200B1
:1083300029BB0ED024BD19D01F93B62B020EA6EC7C
:108340000EF0020FD8B0FF0EE806B6651F831200CC
:10835000B62B3C0EB6631200B66B1F93DE2B1E0EBF
:10836000A6EC0EF0DE631F8312001F93B62B050EE2
:10837000B6651F83120008EC42F01FB3E4EC41F035
:108380001FB3F7EC41F0209D96519863208D9751D3
:108390009963208D20BD65EC1DF0209F8C51946366
:1083A000208F8D519563208F24BD208F20BFEDEC51
:1083B00020F0120089EC46F01EEC42F08EEC23F027
:1083C000A8EC47F01F95120090C151F191C152F1F4
:1083D0008EC153F18FC154F105EC0AF01EA71200B3
:1083E0008EC190F18FC191F18EEC23F01200ABC1E0
:1083F00051F1ACC152F196C153F197C154F105EC62
:108400000AF01EB7120096C1ABF197C1ACF1120091
:108410002199000EA6EC0EF0516F526B8EC153F1F4
:108420008FC154F105EC0AF01EA705D01FB7B66B3B
:108430001F83218912001FA71F93120022B709D0A2
:108440000C0EC26501D01200070EAF6F278B22877A
:1084500012000D0EC265F8D7229712008EC115F1D9
:108460008FC116F11551112716511223000E132337
:1084700014231551112716511223000E1323142310
:1084800017C14DF118C14EF111C147F112C148F1A8
:1084900013C149F114C14AF160EC0AF047C192F1ED
:1084A00048C193F11200510EEDEC18F0906B916BF6
:1084B000926B936B17EC0EF05A0ED0EC0BF0000E93
:1084C000A864E0EC0DF0116B126B136B146B010ED2
:1084D000176F186B010EDC6FDD6BDF6BE06BDA6B17
:1084E000DB6BA46BA56BA66BA76BDE6BB66BB76B78
:1084F000AF6B279B2A9BD16924912B952B9D25EC53
:108500002CF0A3C103F5A2C102F596C1ABF197C14E
:10851000ACF10A6B0AC14EF20AC14FF202EE50F002
:10852000200E0A6FEE6A0A2FFDD702EE70F0200EC1
:108530000A6F010EEE6E0A2FFCD702EE90F0EE6A83
:10854000EE6A2B83290EA6EC0EF0316F010E31631B
:108550002B93140EA6EC0EF0A86F150EA6EC0EF0E1
:10856000B06F160EA6EC0EF0B16F170EA6EC0EF063
:10857000B26F180EA6EC0EF0B36F190EA6EC0EF04B
:10858000B46F1A0EA6EC0EF0B56F29AB02D0010E37
:10859000A86F240ED0EC0BF028B1A8CF18F5A8CF07
:1085A00058F181962297219B1F9D1F97258324AD0B
:1085B0001AEC0CF0210ED0EC0BF0A8CFD0F1D005C6
:1085C000040DF350070FA96EF9EC0BF0A8CF11F5CD
:1085D000D005040DF350060FA96EF9EC0BF0A8CFEF
:1085E000CFF111C50AF1D880640E0A55D880A8567B
:1085F000A8CF10F52A95120023B718D023A912008E
:108600002397239929991F8D1F9FB86B29BB0AD0E7
:10861000010EE8CF7FF0040E90EC09F0000EE8CFD9
:108620007FF012008D0E90EC09F012002397239931
:108630001FAD14D029AB03D01F931F9D12001F8FB5
:108640001F9DB6EC26F02EEC25F02B992A9F010EEB
:10865000B96FC8EC26F02399239712002BB7AAD044
:108660008188060EAF6F278B2BA31200116B126B44
:10867000136B146B020E176F186B2EEC42F0120086
:1086800023B715D023A912002CB9FFD025B91CD1CE
:1086900025BDF3D02399B86BB92B060E2ABD040E65
:1086A000B96302D0010EB96FC8EC26F0120023970F
:1086B00023991F8F1F9DB86B2CB9E7D025BBB0D174
:1086C00025B902D125BDD9D025B500D12BB9E9EF07
:1086D00043F02ABF0BD0B94FDAD0B94F8AD1B94F86
:1086E00053D0B94F45D0B94FE9D11200B94FBCD0E2
:1086F000B94F17D0B94FC3D0B94F03D0B94FDED15E
:1087000012002B732BA30AD0116B126B136B146B1B
:10871000020E176F186B2EEC42F0D0D179EC24F0DA
:10872000CDD15A0ED0EC0BF0A86608D017EC0EF0A5
:10873000010EA86E5A0ECEEC0BF007D0E0EC0DF057
:10874000000EA86E5A0ECEEC0BF0D2EC1DF065ECCC
:108750001DF0EDEC20F08EEC23F029BBAFD127BF4C
:10876000ADD124B13EEC1AF024A107EC1AF0A6D149
:10877000B6EC26F04CEC25F0010EB96F2A8FC8EC50
:1087800026F023992397120028B126D12585B6EC2F
:1087900026F0CFC1A8FF180ECEEC0BF011C5A8FF34
:1087A000190ECEEC0BF05FEC25F0010EB96FC8ECA2
:1087B00026F012001F8F1F9D239923972B89B6EC5B
:1087C00026F098EC25F02A9F010EB96FC8EC26F030
:1087D0001200B94F73D1B94F39D0B94F3ED0B94F0C
:1087E0002ED0B94F25D06AD198EC25F0980E516F54
:1087F0003A0E526FC5C153F1C6C154F105EC0AF0EF
:108800001EA705D0980EC56F3A0EC66F1200E80E6F
:10881000516F030E526FC5C153F1C6C154F105EC3F
:108820000AF01EB71200E80EC56F030EC66F1200E5
:10883000E80EC55F030EC65B050EB96FD5D7E80E0F
:10884000C527030EC623040EB96FCED7640EC52705
:10885000000EC623020EB96FC7D7640EC55F000EA7
:10886000C65B030EB96FC0D7258DB6EC26F030EC91
:1088700080F0010199EC27F01200259D1FD12C8971
:10888000B6EC26F08EEC29F012002C9917D1258930
:10889000220ED0EC0BF0030EA8640DD00CD02A856C
:1088A00059EC0DF095EC2AF023C5CDF1CD671200FF
:1088B000A7EC2AF01200B6EC26F023C5CDF1CD6767
:1088C0001200E3EC25F012002599F8D0B94F6FD0D3
:1088D000B94F4ED0B94F38D0B94F17D0B94F01D09A
:1088E0001200190ED0EC0BF0A8CF31F13107FF0EBA
:1088F000316301D0312B31C1A8FF190ECEEC0BF042
:108900005FEC25F0050EB96F1200190ED0EC0BF0DC
:10891000A8CF31F1312B650E316302D0040E316FD7
:10892000180ED0EC0BF0A8503125326F650E326373
:1089300001D0310731C1A8FF190ECEEC0BF05FEC6E
:1089400025F0040EB96F1200180ED0EC0BF0A8CF72
:1089500031F13107030E316301D0312B31C1A8FF52
:10896000180ECEEC0BF05FEC25F0030EB96F120081
:10897000180ED0EC0BF0A8CF31F1312B650E31631E
:1089800002D0050E316F190ED0EC0BF0A850312536
:10899000326F650E326301D0310731C1A8FF180E66
:1089A000CEEC0BF05FEC25F0020EB96F1200190E41
:1089B000D0EC0BF0A8CF11F5180ED0EC0BF0A8CF2F
:1089C000CFF111C50AF1D880640E0A55A856A8CF78
:1089D00010F52787278B72D0258BB6EC26F02891CF
:1089E000298930EC26F02881010EB96FC8EC26F0F9
:1089F000120028B10AD0258BB6EC26F030EC26F018
:108A0000010EB96FC8EC26F012002A8D258BB6EC4A
:108A100026F081EC26F0010EB96FC8EC26F01200AA
:108A200029B912D028A110D02B95BEEC1DF0230E31
:108A3000B925A96EF9EC0BF0A8CF18F5A8CF58F11D
:108A40002A9D2789278B3AD02B85316B31C118F5A8
:108A5000259BB9C1D0F1B905040DF350070FA96EDC
:108A6000F9EC0BF0A8CF11F5B905040DF350060F82
:108A7000A96EF9EC0BF0A8CFCFF111C50AF1D8809F
:108A8000640E0A55A856A8CF10F52789278B16D053
:108A90001FAF12002CB943D02BB93CD025A908D068
:108AA0002AB531D023C5CDF1CD6702D0E3EC25F056
:108AB000B82B0A0EA6EC0EF0B86512002AA50DD050
:108AC0002A9559EC0DF065EC1DF08EEC23F024B1E5
:108AD0003EEC1AF024A107EC1AF02A951F9F1F9D67
:108AE000D2EC1DF0B6EC26F0E3EC19F0B6EC23F076
:108AF000B86B25992C99259B259D25952A9D2B9909
:108B000023972399120023C5CDF1CD67D1D7A7ECC8
:108B10002AF0CED798EC25F0C8EC26F0C9D78EEC19
:108B200029F0C6D729EE4AF0100E386FDE660DD058
:108B3000382FFCD759EC0DF0010E90EC09F0020E25
:108B400090EC09F070EC80F00101A9EC0CF01AEC4B
:108B50000CF0A46BA56B939C939E819C819E1FB58A
:108B600009D81FB14FD81FA9BEEF48F0000003007D
:108B70000000F5D789EC46F02BB14DEC46F021EC26
:108B80003BF014EC3BF0A52B0E0EA56526D070D85B
:108B9000A8EC47F01AEC80F00101A0C1A2F1A1C13C
:108BA000A3F18CC1A0F18DC1A1F1A56B070EBAECA8
:108BB0000EF031C151F132C152F1A0C153F1A1C146
:108BC00054F105EC0AF01EB701D007D0070EBAEC3D
:108BD0000EF031C1A0F132C1A1F18CC100F58DC1FF
:108BE00001F50B0EA6EC0EF00A6F0AC112F50C0E81
:108BF000A6EC0EF00A6F0AC113F540EC80F00101FB
:108C00001F9512005BEC3BF026A104D0818600008A
:108C1000030000008196A42B050EA46512D028D86D
:108C2000060EBAEC0EF031C151F132C152F18CC1D5
:108C300053F18DC154F105EC0AF01F891EB71F993D
:108C4000A46B1F9123B70AD023B908D0F292F090F9
:108C50002993299123992397D59E1200F292F0909F
:108C60002993299123992397D59E1F99268712002E
:108C700020EC17F00300000003000000030023ECC9
:108C800017F013EC17F003000000030000000300CE
:108C90001AEC17F0FBEC15F01200FA0E06EC0BF0D4
:108CA000FA0E06EC0BF0FA0E06EC0BF0FA0E06ECE0
:108CB0000BF089EC46F02BA11200F26AF16AF06A1F
:108CC000C2901AEC0CF0100E926E806A936A816A60
:108CD0001D0E946E826A956A836A966A846AD56A62
:108CE000CD6ACA6A9B6A020ED36ED180E7C136F1A3
:108CF0000F0E386F03000000382FFCD78188040066
:108D0000050EDAEC0AF0819803000000362FF6D742
:108D1000EDD7C2800000C282C2B2FED7C4CF4CF1F0
:108D2000C3CF4BF1C60E4D6F030E4E6F1CEC0AF015
:108D3000640E4D6F4E6B60EC0AF047C1C1F148C143
:108D4000C2F1C290C1C153F1C2C154F1280E516F9A
:108D50000A0E526F05EC0AF02B911EB703D0020EDB
:108D6000E76F2B818CC153F18DC154F1990E516F76
:108D70003A0E526F05EC0AF02B911EA703D0030E9A
:108D8000E76F2B81289B289D280ED0EC0BF0A8CFF5
:108D900053F1290ED0EC0BF0A8CF54F1D00E516F47
:108DA000070E526F05EC0AF01EA7288B940E516F28
:108DB000110E526F05EC0AF01EA7288D28AB6DD05E
:108DC00028AD6BD0680EA86E280ECEEC0BF0100EFE
:108DD000A86E290ECEEC0BF007C1A8FF2A0ECEEC30
:108DE0000BF006C1A8FF2B0ECEEC0BF008C1A8FFBC
:108DF0002C0ECEEC0BF096C1A8FF2D0ECEEC0BF096
:108E000097C1A8FF2E0ECEEC0BF0A86A2F0ECEEC69
:108E10000BF0300ECEEC0BF0310ECEEC0BF0320E30
:108E2000CEEC0BF0330ECEEC0BF0340ECEEC0BF0A0
:108E3000350ECEEC0BF096C1A8FF360ECEEC0BF043
:108E400097C1A8FF370ECEEC0BF007C1A8FF380E74
:108E5000CEEC0BF006C1A8FF390ECEEC0BF008C12A
:108E6000A8FF3A0ECEEC0BF096C1A8FF3B0ECEEC5D
:108E70000BF097C1A8FF3C0ECEEC0BF007C1A8FF8A
:108E80003D0ECEEC0BF006C1A8FF3E0ECEEC0BF073
:108E900008C1A8FF3F0ECEEC0BF0280ED0EC0BF073
:108EA000A8CF53F1290ED0EC0BF0A8CF54F1C1C1DB
:108EB00051F1C2C152F105EC0AF01EA71200C1C166
:108EC000A8FF280ECEEC0BF0C2C1A8FF290ECEECF5
:108ED0000BF007C1A8FF2A0ECEEC0BF006C1A8FFCD
:108EE0002B0ECEEC0BF008C1A8FF2C0ECEEC0BF035
:108EF00096C1A8FF2D0ECEEC0BF097C1A8FF2E0E49
:108F0000CEEC0BF01200800ECF6ECE6A3C0E0361E9
:108F100011D03C0E04610ED0180E05610BD0200E4E
:108F2000066108D00C0E076105D0640E086102D0FE
:108F30009D801200000E036F000E046F0C0E056F73
:108F4000010E066F080E076F0A0E086F9D80120053
:108F5000360ED0EC0BF0A8CF53F1370ED0EC0BF05F
:108F6000A8CF54F196C151F197C152F105EC0AF026
:108F70001EA719D096C1A8FF360ECEEC0BF097C1F4
:108F8000A8FF370ECEEC0BF007C1A8FF380ECEECD1
:108F90000BF006C1A8FF390ECEEC0BF008C1A8FFFC
:108FA0003A0ECEEC0BF03B0ED0EC0BF0A8CF53F109
:108FB0003C0ED0EC0BF0A8CF54F196C151F197C103
:108FC00052F105EC0AF01EB7120096C1A8FF3B0E45
:108FD000CEEC0BF097C1A8FF3C0ECEEC0BF007C116
:108FE000A8FF3D0ECEEC0BF006C1A8FF3E0ECEEC66
:108FF0000BF008C1A8FF3F0ECEEC0BF01200239B34
:109000009D9A81869E9A620EAD6E22EC0CF028EC41
:109010000CF0AECF05F1180E0561056B28EC0CF0D5
:10902000AECF04F13C0E0461046B28EC0CF0AECF23
:1090300003F13C0E0361036B28EC0CF0AECF07F19B
:109040000C0E076501D0076F28EC0CF0AECF06F1CF
:1090500007C131F1314F1F0E314F1C0E314F1F0E22
:10906000314F1E0E314F1F0E314F1E0E314F1F0E4E
:10907000314F1F0E314F1E0E314F1F0E314F1E0E3E
:10908000314F1F0E066502D0010E066F28EC0CF062
:10909000AECF08F1640E0861086B81969E9A1F8519
:1090A0009D8AA5EF3AF0010186EC49F01FB31DEC53
:1090B00019F0FC6A01EE09F0EE6A0A0EEA62FCD7CA
:1090C0001AEC0CF083EC47F029EC17F0229D22AD4E
:1090D000FED78E6B8F6B196B1A6B1F8938EC46F0BD
:1090E0001F998CC19EF18DC19FF18CC1A0F18DC1E2
:1090F000A1F18CC1A2F18DC1A3F1CB2B0A6B0AC1E6
:1091000011F54F0E0A6F0AC110F58CC100F58DC123
:1091100001F5000EE8CF4CF220EC80F0010130ECBC
:1091200080F0010118EC80F0010134EC3BF001010A
:1091300040EC80F00101010EA96E010EAA6EF9EC5F
:109140000BF0A8CF38F1A92AF9EC0BF0A8CF39F130
:10915000AA6A010E386304D0470E396301D00ED0DD
:10916000010EA96E010EAA6E010EA86EFDEC0BF0A9
:10917000A92A470EA86EFDEC0BF0AA6A8198819689
:10918000300EA6EC0EF0E8CFF8F11E6B1F6B206BD3
:10919000216B226B236B246B256B266B276B286B53
:1091A000296B2A6B2B6B2C6B33EC38F097EC0DF0A2
:1091B000000EE8CF7CF0000EE8CF7DF0000EE8CF87
:1091C0007EF0000EE8CF7FF0FF0E2D6F2DC17AF0FC
:1091D000FF0E2D6F2DC17BF0BFEC2CF0A2C19EF1D4
:1091E000A3C19FF1AA6A5C0ED0EC0BF0300EA8620E
:1091F00001D006D00ED8300EA86E5C0ECEEC0BF06F
:10920000270ED0EC0BF02985010EA862299530EFCE
:109210003AF006EC29F0140E65D0279F2891299B7F
:10922000000E0A6F0AC11FF55A0E0A6F0AC115F522
:109230000AC114F5AA6A220ED0EC0BF0010EA86246
:1092400002D0278F1200020EA86202D028811200DD
:10925000030EA86202D0298B1200040EA8620FD060
:10926000010E0A6F0AC11FF5200EA6EC0EF0A8CF62
:1092700015F5210EA6EC0EF0A8CF14F51200050E80
:10928000A86212002881010E0A6F0AC11FF5200E84
:10929000A6EC0EF0A8CF15F5210EA6EC0EF0A8CF87
:1092A00014F5120059EC0DF0C4EC28F00A0E386FDA
:1092B000C80E06EC0BF0239723991FB108EC42F07F
:1092C0001FB138071F91386701D012001FB3120079
:1092D00023B7120023B91200F0D759EC0DF0E5ECDA
:1092E00028F0E4D7386FC80E06EC0BF023972399CB
:1092F0001FB108EC42F01FB138071F91386701D049
:10930000120023B7120023B91200F2D76C0ED36EED
:10931000110E926E806A030E936E816ADD0E946E5A
:10932000826A000E966E846A000E956E836A400E05
:109330009B6E1F0ED56E070ECD6ED00EF26E050E13
:10934000F16E080EF06E210E9D6E000EA06ED06ABA
:10935000000EC26E0E0EC16E8A0EC06EC66A000E80
:10936000C76E280EC66E000EC56E080EC86EBD6AAA
:10937000BA6A070EB46E200E6F6E240EAC6E900E9D
:10938000AB6E080EB86EB06A220EAF6EAE6A9E6A01
:109390001200010EE86F0F0EE96F010EB96FB76B87
:1093A0001F8F2087E0EC0DF059EC0DF019EC1DF04B
:1093B0002397239920912093CFEC1AF0FCEC1BF01B
:1093C00055EC11F01FA109D025EC3CF008EC42F05F
:1093D0005BEC3BF089EC46F01F9120B1FAEF49F0CD
:1093E0001FAF04EF4AF01FB904EF4AF01FB3BEEFFE
:1093F00048F0E6D7B94F1CD0B94F0AD0B94F10D0BA
:10940000B94F6FD0B94F37D0040EB96F7CEF11F060
:10941000020EE827C70EE861E86F020EB96FC8D7E1
:10942000030EE927630EE961E96F030EB96FC0D738
:10943000248D2B87E9C14BF14C6B640E4D6F4E6B45
:109440001CEC0AF0E80E4727030E482347C1C5F17C
:1094500048C1C6F1C5C18CF1C6C18DF120912093E0
:109460001F9F23972399DBEC4AF01F83500EEDECEE
:1094700018F031EF3CF059EC0DF0EAEC2AF047EC33
:1094800044F00BEC0CF002EE50F0200E0A6FEECF21
:10949000ADFF22EC0CF00A2FFAD7010EE8CF7FF0D7
:1094A000BC0E90EC09F0000EE8CF7FF023972399D3
:1094B0001FA109D025EC3CF008EC42F05BEC3BF03E
:1094C00089EC46F01F9123B709D023B907D01FB903
:1094D0007AEF11F01FB3BEEF48F0EAD7050EB96F6F
:1094E0005ED753EC42F0248D2B87E9C14BF14C6BD6
:1094F000640E4D6F4E6B1CEC0AF0E80E4727030E0E
:10950000482347C1C5F148C1C6F1C5C18CF1C6C1E8
:109510008DF1DBEC4AF0010EE8CF7FF00C0E90EC01
:1095200009F0000EE8CF7FF043EC3DF0E1EC3DF0B8
:1095300000EC80F0010123C5CDF1CD67F5D7010E18
:10954000E8CF4CF2FF0EE8CF23F5CFEC1AF081788C
:1095500043EC3DF0E1EC3DF000EC80F00101430E06
:10956000EDEC18F0E82FF1D7000EE8CF4CF2FF0E2B
:10957000E8CF23F514D08188E6EC4AF0249D2B97A0
:10958000FA0E06EC0BF0FA0E06EC0BF0FA0E06ECF7
:109590000BF08198010EE86F050EB96F00D743EC10
:1095A0003DF0E1EC3DF000EC80F0010123C5CDF190
:1095B000CD67F5D7E0D72C81530EEDEC18F062ECB7
:1095C00080F00101540EEDEC18F012002C91530EB6
:1095D000EDEC18F064EC80F00101540EEDEC18F0A5
:1095E000470EEDEC18F030EC80F00101FBEC3FF0A1
:0E95F000480EEDEC18F028EC80F0010112009E
:109A0000AF9BAFAFAFAFD1AFB205B007B008AF09F2
:109A1000AF09AF09AF09B108B2079B049F9F9F9F91
:109A2000AE9FFFFFFFFFFFFFFFFFFFFFFFFFFFFFF7
:109A3000FFFFFFFFFF8F82FFAC04A1149B1A96204B
:109A400092248F288A0E8C10940B8A0C9609870F0B
:109A5000960885129707830785079706850783076A
:109A600096068708820796058A07810696058C0761
:109A7000810594058E088005940490078005930461
:109A80009107800591049208800590049407800551
:109A90008E05950780058C05960880058A06960830
:109AA000820588069707820685079708840683073C
:109AB00097088507800898078707970F8908950DED
:109AC0008B0A8C108E0E912894269922A01CAA1520
:109AD0009707FFFFD7FFB701B403B404B403B4047E
:109AE000B304B304B305B205B206B205B2068136BB
:109AF0008137813781378137FF37FFFFFFFFACFFA9
:109B0000FFFF90FF8903A8008705A5038607A3052B
:109B10008508A007840A9F08840B9F06830D9F0673
:109B2000820E9F06810882049E05830882049E049B
:109B3000840881049D05850881049C0587078104AC
:109B40009C04880781049B04890781049A048A077E
:109B5000810499048B07810498048C07810496057D
:109B60008D07810495058E07810494058F07810474
:109B70009206900782049006910782048E0792074E
:109B800083048B07930883048609940A8404951937
:109B900085049617860498148704991289049B0EED
:109BA0008C049D08B305BA05FFFF8EFFB7008A023B
:109BB000A8018804A5038607A3058608A5058407D0
:109BC000A7058406A8058206AA058205AA058105BF
:109BD00091059504800591059504800591059504EE
:109BE00080059204950480059204950480059204F2
:109BF00095048005920494058005900594068005DF
:109C00009005940680058F05920882058E059208BE
:109C100082058C06900A82068A078E0C84068707C6
:109C200081068C06850781158907870883138918A3
:109C300085118B16870F8D148A0C91128E07AC0E2E
:109C4000FF0AFFB88BFFB205B006AF08AD09AC0B39
:109C5000AA0CA90E8107A7058208A6058407A405FA
:109C60008607A3058707A10589079F058A089E0522
:109C70008C079C058D089B058F0799059008980512
:109C80009207960594079505950793059707920502
:109C9000813581378137813781378137A437B305E3
:109CA000B305B305B305B305B3058F05FFFF8CFFFF
:109CB000A20192009203901085058F1C84078E1DCF
:109CC00083088E1D8308911C8207931B82068E05D4
:109CD000950581068E05970481058E0597048105FB
:109CE0008D05980580058D05990480058D059904DD
:109CF00080058D05990480058D05990480058D05E5
:109D0000990480058D05990480058D0599048005C9
:109D10008D05990480058D05970581058D059705AD
:109D200081058E05950581068E05930682068E05B2
:109D3000910782078F058D0883089005870A830B9A
:109D40009105841C9205851A930586189405A5151E
:109D5000AA11C50CFFFF11F11BA2219A269429908C
:109D60002B8E0D8C05850E850B880588098B088840
:109D70000689088E0786058B07910784058B069355
:109D80000683058C06950582058D05960681048D52
:109D900006970580058D05980580058D059804803A
:109DA000048E0B99048E0B99058E0B98058E0B98DB
:109DB000058E05980480068E05960481058F05960C
:109DC0000581068E05940582078F07900583098E0D
:109DD000088C07840B8D0A8607851B8E05871990D2
:109DE00003891792008B13960FA707ADFFC8FFFFDB
:109DF000059605B305B305B305B305B301AF0581FA
:109E000004AC058107A905810AA605810CA405817A
:109E10000FA10581129E0581139B0583139805866A
:109E2000129605891293058C1290058F118E05925A
:109E3000118B0595108905981086059B0F84059E4A
:109E4000108115A012A310A60DA80BAB09AD06AF8B
:109E500004B2A7FFFFFF03CA0BB10FAB0790118F2E
:109E60000C8D148A0F8A1688118818861486078428
:109E7000088715850683078B068408860681068D6C
:109E8000068307890480069005820C8B0591058165
:109E90000A8D05920481088F05940480069005952B
:109EA000048006900B9505910B9505910B950592F5
:109EB0000B94069105940480079105930580088F03
:109EC000049305810A8E059106810C8C068F06820B
:109ED00006890681058E088308850781068C15840E
:109EE0000883078813860A850A82118716870F89D7
:109EF00014890C8B128C068F10900CAA06AFFFC52C
:109F0000E9FFAC09980F8D0095138A029217880417
:109F1000901986068E1B850788098F0A83068D088F
:109F20009007820590078F078205930690058005AC
:109F300094068F06800596058F05800597058F048A
:109F4000800598048F04800598048E05980B8E0573
:109F5000980B8F04800598048E04810597058E0464
:109F6000810596058D05810695068E048305940569
:109F70008D05830693068D04850690078B0586075D
:109F80008D098A058808880B8706890C8C2D8F2BF4
:109F9000932796249D1FA917D30700FFFFFFFFFFFC
:109FA000000022003500D2000001A8014302AC02EB
:109FB0005403ED035404FF049A0500EE00F00D0E67
:109FC000EE6AEA62FDD71200FFFFFFFFFFFFFFFF0F
:109FD000FFFFFFFFFFFFFFFFFFFFFFFFFFFFFFFF91
:109FE000FFFFFFFFFFFFFFFFFFFFFFFFFFFFFFFF81
:109FF000FFFFFFFFFFFFFFFFFFFFFFFFFFFFFFFF71
:10A0000000000F0016006B008300DC002D016601CC
:10A01000C10116024C02AB0202031B032A034403D4
:10A020006F0375039F9F03BA049A059A0499039BD3
:10A030009F9F9FC0BF9F9F7FBF9F03CD0E96128E95
:10A04000168A0487078B0385038C04800383048BA3
:10A0500004820282048B03840281038B02870281C3
:10A06000038A028802810488038902800387028BA5
:10A0700003810385028C03820482038C03830480A2
:10A08000038C0685048C168713890E8E0395FFCDED
:10A090000084019E029C029B029C039B029B1D9BD1
:10A0A0001D811D81FFFFFCC0850194008403910286
:10A0B0008305900382069003820790028103810248
:10A0C0008F02820481028E02830481028D02840445
:10A0D00081028D02850381028C02860381028A033C
:10A0E000870382028802880482028603890483022D
:10A0F0008A0D84028C0A85028D0887029003E00293
:10A100009AFF8501920283049303820495028203DD
:10A110009602810289028A02810289028A028102F0
:10A1200089028A02810289028A02810288028A03E4
:10A130008202870289048202850387068303810ADB
:10A1400084038404810A870C84068A0A8802FF0734
:10A15000D3849A0299049705960781039402820496
:10A160009302840391028504900287038E0288047F
:10A170008D028A038B028B048A02811C811D811D42
:10A18000941D9C029C029C02C80200FA068D028863
:10A190000F8304870F82038809820281038A028168
:10A1A0000287028C02810287028C02810187028D64
:10A1B00002810187028E02800187038D028002875F
:10A1C000028C02810287028C02810387038A02814A
:10A1D0000388048802810588058402820E8902832F
:10A1E0000C8A0894ECE591088B1188158517840575
:10A1F0008602840585038902830386038A0281031C
:10A2000086038C02810287028C02810287028D0202
:10A21000800287028C02810287028C0281028702FF
:10A220008B038102880289038302870284058305E8
:10A230008703850E8A00950CE60680FF9C029C022F
:10A240009C029702810294028105910281088F028B
:10A2500082098C0285098902880987028B08840299
:10A260008D0982029008930B950998069A04FC01C7
:10A2700005F4038A088807870A8509850483058110
:10A280000B8303810485028206850388028105878A
:10A29000028902810388028A02810388028A02817C
:10A2A0000289028A02810388028A02810488028963
:10A2B00003810686028803820383038102860B835F
:10A2C0000581048208840B84058709860597E7E5E4
:10A2D00098048B098600890C8402880E8203880307
:10A2E000880382028A02870381028C02870281022C
:10A2F0008C02870280038C02870281028C02870213
:10A3000081028C02870281028A0387028203890309
:10A3100086028303870485028504810781038708F9
:10A320008A168F12E90C9F9F03AB038A048B048962
:10A33000048B0589048A0489028C038B9F9F9FC02C
:10A34000C89F9401940A940A96089F05B99FA9FF93
:10A350009B009403940A95099806FF0302830A94CC
:10A360000A9407940497BAFF15C815891589028BBA
:10A37000019B019C019D029D049C159A148A138BDC
:10A38000028A029B019C019D029D159C1589148ADD
:10A39000118DFFA0FFFFFFFF00FF00000E001B005C
:10A3A00048007D00B400E700F0000D012A014B01D8
:10A3B0006401700185018E01A301D601E20115023D
:10A3C000460267029C02CB02EA02210352036003A9
:10A3D00071039C03CD03F8031B045C047D04B804E3
:10A3E000E5040E05410564059705AC05CD05EA05B4
:10A3F0000F0624063D0656067F06A406D50600076E
:10A40000390752076B0784079D07C607DF0718083F
:10A4100037084C086B087C089508A108D408F9088F
:10A42000200945097A099B09E409F909140A330A44
:10A43000540A710A8A0A9F0AC80AED0A120B270BEE
:10A440005A0B770B8C0BA50BBE0BE30B040C390CD2
:10A450005C0C630C860C9F0CAD0CD60C050D2A0D04
:10A46000610D6C0DAB0DB80D050E3C0E5D0E700E42
:10A47000730EBA0ECB0EE40E150F3C0F610F6B0F6F
:10A48000860F8A0FDB0FE20F03F8018A0C85028228
:10A490000A85028394FF00CD0591039101C70591C0
:10A4A00003919DDA83018F0183018F018301880667
:10A4B000870D81078F0183018F0183018F01820145
:10A4C0008607890D83058F0183018F018301A20017
:10A4D00002B40186048A0186018802810185008810
:10A4E000018300860287028201851285018502842C
:10A4F000018400870185018301880284018201892A
:10A50000058403929A9F9203880585018301850142
:10A51000860283018400890282058B0382039202F2
:10A5200082028C02830289048402820186018503EF
:10A53000830186008701820191019D0403A4069195
:10A5400004880281028208860185008602840185D2
:10A5500000860384018401860582018306860282C7
:10A560000180038803850294069201900082FF9D7A
:10A570000194069002918BFF07E70C8C03890387F7
:10A580000286028B0184028E018201910181029177
:10A5900000800093B0B093008100910181018F028F
:10A5A00082028D0284028B028602870389038D0B4F
:10A5B000E707009F019601950282009002810491B5
:10A5C000078D078F04940092028101900183018F0F
:10A5D0000095A0A6950195019501950191018B0A21
:10A5E000900B9501950195019501A40188FF8201C9
:10A5F0008F0190069404FC0001B801950195019526
:10A60000019501950195019501950195FFBC018783
:10A610000295029494FF01C1039304900490049066
:10A6200003900391039103910193A0C490028B0ABC
:10A6300085028903860187058601830186018600DC
:10A6400084018601840085028601820186028601DA
:10A6500080028701880184048B03900AA30201CA47
:10A66000019501941095108694FF00B3018B01872A
:10A670000389018604890186028801800086018899
:10A68000018200860187018301860185018402869B
:10A69000018301850687018604880187BFB488018C
:10A6A0008B0087018C01860185008501860185006C
:10A6B0008501860185008501860183018502860169
:10A6C000810280018301880182049205B70300A4FE
:10A6D0000294049202910180028F0182028E018312
:10A6E000028C0185108B1086029001940096B7A110
:10A6F0008501880083088702820285018701840022
:10A700008700860184008700860184008700860117
:10A710008400860186018400850187018500870801
:10A720008600B60608B50C8C028901820283018777
:10A7300001830186018601830186008600840187EA
:10A7400000860184018601860283018401870884D2
:10A75000058FB1B7960096008D0086018A008604A9
:10A760008700880585008B0482008D059006930381
:10A77000C30104BB04890682028702800180018331
:10A780000187028301850086018501850086018598
:10A790000185018602830185028601810180018392
:10A7A0000588068102890484B3B68605880084077B
:10A7B0008701840284018601860184008601870066
:10A7C000830186018700840086018501830187015A
:10A7D0008402820188028B0DB80901FE0186028C79
:10A7E0000285028B028594FF01FF018601820286A9
:10A7F0000685028704850094A0FC950193029303CB
:10A80000810091018101900183018F0184018D01FB
:10A8100085018D0186018B0187018B0188018901EA
:10A8200089019E01009E00840090008400900084B5
:10A8300000900084009000840090008400900084C8
:10A8400000900084009000840090008400900084B8
:10A85000009000849AA189018A0188018A018701F8
:10A860008C0186018C0185018E0184018E0183019A
:10A870009001810192018100920194039402A4014C
:10A8800001B101950194019501940188028201842E
:10A890000486028101850284018402860282068F79
:10A8A00004919DBF8D0781048A04870288028B0171
:10A8B0008701840183038700840082058601830069
:10A8C0008201820186018300840082008601820168
:10A8D0008400820086018102830082018701820A4E
:10A8E0008A00A10802A70491048F068F048D0182BB
:10A8F000038B0185048C0183048F018005910494EE
:10A9000004950294999C8610861085008501860125
:10A910008500860086018500860086018500860008
:10A9200086018500850186018301850286018301F8
:10A9300084028702800581028902820393059F02B7
:10A94000069E0A8E038A0385018902890187028B8C
:10A950000086018D0086018D0086018D0186018CA7
:10A960000186018B028802880089008A999E8610E0
:10A9700086108D0086018D0086018D0086018D0078
:10A9800086018C0186018C0186018A02880186037A
:10A990008B028E0AA20510B1108600860185018502
:10A9A0000086018501850086018501850086018577
:10A9B0000185008601850185008601850185008667
:10A9C000018501850086018DB1B486108610850051
:10A9D0008E0185008F0085008F0085008F00850027
:10A9E0008F0085008F0085008F00C400069E0B8DB0
:10A9F000028A02870288018A0187018C0086018D04
:10AA00000086018D0086008701840186008601840E
:10AA10000186008600840288068400890585B19E2F
:10AA200086108D10950195019501950195018E0176
:10AA30008610B41000B1008E0086018D0086018D55
:10AA40000086018D108610860086018D0086018D9E
:10AA50000086018DBFCC9601950186018D0086018F
:10AA60008D0086018C008701870F890D9600960066
:10AA7000AC0010991086028D02930493029102801B
:10AA8000028F0282018D0385018A02880188038A70
:10AA90000086018D0096B19C861095109501950158
:10AAA00095019501950195019501B40110991086C4
:10AAB00003870395039503950293029203920391F2
:10AAC00010921086999C8610861095039502950326
:10AAD0009503950395039502870386109C10089DA6
:10AAE0000C8C028903870187018B0187018C00860A
:10AAF000018D0086018D0186018C0186018B028803
:10AB000002880C89088CB1A08610861086008E0001
:10AB100086008E0086008E0086008E0084018E01E5
:10AB200084018E0182028F029206A702089D0C8C7E
:10AB3000028902880187028B0186018C0086028EC1
:10AB40000084048E0182018C01810182018C0181CB
:10AB50000283028801820C8401830886B1A08610DA
:10AB6000861086008E0086008E0086008E0086008D
:10AB70008D0184018B04840180018903830788038C
:10AB800086058A028A009C0003B302860588018636
:10AB90000187028201860186018301860086018584
:10ABA0000185008601850185008601850185018674
:10ABB0000185028302860284028101880585019352
:10ABC00099A0960096009600960096008610861032
:10ABD0009600960096009600AC000C990E8A02959D
:10ABE00001950196019501950195019402940E87B6
:10ABF0000C8899A0950194049405940594059205F8
:10AC00008F048F048F048F049204AB0105990A927C
:10AC100009920490058E048E05900694069406927F
:10AC20000989068AA9A686008B0186028803880303
:10AC300084038B0381038F0391058F0581038C03AC
:10AC400085028803870387038B0196029C00009985
:10AC500002960395039503950A94098D048B04903D
:10AC6000039002920094A9AC86008C0086028A00B0
:10AC700086048900800286018700810386018500A1
:10AC80008303860184008502860182008603860193
:10AC90008000880386018A0386018B0295019C014E
:10ACA00015DF0181019101810191018101910181F2
:10ACB0000191018101910181019100820091B0B265
:10ACC00095019503950395039503940495049503C5
:10ACD0009503B30100B000910182019101810191BE
:10ACE0000181019101810191018101910181019114
:10ACF0001581CEE19401920292029402960295028D
:10AD00009503D60100AB009600960096009600963B
:10AD1000009600960096009600960096E09A95019F
:10AD2000950395029502FF00A68993018C04830187
:10AD300080018B02830082018A01830184008A00E2
:10AD4000830184008A00830184008A0083018300D8
:10AD50008C00820182008C018C0BB40A12AF11842A
:10AD6000018C0186008C0188018A0188018A018892
:10AD7000018A0188018B0286038B0283088D04906F
:10AD8000B8A08F068D0884028C0286018A02880191
:10AD90008A0188018A0188018A0188018B01860164
:10ADA0008C0185028D01A60004A10890028D028409
:10ADB000018C0286018A0188018A0188018A018842
:10ADC000008B0088018C018611861284A2B4920245
:10ADD0008E0780048C03810182018B018201830133
:10ADE0008A01820183018A01820183018A01820131
:10ADF00083018B01810183018B0182058D01830415
:10AE0000B50001B601950195109003850181018F70
:10AE10000183008F0184018E0184018E00840190E2
:10AE20000295AAAB8902810480018704810B860107
:10AE300083018101830186008500820083008501F2
:10AE400085008200830085018500820083008501E2
:10AE500083018201830086018305830086008405C7
:10AE600081018601890087048B009A0112AF128448
:10AE7000018C019400950195019502950B950A8C22
:10AE8000CDB488018A0188018A0188018501820187
:10AE9000850C8201950C95019501CC0101C40196A8
:10AEA0000185018D0185018D0185018D0185018C53
:10AEB0000181108202810F810182AFDC84128F1226
:10AEC0009402940192038001900282018E02840117
:10AED0008C0286018A03890096019C0000B0018ED5
:10AEE0000184018E0184018E0184018E12841284FA
:10AEF00001950195019500969DB48A0C8B0C9500E7
:10AF0000950195018B0C8B0B9401950195018B0C90
:10AF10009C0B0CB50C8A018C019400950195019550
:10AF200002950B950A8CA1B491048E0782028C03C2
:10AF300086018B0188018A0188018A0188018A01C2
:10AF400088018B0186018C0183038D029008A00487
:10AF500011B5108501870186008C0088018B01885E
:10AF6000018A0188018A0188018B0286028B028492
:10AF7000088D0490A1A090048D0883028C038700A3
:10AF80008A0288018A0188018A0188018B01880070
:10AF90008C0086018C01860FAF110CCD0C8A018CC0
:10AFA0000194009501950195019501960095B8A72A
:10AFB00085008C0183048C0184048A018201830151
:10AFC0008A01820183018A01820183018A0183014E
:10AFD00082018B01830082018B0182018D05830038
:10AFE000B60301B5019501950E920F88018A01887B
:10AFF000018A0188018A0188018A01880194B5B516
:10B000008C0A950B950296019600950095008B0190
:10B010008A0CB40C009D0396049404950494049443
:10B020000393039103910490039000939DA89305CB
:10B03000930893058F038F04920495039405930559
:10B040008C038B09A20601B50188028A0286028C54
:10B050000382028E02800491049202910280028E89
:10B060000383028B0286008A0189ACB486018C02BC
:10B0700085018905880187048A0184048E0191076E
:10B080008F0490048F0490049303A70100A9018A00
:10B090000287018A0386018A0485018A028401806D
:10B0A000018A02820182018A02810183018A02806F
:10B0B0000184048A0185028A0187018A0188019539
:10B0C000A29C960095019301810586028107830861
:10B0D0008A06810291018101920181009201810021
:10B0E0009201C80090FF8115FF15C8909201810060
:10B0F0009201810092018100910182018506810106
:10B10000830381078A0881058F019501BA01009F99
:10B11000019501950194019501960295019501957E
:10B12000019501940195F8A6890185048103850C98
:10B130008302FF0AA19491028E0782038C03860189
:10B140008B0188018A0186008607860E84088701A4
:10B15000810088018A0187018B028601B60100A95E
:10B16000018C0186048902850E8702870682018090
:10B170000187018300860087018401860086018D96
:10B180000186008D0186008D01950195B49C860095
:10B190008E008F0882018F0184018F0084018E014F
:10B1A00084018E018401900082018F018E08860047
:10B1B000B90001B100870081038901840081038BFC
:10B1C00001820081028D018100810A8F0A8C038A2D
:10B1D00001800081038B0182008103890184008149
:10B1E0000189018600810089FFAC099008820981EC
:10B1F000088290FF02B800850486048002830784D9
:10B20000018101840184018201830184018201831F
:10B21000018301840182018401820184008301840D
:10B2200001830182018402840780018504830480F4
:10B23000018EC8BB94019502C50194019502DC0101
:10B2400002890791018E0285018B02820082008BA8
:10B2500005810082018900810183008100890181CB
:10B2600001840080008901810184008001890180BE
:10B2700000840081008A018101820081018A0081AD
:10B280000185018B0186028D02820490BC898F01A9
:10B2900081038A01810181048A0182008101800188
:10B2A0008A018200820080018A018200820080017E
:10B2B0008A018101810081018A0181088B01810756
:10B2C0009501B80101BA03940292018002900182B3
:10B2D000018F018401910394029201800290018206
:10B2E000018F0184D0B6950190018B0C8D0A8F08D7
:10B2F000910693049502BC00FFFF89CF91028E074F
:10B3000085018B0288018B00800081078900800104
:10B310008107890081008200840089008100820009
:10B32000840089008001800182038A0081008102FB
:10B3300081018A0088018B0186018D0182029002C1
:10B34000890400C900960096009600960096009623
:10B350000096CBDC930191058101900183018F015F
:10B3600083018F01830191009205D803009F00871C
:10B37000008D0187008C0187008C0187008C01877C
:10B380000B8701810B870181008C0187008C01876D
:10B39000008C0187008C0187008C0087CA9D860085
:10B3A0008D0084018C0284018C03840180008C0157
:10B3B000830180018C01820181018D0182048E0153
:10B3C0008302D30100D1018E0184018D0186018C9D
:10B3D00000820182018C00820182018C0181018244
:10B3E000058D0180018F0381FFD4019103930193A7
:10B3F00000959DF68511950B960195019501950196
:10B4000094008B02950B9502950195018500FFFF35
:10B4100080CE0195029403920491008604890386EC
:10B4200005870286068504860782048709800F86C1
:10B4300007870780068706800788058008870381BD
:10B4400007880180018106880580058907800488B6
:10B450000A8003860C8002850C8001860B800C8894
:10B46000088B8F8BFFFFFFFF90EC5BF0120000005A
:10B47000849083C083FF80948084120085C000F094
:10B48000016A00C086F084C087F0848086C083FF94
:10B490008094808487C083FF8094808412008EC053
:10B4A00083FF809480848094808412007AC083FF1C
:10B4B000809480847BC083FF80948084120000018C
:10B4C000350E836FD5DF00017D510001846F856BE0
:10B4D0000001D89084378537D1DF0001360E836FA5
:10B4E000C7DF00013F0E846F010E856FC7DF0001CB
:10B4F000370E836FBDDF00017C510001846F856BC7
:10B50000020E00017E5D07E13A0E00018427000E65
:10B510000001852310D000017E0507E1200E000107
:10B520008427000E0001852306D0180E0001842711
:10B53000000E0001852300018407000E855B0001D9
:10B54000EF0ED8808455000E855504E2EF0E000101
:10B55000846F856B7CC000F000C001F0006A005071
:10B560000001841301500001851388DF0001200EC3
:10B57000836F7EDF00017C510001846F856B7EDF6D
:10B580000001210E836F74DF00017D510001846F83
:10B59000856B0001D8908437853770DF1200200E4C
:10B5A0000001825D03E10001B60E826F000182514D
:10B5B0007E0803E2220E0001825F210E0001825DFF
:10B5C00004E300018251A30803E20001820E826FAE
:10B5D000210E0001825DF66EF76AD890F636F736D6
:10B5E0009A0EF626A30EF7220900F5CF88F00A007E
:10B5F000F5CF89F000018229DF0FF66EF76AD89047
:10B60000F636F7369A0EF626A30EF7220900F5CF86
:10B610008AF00A00F5CF8BF01200270E0001825D40
:10B6200003E100013B0E826F220E0001825D03E107
:10B6300000013C0E826F6D0E0001825D03E100018E
:10B640003D0E826F200E0001825D03E100013E0E7F
:10B65000826F2E0E0001825D04E3000182513E08DC
:10B6600003E200013E0E826F2E0E0001825DF66E37
:10B67000F76AD890F636F736000EF626A00EF722B7
:10B680000900F5CF88F00A00F5CF89F00001822982
:10B69000D20FF66EF76AD890F636F736000EF62619
:10B6A000A00EF7220900F5CF8AF00A00F5CF8BF043
:10B6B0001200200E0001825D03E100012F0E826F57
:10B6C0002E0E0001825D04E300018251390803E27D
:10B6D00000012F0E826F2E0E0001825DF66EF76A5A
:10B6E000D890F636F736A00EF6269F0EF722090000
:10B6F000F5CF88F00A00F5CF89F000018229D20F3A
:10B70000F66EF76AD890F636F736A00EF6269F0E3C
:10B71000F7220900F5CF8AF00A00F5CF8BF012006E
:10B7200000017C51006E016A013404E20050E60819
:10B73000000E015403E20001E60E7C6F00017D5112
:10B74000006E016A013404E200509B08000E0154AF
:10B7500003E200019B0E7D6FB2DE0001220E836FBB
:10B7600087DE84800001816B00018151EA6A600FED
:10B77000E96E000EEA22EFCF82F00001825106E16D
:10B7800000013A0E826F0001190E816FF86A000104
:10B79000825101E1DCD01A0E0001815D01E3D7D0B6
:10B7A000020E00017E5D02E184DF06D000017E050D
:10B7B00002E133DF01D0F3DE00018E6B88C08CF034
:10B7C00089C08DF000018A5100018C5D00018B5110
:10B7D00000018D5901E3AFD0020E00017E5D1DE135
:10B7E0008CC0F6FF8DC0F7FF010E0F0B05E0D8905F
:10B7F000F732F632E806FBE1010ED890F636F7365E
:10B80000E806FBE1000EF6269A0EF7220900F5CFB6
:10B8100084F00A00F5CF85F03CD000017E051DE1E3
:10B820008CC0F6FF8DC0F7FF010E0F0B05E0D8901E
:10B83000F732F632E806FBE1010ED890F636F7361D
:10B84000E806FBE1240EF626A00EF7220900F5CF4C
:10B8500084F00A00F5CF85F01CD08CC0F6FF8DC0B7
:10B86000F7FF010E0F0B05E0D890F732F632E8062D
:10B87000FBE1010ED890F636F736E806FBE1880EBC
:10B88000F626A40EF7220900F5CF84F00A00F5CFC2
:10B8900085F000018C51010B05E00001845100018D
:10B8A000806F05D085C000F0016A00C080F0000103
:10B8B0008051006E016A0050800B1DE07F0E000178
:10B8C000805F00017F5109E000018051000804E21F
:10B8D00000018007EBDDF8D70DD08EC083FF00019B
:10B8E0008051000807E200018007809480848094E2
:10B8F0008084F5D71BD00001802B00017F510EE022
:10B900008EC083FF00018051000807E2000180071C
:10B910008094808480948084F5D708D00001805181
:10B92000000804E200018007C1DDF8D700018C2B7C
:10B93000000E8D2347D70001812B00018151EA6A57
:10B94000600FE96E000EEA22EFCF82F020D70001EF
:10B95000836B8EDD1200FFFFFFFFFFFFFFFFFFFF86
:02B96000FFFFE7
:10C000000901306B316B326B336B3451040B04E03C
:10C01000080E346F356B03D0040E346F356B366BFE
:10C02000376B386936C4B5F937C4B6F938C4B7F9CF
:10C0300039C4B8F93AC4B9F93BC4BAF93CC4BBF93C
:10C040003DC4BCF91FC583F91EC584F90EC485F92A
:10C050000FC486F910C487F911C488F997C289F909
:10C0600098C28AF999C28BF99AC28CF99BC28DF950
:10C070009CC28EF99DC28FF99EC290F9F3C591F9C9
:10C08000F4C592F9F5C593F9F6C594F9F7C595F994
:10C09000F8C596F9F9C597F9FAC598F9FBC599F964
:10C0A000FCC59AF9FDC59BF9FEC59CF95FC99DF9D0
:10C0B00060C99EF961C99FF962C9A0F963C9A1F974
:10C0C00064C9A2F965C9A3F966C9A4F96FC9A5F93C
:10C0D00070C9A6F971C9A7F972C9A8F977C9A9F9F0
:10C0E00078C9AAF979C9ABF97AC9ACF97BC9ADF9B4
:10C0F0007CC9AEF97DC9AFF97EC9B0F97FC9B1F984
:10C1000080C9B2F981C9B3F982C9B4F905011F51D7
:10C1100002E0090130812C6A2D6A2E6A2F6AF3C56C
:10C1200027F0F4C528F0F5C529F0F6C52AF0C2ECD1
:10C130006EF0010A02E009013083100E0901BE6FA2
:10C14000BF6B200EBFAF02D0D89003D0BE5D000EF3
:10C15000BF592DE2BEC9E9FFBFC9EAFFD890E93651
:10C16000EA36D890E936EA36800EE926040EEA224D
:10C17000EECF00F0EECF01F0EECF02F0EFCF03F004
:10C180002C6A2D6A2E6A2F6A00C027F001C028F0A1
:10C1900002C029F003C02AF0C2EC6EF0010A02E0EE
:10C1A000090130850901BE2B000EBF23CAD72C6AB6
:10C1B0002D6A2E6A2F6AF7C527F0F8C528F0F9C551
:10C1C00029F0FAC52AF0C2EC6EF0010A02E009017A
:10C1D0003087A40E2C6E700E2D6E7D0E2E6E3F0ECF
:10C1E0002F6E77C927F078C928F079C929F07AC964
:10C1F0002AF0D2EC6EF0010A02E109013089660EE4
:10C200002C6E2D6EA60E2E6E3F0E2F6E77C927F068
:10C2100078C928F079C929F07AC92AF0C9EC6EF0FA
:10C22000010A02E10901308B5C0E2C6E8F0E2D6E1F
:10C23000420E2E6E3E0E2F6E97C227F098C228F047
:10C2400099C229F09AC22AF0D2EC6EF0010A02E1FA
:10C250000901308DAE0E2C6E470E2D6E810E2E6EA6
:10C260003F0E2F6E97C227F098C228F099C229F08E
:10C270009AC22AF0C9EC6EF0010A02E10901308F7E
:10C280009A0E2C6E990E2D6E190E2E6E3F0E2F6E7D
:10C290009BC227F09CC228F09DC229F09EC22AF0C2
:10C2A000D2EC6EF0010A02E109013181AE0E2C6E72
:10C2B000470E2D6E810E2E6E3F0E2F6E9BC227F005
:10C2C0009CC228F09DC229F09EC22AF0C9EC6EF0F3
:10C2D000010A02E1090131833AC42CF03BC42DF07C
:10C2E0003CC42EF03DC42FF036C427F037C428F0EC
:10C2F00038C429F039C42AF0F8EC6CF027C000F0FB
:10C3000028C001F029C002F02AC003F0330E2C6EC1
:10C310002D6E730E2E6E3F0E2F6E00C027F001C0E3
:10C3200028F002C029F003C02AF0C9EC6EF0010A1F
:10C3300002E1090131853AC42CF03BC42DF03CC424
:10C340002EF03DC42FF036C427F037C428F038C48F
:10C3500029F039C42AF0F8EC6CF027C000F028C0AE
:10C3600001F029C002F02AC003F0CD0E2C6ECC0ED5
:10C370002D6E4C0E2E6E3D0E2F6E00C027F001C0AC
:10C3800028F002C029F003C02AF0D2EC6EF0010AB6
:10C3900002E1090131872C6A2D6A800E2E6E3E0E55
:10C3A0002F6E7FC927F080C928F081C929F082C982
:10C3B0002AF0C9EC6EF0010A02E109013189050198
:10C3C0001E51080802E20901318B2C6A2D6A2E6A7F
:10C3D0002F6AA5C927F0A6C928F0A7C929F0A8C9BE
:10C3E0002AF0C2EC6EF0010A2FE063C92CF064C998
:10C3F0002DF065C92EF066C92FF05FC927F060C91E
:10C4000028F061C929F062C92AF0F8EC6CF027C065
:10C4100000F028C001F029C002F02AC003F0330E5A
:10C420002C6E2D6E730E2E6E3F0E2F6E00C027F0F9
:10C4300001C028F002C029F003C02AF0C9EC6EF058
:10C44000010A02E10901318D2C6A2D6A2E6A2F6AD8
:10C45000A5C927F0A6C928F0A7C929F0A8C92AF0BC
:10C46000C2EC6EF0010A30E063C92CF064C92DF013
:10C4700065C92EF066C92FF05FC927F060C928F0A2
:10C4800061C929F062C92AF0F8EC6CF027C000F00D
:10C4900028C001F029C002F02AC003F0CD0E2C6E96
:10C4A000CC0E2D6E4C0E2E6E3D0E2F6E00C027F062
:10C4B00001C028F002C029F003C02AF0D2EC6EF0CF
:10C4C000010A02E10901318F2C6A2D6A400E2E6E9D
:10C4D0002F6E0AC427F00BC428F00CC429F00DC439
:10C4E0002AF0C9EC6EF0010A02E1090132810AC4A6
:10C4F0002CF00BC42DF00CC42EF00DC42FF00EC484
:10C5000027F00FC428F010C429F011C42AF0F7EC6A
:10C510006CF027C000F028C001F029C002F02AC04A
:10C5200003F0CD0E2C6ECC0E2D6E4C0E2E6E3E0EEC
:10C530002F6E00C027F001C028F002C029F003C010
:10C540002AF0C9EC6EF0010A02E1090132832C6A7B
:10C550002D6A400E2E6E3F0E2F6E0EC427F00FC4B4
:10C5600028F010C429F011C42AF0D2EC6EF0010AB0
:10C5700002E1090132857B0E2C6E140E2D6E8E0E9B
:10C580002E6E3F0E2F6E0EC427F00FC428F010C47D
:10C5900029F011C42AF0C9EC6EF0010A02E1090188
:10C5A0003287330E2C6E2D6E2E6E3F0E2F6E7BC992
:10C5B00027F07CC928F07DC929F07EC92AF0D2EC89
:10C5C0006EF0010A02E109013289AE0E2C6E470EAF
:10C5D0002D6E810E2E6E3F0E2F6E7BC927F07CC90B
:10C5E00028F07DC929F07EC92AF0C9EC6EF0010A55
:10C5F00002E10901328B9BC22CF09CC22DF09DC23E
:10C600002EF09EC22FF097C227F098C228F099C250
:10C6100029F09AC22AF0C9EC6EF0010A02E1090180
:10C62000328D12000901349536951200FF0E090172
:10C63000385D20E10501B80ED88000550B0E01557C
:10C6400019E222C538F938C900F0016A00BE016854
:10C65000FF0E001801E101500DE138C900F0016A38
:10C6600000BE0168FE0E001801E1015002E0000E5C
:10C6700001D0010E1200D9CFE6FFE1CFD9FF0901A9
:10C68000C06BC16B36C42CF037C42DF038C42EF00B
:10C6900039C42FF0B5C927F0B6C928F0B7C929F0B9
:10C6A000B8C92AF0C2EC6EF0010A14E13AC42CF0C9
:10C6B0003BC42DF03CC42EF03DC42FF0B9C927F087
:10C6C000BAC928F0BBC929F0BCC92AF0C2EC6EF087
:10C6D000010A02E00901C081F3C52CF0F4C52DF078
:10C6E000F5C52EF0F6C52FF091C927F092C928F0B4
:10C6F00093C929F094C92AF0C2EC6EF0010A02E055
:10C700000901C08377C92CF078C92DF079C92EF0C2
:10C710007AC92FF0A9C927F0AAC928F0ABC929F016
:10C72000ACC92AF0C2EC6EF0010A14E17BC92CF00E
:10C730007CC92DF07DC92EF07EC92FF0ADC927F040
:10C74000AEC928F0AFC929F0B0C92AF0C2EC6EF02A
:10C75000010A02E00901C08905011F510901835D39
:10C7600001E0C08B0EC42CF00FC42DF010C42EF0CD
:10C7700011C42FF085C927F086C928F087C929F090
:10C7800088C92AF0C2EC6EF0010A02E00901C08DEE
:10C790003AD0100E0901BE6FBF6B200EBFAF02D0A2
:10C7A000D89003D0BE5D000EBF592DE2BEC9E9FF8F
:10C7B000BFC9EAFFD890E936EA36D890E936EA36BA
:10C7C000800EE926040EEA22EECF00F0EECF01F053
:10C7D000EECF02F0EFCF03F02C6A2D6A2E6A2F6A9B
:10C7E00000C027F001C028F002C029F003C02AF0E1
:10C7F000C2EC6EF0010A02E00901C08F0901BE2BF4
:10C80000000EBF23CAD7FBC52CF0FCC52DF0FDC51B
:10C810002EF0FEC52FF099C927F09AC928F09BC9C0
:10C8200029F09CC92AF0C2EC6EF0010A02E009016D
:10C83000C1816FC92CF070C92DF071C92EF072C979
:10C840002FF0A5C927F0A6C928F0A7C929F0A8C9C3
:10C850002AF0C2EC6EF0010A28E15FC92CF060C931
:10C860002DF061C92EF062C92FF09DC927F09EC935
:10C8700028F09FC929F0A0C92AF0C2EC6EF0010A85
:10C8800014E163C92CF064C92DF065C92EF066C9A6
:10C890002FF0A1C927F0A2C928F0A3C929F0A4C983
:10C8A0002AF0C2EC6EF0010A02E00901C1837FC9DF
:10C8B0002CF080C92DF081C92EF082C92FF0B1C9AA
:10C8C00027F0B2C928F0B3C929F0B4C92AF0C2ECE4
:10C8D0006EF0010A02E00901C18505011E5109013E
:10C8E000845D01E0C18797C22CF098C22DF099C2F7
:10C8F0002EF09AC22FF089C927F08AC928F08BC977
:10C9000029F08CC92AF0C2EC6EF0010A14E19BC236
:10C910002CF09CC22DF09DC22EF09EC22FF08DC92E
:10C9200027F08EC928F08FC929F090C92AF0C2ECEF
:10C930006EF0010A02E00901C1892C6A2D6A500ECD
:10C940002E6E410E2F6E0AC427F00BC428F00CC4C3
:10C9500029F00DC42AF0C9EC6EF0010A02E10901C8
:10C96000C18D0AC42CF00BC42DF00CC42EF00DC4E4
:10C970002FF00EC427F00FC428F010C429F011C402
:10C980002AF0F7EC6CF027C000F028C001F029C0B5
:10C9900002F02AC003F0CD0E2C6ECC0E2D6E4C0E84
:10C9A0002E6E3E0E2F6E00C027F001C028F002C090
:10C9B00029F003C02AF0C9EC6EF0010A02E1090176
:10C9C000C18FFE0EDB5006E00901C0513613C15184
:10C9D000371305D00901C0513413C1513513E55245
:10C9E000E7CFD9FF1200E66A46DEE5521200010EDB
:10C9F000E66E41DEE55212000201706B05011F0573
:10CA000001E0D7D30201925101E04CD1F00E2C6E1F
:10CA1000850E2D6E990E2E6E3E0E2F6EBBC227F028
:10CA2000BCC228F0BDC229F0BEC22AF08EEC6DF067
:10CA300027C016F428C017F429C018F42AC019F426
:10CA4000A40E2C6E700E2D6E7D0E2E6E3F0E2F6E70
:10CA500016C427F017C428F018C429F019C42AF006
:10CA6000F8EC6CF093EC6EF028C004F429C005F4E7
:10CA700004011F0ED8800455000E055503E21F0E59
:10CA8000046F056B000E045D000E055902E2046B95
:10CA9000056B04C4C6F2030E0201C603F3CFC5F250
:10CAA000C5C229F0D1EC6CF027C000F028C001F01D
:10CAB00029C002F02AC003F0960E2C6EB20E2D6E25
:10CAC000CC0E2E6E3D0E2F6E00C027F001C028F058
:10CAD00002C029F003C02AF0E1EC6DF027C016F483
:10CAE00028C017F429C018F42AC019F47FC92CF003
:10CAF00080C92DF081C92EF082C92FF016C427F00D
:10CB000017C428F018C429F019C42AF0F8EC6CF006
:10CB100027C000F028C001F029C002F02AC003F0AD
:10CB20000EC42CF00FC42DF010C42EF011C42FF041
:10CB300000C027F001C028F002C029F003C02AF08D
:10CB4000F8EC6CF027C0E8F228C0E9F229C0EAF25C
:10CB50002AC0EBF20201C65105E1A76BA86BA96BD5
:10CB6000AA6B26D0C6C229F0D1EC6CF027C000F029
:10CB700028C001F029C002F02AC003F000C02CF048
:10CB800001C02DF002C02EF003C02FF09FC227F08D
:10CB9000A0C228F0A1C229F0A2C22AF08EEC6DF04A
:10CBA00027C0A7F228C0A8F229C0A9F22AC0AAF279
:10CBB0002C6A2D6A2E6A2F6AA7C227F0A8C228F015
:10CBC000A9C229F0AAC22AF0D2EC6EF0010A05E14E
:10CBD0000201A76BA86BA96BAA6B9FC22CF0A0C225
:10CBE0002DF0A1C22EF0A2C22FF0A7C227F0A8C23A
:10CBF00028F0A9C229F0AAC22AF0C9EC6EF0010AF5
:10CC000008E19FC2A7F2A0C2A8F2A1C2A9F2A2C2E3
:10CC1000AAF22C6A400E2D6E1C0E2E6E460E2F6E42
:10CC2000A7C227F0A8C228F0A9C229F0AAC22AF0F8
:10CC3000E1EC6DF093EC6EF028C042F229C043F2B3
:10CC40002C6A2D6A7A0E2E6E440E2F6EE8C227F0E3
:10CC5000E9C228F0EAC229F0EBC22AF0E1EC6DF05B
:10CC600093EC6EF028C048F229C049F22C6A2D6A74
:10CC70007A0E2E6E440E2F6EAFC227F0B0C228F08F
:10CC8000B1C229F0B2C22AF0E1EC6DF093EC6EF083
:10CC900028C04AF229C04BF2C6C24EF20201010E70
:10CCA000926FC76BC75153E1C6C2C7F2C7C229F022
:10CCB000D1EC6CF027C004F028C005F029C006F0C4
:10CCC0002AC007F0A7C22CF0A8C22DF0A9C22EF0EE
:10CCD000AAC22FF004C027F005C028F006C029F032
:10CCE00007C02AF0E1EC6DF027C000F028C001F089
:10CCF00029C002F02AC003F000C02CF001C02DF0C2
:10CD000002C02EF003C02FF09BC227F09CC228F077
:10CD10009DC229F09EC22AF0F7EC6CF027C0A3F266
:10CD200028C0A4F229C0A5F22AC0A6F20201C75168
:10CD3000EA6A700FE96E020EEA22EF500401046FF6
:10CD4000056B04C408F30301210E096F04D0010E22
:10CD50000401046F056B0401010E041901E1055182
:10CD600001E091D10201C7050401046F056B010EBA
:10CD7000041901E1055101E07FD0C3C228F0C4C20B
:10CD800029F004C42DF005C42EF04EEC6EF026C040
:10CD900004F027C005F004C028F005C029F0E2EC3B
:10CDA0006CF027C000F028C001F029C002F02AC0B2
:10CDB00003F0960E2C6EB20E2D6ECC0E2E6E3D0E26
:10CDC0002F6E00C027F001C028F002C029F003C078
:10CDD0002AF0E1EC6DF027C016F428C017F429C042
:10CDE00018F42AC019F42C6A2D6A400E2E6E2F6E8C
:10CDF000A7C227F0A8C228F0A9C229F0AAC22AF027
:10CE00008EEC6DF027C000F028C001F029C002F0C0
:10CE10002AC003F0C3C208F0C4C209F0060ED880CD
:10CE20000856000E095608C028F009C029F0E2ECA7
:10CE30006CF027C004F028C005F029C006F02AC015
:10CE400007F004C02CF005C02DF006C02EF007C07E
:10CE50002FF000C027F001C028F002C029F003C065
:10CE60002AF0E1EC6DF027C0ABF228C0ACF229C08B
:10CE7000ADF22AC0AEF25FD0045105111FE1166B6E
:10CE8000176B186B196BA3C22CF0A4C22DF0A5C2AE
:10CE90002EF0A6C22FF09BC227F09CC228F09DC2A4
:10CEA00029F09EC22AF0F7EC6CF027C0ABF228C044
:10CEB000ACF229C0ADF22AC0AEF23DD0030E286E0E
:10CEC000296A04C42DF005C42EF04EEC6EF026C085
:10CED00004F027C005F004C028F005C029F0E2ECFA
:10CEE0006CF027C000F028C001F029C002F02AC071
:10CEF00003F0960E2C6EB20E2D6ECC0E2E6E3D0EE5
:10CF00002F6E00C027F001C028F002C029F003C036
:10CF10002AF0E1EC6DF027C016F428C017F429C000
:10CF200018F42AC019F4A7C2ABF2A8C2ACF2A9C285
:10CF3000ADF2AAC2AEF20EC42CF00FC42DF010C494
:10CF40002EF011C42FF016C427F017C428F018C40F
:10CF500029F019C42AF0F8EC6CF027C016F428C0A8
:10CF600017F429C018F42AC019F4ABC22CF0ACC2D3
:10CF70002DF0ADC22EF0AEC22FF0A3C227F0A4C296
:10CF800028F0A5C229F0A6C22AF0F8EC6CF027C060
:10CF900004F028C005F029C006F02AC007F0B3C28B
:10CFA0002CF0B4C22DF0B5C22EF0B6C22FF004C0E2
:10CFB00027F005C028F006C029F007C02AF0E1ECF0
:10CFC0006DF027C000F028C001F029C002F02AC08F
:10CFD00003F0AFC22CF0B0C22DF0B1C22EF0B2C23D
:10CFE0002FF000C027F001C028F002C029F003C0D4
:10CFF0002AF0F8EC6CF027C012F428C013F429C012
:10D0000014F42AC015F416C42CF017C42DF018C45B
:10D010002EF019C42FF012C427F013C428F014C442
:10D0200029F015C42AF0C9EC6EF0010A04E10401EC
:10D03000046B056B27D004C4C7F2ABC22CF0ACC2A2
:10D040002DF0ADC22EF0AEC22FF0A3C227F0A4C2C5
:10D0500028F0A5C229F0A6C22AF0F8EC6CF027C08F
:10D06000A3F228C0A4F229C0A5F22AC0A6F20201A8
:10D07000C751EA6A700FE96E020EEA22EF5004010E
:10D08000046F056B68D60201C751000801E386D022
:10D09000F00E006E850E016E990E026E3E0E036E4E
:10D0A000C7C229F0D1EC6CF027C004F028C005F00D
:10D0B00029C006F02AC007F004C02CF005C02DF0EE
:10D0C00006C02EF007C02FF000C027F001C028F0E6
:10D0D00002C029F003C02AF0E1EC6DF027C016F47D
:10D0E00028C017F429C018F42AC019F47FC92CF0FD
:10D0F00080C92DF081C92EF082C92FF016C427F007
:10D1000017C428F018C429F019C42AF0F8EC6CF000
:10D1100027C000F028C001F029C002F02AC003F0A7
:10D120000EC42CF00FC42DF010C42EF011C42FF03B
:10D1300000C027F001C028F002C029F003C02AF087
:10D14000F8EC6CF027C022F428C023F429C024F4A2
:10D150002AC025F40201C70505E1C3C2BFF2C4C25B
:10D16000C0F205D0030EC703F350BF6FC06B210E92
:10D170000301095D12E1C7C209F30201C751EA6A5E
:10D18000700FE96E020EEA22EFCF0AF303010C29B9
:10D190000C6F640E0C5D01E10C6B0AD00EC422F41E
:10D1A0000FC423F410C424F411C425F4BF6BC06B66
:10D1B000E8D00EC42CF00FC42DF010C42EF011C412
:10D1C0002FF076C427F077C428F078C429F079C40A
:10D1D0002AF0F7EC6CF027C012F428C013F429C031
:10D1E00014F42AC015F42C6A2D6A2E6A2F6A12C410
:10D1F00027F013C428F014C429F015C42AF0D2EC87
:10D200006EF0010A01E1B2D0F00E2C6E850E2D6E8B
:10D21000990E2E6E3E0E2F6E12C427F013C428F006
:10D2200014C429F015C42AF08EEC6DF027C012F456
:10D2300028C013F429C014F42AC015F4A40E2C6ECF
:10D24000700E2D6E7D0E2E6E3F0E2F6E12C427F0C7
:10D2500013C428F014C429F015C42AF0F8EC6CF0BB
:10D2600093EC6EF028C0BFF229C0C0F2030E286E06
:10D27000296ABFC22DF0C0C22EF04EEC6EF026C05F
:10D28000BFF227C0C0F20201BF51C01109E10EC4B4
:10D2900022F40FC423F410C424F411C425F465D07F
:10D2A000C351BF5DC451C05904E2C3C2BFF2C4C27E
:10D2B000C0F2BFC228F0C0C229F0E2EC6CF027C077
:10D2C00000F028C001F029C002F02AC003F0960E39
:10D2D0002C6EB20E2D6ECC0E2E6E3D0E2F6E00C03B
:10D2E00027F001C028F002C029F003C02AF0E1ECC9
:10D2F0006DF027C012F428C013F429C014F42AC01A
:10D3000015F47FC92CF080C92DF081C92EF082C997
:10D310002FF012C427F013C428F014C429F015C448
:10D320002AF0F8EC6CF027C000F028C001F029C00A
:10D3300002F02AC003F00EC42CF00FC42DF010C46C
:10D340002EF011C42FF000C027F001C028F002C059
:10D3500029F003C02AF0F8EC6CF027C022F428C0B2
:10D3600023F429C024F42AC025F40BD00EC422F4DF
:10D370000FC423F410C424F411C425F40201BF6BBC
:10D38000C06B120005011F051DE1200E0401046F92
:10D39000056B006B0451005D000E055513E2005152
:10D3A000EA6AC80FE96E020EEA22EF50E66E0051FB
:10D3B000EA6A500FE96E020EEA22E552E750EF6E7C
:10D3C000002BE8D7120005011F050EE10401006BD8
:10D3D000200E005D09E20051EA6AC80FE96E020EF4
:10D3E000EA22EF6A002BF4D7120005011F0523E1A2
:10D3F0000201C751EA6AC80FE96E020EEA22EF5035
:10D40000006E016AD890015004E6FF0E005C000E29
:10D41000015811E2C751EA6AC80FE96E020EEA220A
:10D42000EF28E66EC751EA6AC80FE96E020EEA22DB
:10D43000E552E750EF6E120005011F0501E145D0EE
:10D440002C6A2D6A2E6A2F6A2EC427F02FC428F06A
:10D4500030C429F031C42AF0D2EC6EF0010A1BE18D
:10D460007BC92CF07CC92DF07DC92EF07EC92FF030
:10D470002EC427F02FC428F030C429F031C42AF07C
:10D48000E1EC6DF027C02EF428C02FF429C030F451
:10D490002AC031F41AD077C92CF078C92DF079C997
:10D4A0002EF07AC92FF02EC427F02FC428F030C4F4
:10D4B00029F031C42AF0E1EC6DF027C02EF428C029
:10D4C0002FF429C030F42AC031F412000001130EE9
:10D4D0008A6F1C0E8B6F976BF50E986F996B9A6B1A
:10D4E000300E9B6F390E9C6F86EF6AF000010C0EB8
:10D4F0008A6F100E8B6F976BE10E986F996B9A6B1A
:10D500002E0E9B6F3E0E9C6F86EF6AF00001906BB3
:10D5100090C0DEFF84820001706B0001875103E13F
:10D520000001010E876F0001865103E10001010E29
:10D53000866F00018B510001D880885502E28BC0B4
:10D5400088F00001875100018825410806E2410E5C
:10D550000001D88087550001886F86C092F00001D5
:10D56000916B00019151912BEA6A600FE96E000EF8
:10D57000EA22EFCF93F05BD80001906B0001010E1F
:10D58000946F0001935152E00001940501E1F1D83C
:10D59000FFD8010E000194190001946F0001940559
:10D5A00008E1CED8400E0001925D02E20001922B0C
:10D5B000A5D90001902B040E0001905D02E2000E3F
:10D5C00001D0010E036E3C0E0001935D02E0000EDF
:10D5D00001D0010E026E3A0E0001935D02E0000ED2
:10D5E00001D0010E016E2E0E0001935D02E0000ECF
:10D5F00001D0010E011002100314006E00018A51C7
:10D600000001905D02E2000E01D0010E00100DE05D
:10D6100000019151912BEA6A600FE96E000EEA2237
:10D62000EFCF93F004D80001906BABD7120000014C
:10D630009C51D880935502E3000E01D0010E006E7C
:10D640009B51935D02E3000E01D0010E001006E035
:10D650008C6B8D6B8E6B8F6B956B71D09B51935DCB
:10D660008C6F8D6B8E6B8F6B8B29FE0BE842006E7F
:10D67000016A026A036A8CC026F08DC027F08EC052
:10D6800028F08FC029F000C02BF001C02CF002C0A0
:10D690002DF003C02EF048EC70F022C08CF023C0B7
:10D6A0008DF024C08EF025C08FF08AC000F0016A92
:10D6B000026A036A8CC026F08DC027F08EC028F065
:10D6C0008FC029F000C02BF001C02CF002C02DF05B
:10D6D00003C02EF048EC70F022C08CF023C08DF017
:10D6E00024C08EF025C08FF0000197518C279851EF
:10D6F0008D2399518E239A518F233C0E935D02E026
:10D70000000E01D0010E016E3A0E935D02E0000E94
:10D7100001D0010E006E2E0E935D02E0000E01D0CE
:10D72000010E001001100BE08B51E824006E000187
:10D73000005000018C27000E8D238E238F231200B2
:10D740000001750E966FF0D800018705966FECD832
:10D7500000013F0E966FE8D80001150E966FE4D8D1
:10D7600000019205966FE0D800019205966F94EF44
:10D770006CF00001956B8851955D09E29551EA6A5C
:10D78000000FE96E080EEA22EF6A952BF4D712001B
:10D7900000018C518D118E118F1101E1AED000016D
:10D7A0008C510001956F95C0F6FF8DC000F08EC0C2
:10D7B00001F08FC002F00001036A00500001956F74
:10D7C00095C0F7FF8EC000F08FC001F00001026A23
:10D7D000036A00500001956F95C0F8FF0001956B3A
:10D7E000000188510001955D01E37AD00900F5CF71
:10D7F00096F0000189511CE000018939F00B006EA0
:10D80000F00E00019615005C07E200018939F00B6B
:10D810000001965D0001966F0F0E00019615000144
:10D82000895D06E2000189510001965D0001966F55
:10D83000000194051EE1F00E00019615E66E000150
:10D840009551EA6A000FE96E080EEA22E552E750A8
:10D85000EF6E00019639F00BF00BE66E0001952992
:10D86000EA6A000FE96E080EEA22E552E750EF6E11
:10D8700033D0000196390F0B0F0B006E000195514C
:10D88000EA6A000FE96E080EEA22EF50F00B001072
:10D89000E66E00019551EA6A000FE96E080EEA2271
:10D8A000E552E750EF6E0F0E00019615006E000175
:10D8B0009529EA6A000FE96E080EEA22EF50F00B94
:10D8C0000010E66E00019529EA6A000FE96E080E65
:10D8D000EA22E552E750EF6E020E0001952780D74D
:10D8E00000018B29FE0BE842006E00010050000190
:10D8F0008C27000E8D238E238F231200848200013B
:10D90000956B000188510001955D0DE20001955174
:10D91000EA6A000FE96E080EEA22EFCF96F007D808
:10D920000001952BEED71200849201D8120001015C
:10D9300084900001839096BF8382839096AF8392F8
:10D94000838096BD8382839096AD8392838096BBBD
:10D950008382839096AB8392838096B983828390EF
:10D9600096A98392838096B78382839096A78392A9
:10D97000838096B58382839096A58392838096B3A5
:10D980008382839096A38392838096B183828390CF
:10D9900096A1839283808480010100010001966B2F
:10D9A0001200219E05D0219E29AE02D0296C218E25
:10D9B00029C023F0226A336A326A860E246E256AF1
:10D9C0004CEF6FF0219E08D0219E29AE05D0286C27
:10D9D000291EE86A2922218E29C023F028C022F0BE
:10D9E000336A326A8E0E246E256A4CEF6FF02F7EFA
:10D9F000216A88EC6FF0A0EC6FF021B630EF6FF089
:10DA000021A20AD021AA03D021BE30EF6FF021A4B9
:10DA10003CEF6FF039EF6FF021AA05D021AC3CEF5D
:10DA20006FF039EF6FF021A00AD021A808D021BEF5
:10DA300004D021A402D045EF6FF049EF6FF0326AB5
:10DA4000256A2F502A5C316E10E327C033F028C0BE
:10DA500022F029C023F02AC030F02CC027F02DC0BE
:10DA600028F02EC029F0213A09D02CC033F02DC067
:10DA700022F02EC023F02FC030F0316C219E21BC4B
:10DA8000218E30C024F021B078EF6FF01A0E316093
:10DA900078EF6FF0246A2A6A21A408D0276C281E28
:10DAA000291E2A1EE86A282229222A2221AC08D00F
:10DAB000336C221E231E241EE86A222223222422E3
:10DAC000266A315207E02A34293228322732263298
:10DAD000312EF9D7275033262850222229502322CD
:10DAE0002A50242226C032F0219E24AE0BD0326C64
:10DAF000331E221E231E241EE86A332222222322E2
:10DB00002422218E24A006D0D88023322232333220
:10DB10003232302A30C024F04CEF6FF0216A88ECAA
:10DB20006FF0A0EC6FF021B630EF6FF021A205D0BE
:10DB300021BA30EF6FF037EF6FF021BA43EF6FF09B
:10DB400021A005D021B830EF6FF043EF6FF021B87E
:10DB500037EF6FF0256A7F0E2A24246EE86A2522AB
:10DB60002F50245EE86A255A1A0E306E2A6A326AED
:10DB7000336A226A236A2C50275E2D50285A2E5071
:10DB8000295A000E2A5A09E72C5027262D50282200
:10DB90002E502922000E2A2201D0328AD890273610
:10DBA000283629362A36D89032363336223623366E
:10DBB000302EE1D7295028102710D8A4328A4CEFF4
:10DBC0006FF0216A88EC6FF0A0EC6FF021B630EFB7
:10DBD0006FF021A205D021B830EF6FF037EF6FF072
:10DBE00021AA05D021B030EF6FF037EF6FF021B0F0
:10DBF00002D021A802D043EF6FF0256A2F502A24CB
:10DC0000246EE86A25227E0E245EE86A255A326A6E
:10DC1000336A226A236A2E502902F4CF23F0F3CF0D
:10DC200022F02D502902F3503326F4502222000E08
:10DC300023222E502802F3503326F4502222000EC5
:10DC400023222C502902F3503226F4503322000EA6
:10DC5000222223222D502802F3503226F450332260
:10DC6000000E222223222E502702F3503226F45097
:10DC70003322000E222223222C502802F450322676
:10DC8000000E3322222223222D502702F450322666
:10DC9000000E3322222223224CEF6FF028C032F0F4
:10DCA00028502D02F4CF27F0F3CF26F029502E0272
:10DCB000F4CF29F0F3CF28F02D02F3502726F450AB
:10DCC0002822E86A292232502E02F3502726F450E7
:10DCD0002822E86A2922000C216A88EC6FF021B61C
:10DCE00076EF6EF021A20AD021B403D07F0E296E08
:10DCF00019D0800E296E16D0296A14D021B0FCD715
:10DD0000870E2A60F1D77E0E2A64F6D7860E2A5C2B
:10DD100004E0D89029322A2AF9D721A403D0296C0B
:10DD200029AEEAD71200216A88EC6FF021B69DEF88
:10DD30006EF021A20ED021B405D07F0E296EFF0E09
:10DD4000286E1FD0800E296E286A1BD0296A286A87
:10DD500018D021B0FBD78F0E2A60EDD77E0E2A6433
:10DD6000F5D78E0E2A5C05E0D890293228322A2A6F
:10DD7000F8D721A406D0286C291EE86A292229AEEA
:10DD8000E5D71200DBEC6EF021B6000C21B0010CDF
:10DD9000000CDBEC6EF021B6000C21B0000C21B4BD
:10DDA000000C010CDBEC6EF021B6000C21B0000C75
:10DDB00021A4000C010C216A88EC6FF0A0EC6FF03C
:10DDC00021B6120021AE08D021A004D021A802D093
:10DDD00021801200219012002F502A5C0BE12E505E
:10DDE000295C08E12D50285C05E12C50275C02E1FC
:10DDF00021801200D8A002D0218E10D02A502FC02E
:10DE00002AF02F6E29502EC029F02E6E28502DC0DA
:10DE100028F02D6E27502CC027F02C6E2F502A5C36
:10DE200010E0FF0F09E0219021B403D021AE21843E
:10DE3000120021AE219412002F2AD8902E322D32BA
:10DE40002C322C50275E2D50285A2E50295A29BE8C
:10DE5000EAD7D8902736283629362A2EF8D7C8D7B9
:10DE60007F0E2A6EFF0E296E286E276E12007F0E1F
:10DE700021BEFF0E2A6E02D07F0E2A6E800E296E02
:10DE8000286A276AF3D721AE04D0800E2A6E296A49
:10DE9000F7D72A6A296AF4D7235022103310321098
:10DEA000F8E025BEF0D723BE0CD024502510EBE0BF
:10DEB000D89032363336223623362406D8A02506AB
:10DEC000F2D72550D4E12428D2E032AE11D07F0E13
:10DED000321402E133A00CD0332AE86A2222232232
:10DEE00007E3D880233222323332242A2428BFE0A9
:10DEF0002450C9E033C027F022C028F02334296E13
:10DF000024302A6E29322A9E21BE2A8E36EF6FF0E7
:10DF100029362A3602E32184217E06E121802A6AFD
:10DF2000296A286A276A12002A2803E0D880293241
:10DF30001200D890293202E12182120021861200BB
:10DF40002E362F3602E3218C217E06E121882F6AAE
:10DF50002E6A2D6A2C6A12002F2803E0D8802E32F8
:10DF60001200D8902E32EAE1218A1200D9CFE6FFC2
:10DF7000DACFE6FFE1CFD9FFE2CFDAFF0C0EE124E2
:10DF800002E3E168E652E16ED950FA0FE96EFF0E46
:10DF9000DA20EA6E010EEECFDBFF020EEECFDBFFE2
:10DFA000030EEECFDBFF040EEECFDBFF63D8D950BC
:10DFB000010FE96E000EDA20EA6EEECFE6FFEECF3B
:10DFC000E6FFEECFE6FFEFCFE6FF72EC80F0006EEB
:10DFD000060EE15C02E2E16AE552E16E0050DF6E9E
:10DFE000850EDF1404E04DD8EE6AED6A23D0090EE9
:10DFF000DBCF00F00A0EDBCF01F0820E0026FF0E11
:10E0000001223FD800C0EEFF01C0EDFF7E0EF36E8F
:10E01000090EF3CFDBFF0A0EDB6AD950010FE66E63
:10E02000000EDA20E66E26D834ECBDF0E552E5525B
:10E03000E552E552010EDBCF00F0020EDBCF01F01E
:10E04000030EDBCF02F0040EDBCF03F000C026F09E
:10E0500001C027F002C028F003C029F00C0EE15CDB
:10E0600002E2E16AE552E16EE552E5CFDAFFE7CF81
:10E07000D9FF1200D950050FE66E000EDA20E66EC9
:10E080001200F80EDBCFE9FFF90EDBCFEAFF12003A
:10E0900026502B02F3CF22F0F4CF23F02C02F350C2
:10E0A0002326000EF420246E26502D02F350242641
:10E0B000000EF420256E26502E02F3502526275000
:10E0C0002B02F3502326F4502422000E2522275041
:10E0D0002C02F3502426F450252227502D02F35011
:10E0E000252628502B02F3502426F45025222850B0
:10E0F0002C02F350252629502B02F350252612001E
:10E10000000000000000000000000000000000000F
:10E1100000000000000000000000000000000000FF
:10E1200000000000000009800000000000006FF007
:10E130000000000000003FE00000000000000000C0
:10E1400000000000000000000000000000000000CF
:10E1500000000000000000000000000000000000BF
:10E16000000000000000000000000000000000208F
:10E170000000000000003AF000000000004BFFA08B
:10E18000000000005CFF91000000006DFE710000C7
:10E1900000017EFD60000000018FFD5000000000C6
:10E1A0009FFB400000000000FA300000000000006B
:10E1B000200000000000000000000000000000003F
:10E1C0000000000000000000000169BCCA720000ED
:10E1D000009FFEDCDFFFB2001DF8200005FDFF30D0
:10E1E000AF3000009F902ED0F800002CF50006F014
:10E1F000F80004ED300005F0AF308FB100000CE006
:10E200001DFDF8000016DF40009FFFDCDEFFC300AD
:10E21000000169BCCA73000000000000000000009B
:10E2200000000000000000000000000000000000EE
:10E2300002900000000001300AB00000000004F06D
:10E240002F600000000004F0AF977777777779F0C0
:10E25000FFFFFFFFFFFFFFF012222222222226F003
:10E2600000000000000004F000000000000003D0E7
:10E27000000000000000000000000000000000009E
:10E28000000000000000000000000000000001404D
:10E2900007D0000000007FF04F800000001CFEF05F
:10E2A000CC00000002EF57F0F70000002EE207F06C
:10E2B000F8000001DE2007F0CE10002DE20007F08C
:10E2C0004FD658FE300007F006FFFFB1000007F000
:10E2D0000014520000000580000000000000000053
:10E2E000000000000000000000000000000002002C
:10E2F0000920000000007F506F40000000002ED079
:10E30000DB000059000007F0F800008E000004F068
:10E31000EA0000CF100006F09F3007FF90001EE0DB
:10E320001EFCDF87FB79EF50019DC6007EFFD50004
:10E3300000000000002100000000000000000000BC
:10E340000000000000000000000000002BB00000F2
:10E3500000000006FFE00000000002CF69E00000BE
:10E3600000007FB109E00000002CE60009E0000099
:10E3700007FB100009E00000CFFCCCCCCEFDDDD0C7
:10E38000DEEEEEEEEFFEEEE00000000009E0000041
:10E390000000000008C000000000000000000000B5
:10E3A000000000000000000000000000000012005B
:10E3B00078ABCDED0000CE20FFEDCCFA00005FB0D1
:10E3C000F90006F0000008F0F9000AB0000004F0BF
:10E3D000F9000AC0000004F0F90008F300000BF097
:10E3E000F90001FE6213BF90F900004EFFFFFB0031
:10E3F000110000016AA940000000000000000000B8
:10E40000000000000000000000000356653000001E
:10E41000004BFFFFFFFFA20008FE968F956AFF30BA
:10E420006F9001F800003ED0EC0008F0000006F00C
:10E43000F6000AE0000004F0F70007F3000009F01E
:10E44000CD1001EF7213AF904D20002DFFFFF900AA
:10E4500000000000478610000000000000000000DF
:10E46000000000000000000011000000000000009B
:10E47000FA00000000000000FA0000000000049014
:10E48000FA0000000039EFF0FA0000017DFFE940DA
:10E49000FA0005BFFF940000FA18EFFB50000000DF
:10E4A000FEFFD71000000000FFB4000000000000D5
:10E4B000520000000000000000000000000000000A
:10E4C0000000000000000000000000000278500082
:10E4D00003ADB4007FFFFC003FFCFF66FA43AFA032
:10E4E000CD101CFE70000BF0F50001FE000005F0E1
:10E4F000F50000BF100004F0EC0007FFB0000AF0C8
:10E500006FD9CF78FB329F9007EFE6009FFFFB00AB
:10E51000000100000388500000000000000000001F
:10E520000000000000000000000355200000000073
:10E5300004DFFFFB10000B604FD7459FD0001CE0AD
:10E54000DD000005F50005F0F7000000F80004F01C
:10E55000F8000000F70008F0BE200006F2005FA0FF
:10E560002EF9547F947CFC0002AFFFFFFFFE700089
:10E570000001467775300000000000000000000038
:10E58000000000000000000000000000000000008B
:10E59000000000000000000000000000000000007B
:10E5A000000006A10000098000001FF900006FF0C4
:10E5B00000000DF500003FE000000010000000002A
:10E5C000000000000000000000000000000000004B
:10E5D000000000000000000000000000000000003B
:10E5E000000000000000000000000000000000002B
:10E5F0000000300000000000BAAEF0000000000093
:10E60000FFE930000000000053000000000000009F
:10E610000000100000000000978CF00000000000D7
:10E62000FFFB50000000000075100000000000001B
:10E6300000000000000000000000000000000000DA
:10E6400000000000000000000000000000000000CA
:10E6500000000000000000000000000000000000BA
:10E660000000000000000000756AE00000000000EB
:10E67000FFFD700000000000A83000000000000056
:10E68000000000000000000000000000000000008A
:10E69000000000000000000000000000000000007A
:10E6A000000000000000000000000000000000006A
:10E6B00000100000000000002CFFA000000000007F
:10E6C000DD78FA0000000000F2005F0000000000AA
:10E6D000F0004F1000000000EA23DC000000000002
:10E6E0004FFFE200000000000154000000000000A5
:10E6F000000000000000000000000000000000001A
:10E7000000001111111111100000FFFFFFFFFFF0B9
:10E7100000009FA7777777700000D6000000000008
:10E720000002F300000000000001FFCBBBBBBBB048
:10E7300000004FFEEEEEEEE00000AB200000000017
:10E740000001F100000000000002FA555555555037
:10E750000000AFFFFFFFFFF00000024444444440CC
:10E76000FFFFFFFFFFFFFFFFFFFFFFFFFFFFFFFFB9
:10E77000FFFFFFFFFFFFFFFFFFFFFFFFFFFFFFFFA9
:10E78000FFFFFFFFFFFFFFFFFFFFFFFFFFFFFFFF99
:10E79000FFFFFFFFFFFFFFFFFFFFFFFFFFFFFFFF89
:10F5100000037ACDEEDCA84000000000000018DFF8
:10F52000FFFFFFFFFFFE920000000007EFFFFFDC80
:10F53000BBCEFFFFFF91000000BFFFC76543223332
:10F5400057BFFFFD20000BFFC40000000000002497
:10F550006EFFD1007FFA000000000000000001BF34
:10F56000FA00EFC00000000000000000000DFF20C6
:10F57000FF6000000000000000000005FF60FF4089
:10F5800000000000000000000003FF70FF8000008A
:10F590000000000000000006FF50CFF30000000054
:10F5A00000000000001DFF104FFE300000000000B2
:10F5B000000001CFF80007FFD71000000000000195
:10F5C0007EFFB000005EFFFB9854333458BFFFFA53
:10F5D000000000019FFFFFFFFFFFFFFFFD50000045
:10F5E0000000017BFFFFFFFFFFE94000000000007B
:10F5F00000000246776541000000000000000000A6
:10F6000000000000000000000000000000000000FA
:10F6100000000000000000000000000000000000EA
:10F6200000000000000000010000000000000000D9
:10F6300000000000001FA00000000000000000010A
:10F640004400009F90000000000000000004FF0044
:10F6500002FF50000000000000000004FF000AFF4D
:10F6600010000000000000000004FF003FFC00004C
:10F670000000000000000004FF00BFFC77777777F0
:10F68000777777777779FF00FFFFFFFFFFFFFFFFB7
:10F69000FFFFFFFFFF00FFFFFFFFFFFFFFFFFFFF79
:10F6A000FFFFFF00333333333333333333333336F6
:10F6B000FF00000000000000000000000004FF0048
:10F6C000000000000000000000000004FF00000037
:10F6D00000000000000000000004FF000000000027
:10F6E0000000000000000003CC000000000000004B
:10F6F000000000000000000000000000000000000A
:10F7000000000000000000000000000000000000F9
:10F7100000000000000000000000000000000000E9
:10F7200000000000000000000000000000000000D9
:10F7300000083000000000000000002AFF0000BFA9
:10F74000D10000000000000008FFFF000AFFB30026
:10F75000000000000003DFFFFF004FFA0000000080
:10F760000000006FFFDBFF00CFE0000000000000A2
:10F7700008FFF808FF00FF800000000000009FFE67
:10F780004008FF00FF40000000000009FFD2000811
:10F79000FF00FF4000000000009FFD100008FF0078
:10F7A000FF800000000008FFD1000008FF00FFE01C
:10F7B000000000008FFE20000008FF009FFA0000FC
:10F7C000001AFFE200000008FF002EFFD62138EFEC
:10F7D000FD2000000008FF0004FFFFFFFFFFC10045
:10F7E00000000008FF00003DFFFFFFE700000000F1
:10F7F0000008FF00000059BB950000000000000B4E
:10F80000FF000000000000000000000000000000F9
:10F8100000000000000000000000000000000000E8
:10F8200000000000000000000000000000000000D8
:10F8300000000000000000000000002000000000A8
:10F8400000000000005E300004F80000000000002E
:10F85000000008FFD0001EFE200000000000000095
:10F8600004DFF8007FF50000000000000000002F1A
:10F87000FE00DFC000000007950000000009FF3017
:10F88000FF700000000CF70000000004FF60FF5054
:10F890000000000EF80000000003FF70FF60000091
:10F8A000002FFA0000000004FF60FFB00000007F9E
:10F8B000FE0000000009FF30BFF4000002EFFF70FF
:10F8C0000000002FFE004FFE60005EFDBFF500004F
:10F8D00003EFF70009FFFFDFFFF32FFFB656BFFF6F
:10F8E000C000008FFFFFFE4004FFFFFFFFFC100081
:10F8F00000028CDB7100002BFFFFFE800000000087
:10F90000000000000000156630000000000000004C
:10F9100000000000000000000000000000000000E7
:10F9200000000000000000000000000000000000D7
:10F930000000000000000000000000000004EFC014
:10F940000000000000000000000001AFFFC0000048
:10F9500000000000000000005EFFFFC0000000008B
:10F9600000000000001BFFD4CFC00000000000001A
:10F97000000006EFF800CFC0000000000000000209
:10F98000BFFC3000CFC0000000000000007FFF700F
:10F990000000CFC00000000000002CFFB2000000FB
:10F9A000CFC0000000000007FFE600000000CFC04D
:10F9B0000000000003CFFA1000000000CFC00000DC
:10F9C00000008FFFEAAAAAAAAAAAEFEAAAAAAA0096
:10F9D000FFFFFFFFFFFFFFFFFFFFFFFFFF00FFFF36
:10F9E000FFFFFFFFFFFFFFFFFFFFFF004444444412
:10F9F00044444444DFD44444440000000000000078
:10FA00000000CFC000000000000000000000000067
:10FA1000CFC000000000000000000000000079706E
:10FA200000000000000000000000000000000000D6
:10FA300000000000000000000000000000000000C6
:10FA40000000000000000000000000200000000096
:10FA5000001234567200000003F80000ABCDEFFF37
:10FA6000FFFFF80000001EFF8000FFFFFFFFFFFF09
:10FA7000F900000028FFF300FFDAA98767FFB00054
:10FA80000000007FFB00FF70000006FF1000000078
:10FA9000000CFF10FF7000000BFA000000000005D2
:10FAA000FF50FF7000000DF7000000000002FF7023
:10FAB000FF7000000EF7000000000002FF70FF70F2
:10FAC00000000EFA000000000004FF60FF7000005C
:10FAD0000BFE10000000000AFF30FF70000006FF60
:10FAE000B0000000006FFD00FF70000000DFFD406F
:10FAF000000029FFF500FF700000003FFFFEBABDC7
:10FB0000FFFF9000FF7000000003DFFFFFFFFFF822
:10FB1000000055200000000007DFFFFFEA30000072
:10FB2000000000000000000134420000000000005E
:10FB300000000000000000000000000000000000C5
:10FB400000000000000000000000000000000012A3
:10FB5000333321000000000000000049CEFFFFFF0A
:10FB6000FFEB7100000000007EFFFFFFFFFFFFFFC3
:10FB7000FF900000003DFFFFFCBAFFFBABEFFFFD75
:10FB8000200004FFFE83001CFD2000028EFFD10038
:10FB90001EFF900000BFE100000001CFF900AFF7A9
:10FBA000000005FF50000000001DFF10FFB0000026
:10FBB0000AFE000000000006FF50FF5000000DFB91
:10FBC000000000000002FF70FF2000000DFC00009C
:10FBD00000000003FF60FF3000000AFF200000006B
:10FBE0000008FF30FF70000005FFC1000000004F5B
:10FBF000FD00EFE1000000CFFD50000028FFF40001
:10FC00007FFD0000002DFFFFDBCDFFFF70000CD259
:10FC100000000001BFFFFFFFFFE500000110000032
:10FC20000000039DFFFEB600000000000000000081
:10FC300000000000000000000000000000000000C4
:10FC400000000000000000000000000000000000B4
:10FC500000000000000000000000000000000000A4
:10FC60000000CC7000000000000000000000000058
:10FC7000FF90000000000000000000000000FF9066
:10FC8000000000000000000000000400FF900000E1
:10FC90000000000000000049EF00FF90000000009D
:10FCA000000000049EFFFF00FF9000000000000025
:10FCB00038DFFFFFFE00FF9000000000017DFFFF26
:10FCC000FFD94000FF9000000005BFFFFFFD83004B
:10FCD0000000FF90000039EFFFFFE8300000000057
:10FCE000FF90006CFFFFFE94000000000000FF92F8
:10FCF0008EFFFFFB5000000000000000FFEFFFFF41
:10FD0000D7100000000000000000FFFFFFA400006B
:10FD10000000000000000000FFFD71000000000076
:10FD2000000000000000BA400000000000000000D9
:10FD300000000000000000000000000000000000C3
:10FD400000000000000000000000000000000000B3
:10FD500000000000000000000000000000000000A3
:10FD60000000000000000367620000000000244261
:10FD700000000004DFFFFFB20000003CFFFFC400F2
:10FD8000008FFFFFFFFE300005FFFFFFFF7008FF41
:10FD9000FB77AFFFE1003FFFA78DFFF64FFC200090
:10FDA00002DFF900BFE300008FFEDFB00000002E8D
:10FDB000FF00FF60000008FFFE1000000008FF4089
:10FDC000FF10000000CFF70000000004FF60FF00FC
:10FDD0000000003FF90000000003FF60FF2000006A
:10FDE000005FFF1000000005FF50FF80000003EFE0
:10FDF000FFA00000000AFF20DFF600005EFCCFF845
:10FE00000000004FFD004FFFC89DFFF33FFFA20021
:10FE100006FFF50007FFFFFFFE4006FFFFDCEFFFD8
:10FE2000A000004CFFFF9100005EFFFFFFFA000002
:10FE300000002430000000018EFFFB4000000000A5
:10FE400000000000000000110000000000000000A1
:10FE500000000000000000000000000000000000A2
:10FE6000000000000000000000000002210000006F
:10FE700000000000000000017DFFFFEA30000000EC
:10FE800000044000006EFFFFFFFFFA000000006F5B
:10FE9000E20008FFFFB99BEFFFC0000000BFFA00BF
:10FEA0004FFF70000005EFF80000000CFF10DFF3BB
:10FEB000000000001EFF10000006FF50FF80000041
:10FEC000000006FF50000004FF60FF40000000003B
:10FED00001FF70000004FF60FF300000000001FF20
:10FEE00070000007FF40FF700000000004FF4000AA
:10FEF000000DFE00EFE2000000000BFD0000009F7F
:10FF0000F8007FFD300000007FF400001AFFD100F0
:10FF10000BFFFB520008FF60136AFFFE200000AFDA
:10FF2000FFFFFFFFFFEFFFFFFFC200000004BFFF66
:10FF3000FFFFFFFFFFFFC500000000000269CDEFDB
:10FF4000FFEDB962000000000000000000000000AA
:10FF500000000000000000000000000000000000A1
:10FF600000000000FFFFFFFFFFFFFFFFFFFFFFFF9D
:10FF7000FFFFFFFFFFFFFFFFFFFFFFFFFFFFFFFF91
:10FF8000FFFFFFFFFFFFFFFFFFFFFFFFFFFFFFFF81
:10FF9000FFFFFFFFFFFFFFFFFFFFFFFFFFFFFFFF71
:10FFA000FFFFFFFFFFFFFFFFFFFFFFFFFFFFFFFF61
:10FFB000FFFFFFFFFFFFFFFFFFFFFFFFFFFFFFFF51
:10FFC000FFFFFFFFFFFFFFFFFFFFFFFFFFFFFFFF41
:10FFD000FFFFFFFFFFFFFFFFFFFFFFFFFFFFFFFF31
:10FFE000FFFFFFFFFFFFFFFFFFFFFFFFFFFFFFFF21
:10FFF000FFFFFFFFFFFFFFFFFFFFFFFFFFFFFFFF11
:020000040001F9
:10000000D7EC85F00501206921691200FFFFFFFF91
:10001000FFFFFFFFFFFFFFFFFFFFFFFFFFFFFFFFF0
:10002000EAEC84F088EFA8F0FFFFFFFFFFFFFFFF7F
:10003000FBEFB3F0A3EFB9F0F4EFB9F00000FFFF6E
:1000400080EC83F005011E6B1200FFFFFFFFFFFF36
:1000500003EFB4F0FFFFFFFFFFFFFFFFFFFFFFFF16
:1000600088EFA8F0FFFFFFFFFFFFFFFFFFFFFFFF8D
:10007000FFFFFFFFFFFFFFFFFFFFFFFFFFFFFFFF90
:10008000F9ECACF00501030E236F88EFA8F0FFFF39
:10009000FFFFFFFFFFFFFFFFFFFFFFFFFFFFFFFF70
:1000A000120000EE00F00D0EEE6AEA62FDD71200BB
:1000B00066EF6AF076EF6AF0FFFFFFFFFFFFFFFFDA
:1000C00044EFA7F04FEFBAF083EFBAF0FFFFFFFF66
:1000D000FFFFFFFFFFFFFFFFFFFFFFFFFFFFFFFF30
:1000E00064EFB2F0D9CFE6FFDACFE6FFE1CFD9FF78
:1000F000E2CFDAFFE652006801687F0E026E036A03
:10010000D950FA0FE96EFF0EDA20EA6EEE500016B3
:10011000EE500116EE500216EE5003166AD800C0DB
:10012000EEFF01C0EEFF02C0EEFF03C0EEFFFD0ECA
:10013000DB50800B02E0010E01D0000EE66E59D8B4
:10014000060EE926000EEA22E552E750EF6EFC0E9D
:10015000DBCF00F0FD0EDBCF01F0D890003601368A
:10016000FC0E00C0DBFFFD0E01C0DBFFDB50E66EC6
:1001700040D8040EE926000EEA22E552E750EE6E62
:10018000ED6AFD0EDB50006E016AFF0E001818E1EB
:10019000015016E12ED8EECF00F0EECF01F0EECFF9
:1001A00002F0EFCF03F0005001100210031006E040
:1001B000210E04017E6F7F6B800E0BD0040E09D0E0
:1001C000FD0EDB5008E115D8EE6AEE6AEE6AEE6AC3
:1001D000010EDF6E06D0020EDF6E0BD8EE52EE522D
:1001E000EE8EDF50E552E552E5CFDAFFE7CFD9FFDB
:1001F0001200F80EDBCFE9FFF90EDBCFEAFF1200A9
:10020000BB073BBCFFD03B3C0CF83AF297493AA302
:100210003AE93A6018043A1E099039DF4C01399DD9
:100220003EE5395EED3A39258D333901BAC638CA13
:10023000DC82389E4D8438789D9F3842AC34381823
:10024000C9A33C78BD453BF902CC3BA0443E3B589A
:1002500023623B14FA313AD06DA43A93FBDD3A4F56
:10026000F8033A12718D39DB55AB39AB1277398609
:100270001EEA3952542C3924B2373900DBDA38C936
:1002800044673FA100003F809EED3F5C96533F4195
:10029000B8523F1E19CE3F01CAC13EE1CCCD3ECC83
:1002A00000003EC033333EB3B4393EA8ED913E9CCE
:1002B00026E93E91A1CB3E85F3B63E7D48E93E6EF0
:1002C00006F73FDF06253FB1902E3F98DCC73F85FC
:1002D00008313F6C0C4A3F52020C3F3B73823F2671
:1002E00051EC3F18F3B63F0D86593F08D6A13F04A5
:1002F000A2343F04816F3F0467383F040BE13F03A2
:1003000047AE3F01C2273F26E2193F3851EC3F4834
:10031000068E3F50E9103F578A723F5E18933F6444
:10032000C1553F68154D3F6C91003F6EB7803F70DF
:100330009C783F72538F3F74CFAB3F751DE73F777B
:1003400058103ED91F8A3F1317593F27E8A73F3857
:1003500019653F42B2FF3F4BF1413F53F4F13F5A21
:100360002DE03F60EAB33F6352BD3F6644D03F6833
:1003700085F03F69C7113F6AF4883F6B3C363F6D9B
:10038000AA3BC0B8AA3BC13844FEC19084D4C1D5B1
:10039000CFA2C21B0558C25DAD3BC29C2CCFC2DEB2
:1003A00040F6C31DA22BC352E459C38666EDC3AC0D
:1003B00002D0C3DCA9ABC40C9D93C4330720C46531
:1003C0006C0BC00B6C0BC08BE798C0D959DCC121FA
:1003D000ADBDC16B1F2EC1A7F2BFC1ECFCC7C227C8
:1003E000C193C26D3EA3C29FF7DEC2CB5544C30288
:1003F000540CC326AE9EC354C955C3872522C3AD32
:10040000EC0E3E22F9C93DA9F2A83D5CA08A3D163A
:10041000A1233CCFEC893C92D09A3C4FD3523C1262
:10042000B7263BCF333A3B9B787B3B72CAC03B3D00
:10043000C4D73B14BF583AE84EA53AB6FF0A3A8EE5
:1004400078BE3EBC01903E52DB713E0B57373DC13A
:100450006C183D8674223D3FFBBA3D07C21A3CC072
:10046000AB443C887C103C4CDE0E3C1F74913BFA44
:100470006ABB3BC4B56C3B99E0573B70FA8F3B3C81
:10048000000040800000410000004148000041940D
:10049000000041D833334219333342590000429AA5
:1004A000000042DA000043120000433B0000436FAB
:1004B00080004398000043C3000043F9C000441E7D
:1004C00047AE3FC147AE40410A3D4097AE1440DFC2
:1004D0005C294123AE1441673D7141A4E14841E8E4
:1004E000CCCD4224C28F425C6148428DAE1442B4EE
:1004F000947B42E66B8543133D71433C07AE4370EA
:10050000BEBE3F525D853F14EEEE3ED9FE4C3E9F8F
:10051000D9993E6785273E296EAD3DF54E043DB025
:100520005C8D3D7CEACD3D3D0BB03D152C233CEA76
:1005300012963CB84F6E3C9076823C62DE9F3C3116
:1005400066E03F7D35C63F660D7C3F4507EA3F21AB
:1005500053093EFCC4B53EC2B51C3E92F8A53E58B8
:1005600090BC3E1EB79E3DF148C33DBF42493D97FA
:1005700000D43D6F21693D3C14F53D142E983CE9B3
:10058000FFFFFFFFFFFFFFFFFFFFFFFFFFFFFFFF7B
:10059000FFFFFFFFFFFFFFFFFFFFFFFFFFFFFFFF6B
:1005A000FFFFFFFFFFFFFFFFFFFFFFFFFFFFFFFF5B
:1005B000FFFFFFFFFFFFFFFFFFFFFFFFFFFFFFFF4B
:1005C000FFFFFFFFFFFFFFFFFFFFFFFFFFFFFFFF3B
:1005D000FFFFFFFFFFFFFFFFFFFFFFFFFFFFFFFF2B
:1005E000FFFFFFFFFFFFFFFFFFFFFFFFFFFFFFFF1B
:1005F000FFFFFFFFFFFFFFFFFFFFFFFFFFFFFFFF0B
:100600002E29C943D8A2017C363DA154F0EC130633
:10061000A762F305C7C08C739398D92B4CBCCA82D0
:100620009B1E3C57D4FD16E04267186F178A12E5EF
:100630004EBED6C49EDA49DEFBA08EF52FBB7AEE05
:1006400068A99179B2153F07C2948910220B215FE6
:100650007F809A5D905A27323E35E7CCF7BF0397EB
:1006600019FFB330A548D1B55ED72A9256ACC6AAB9
:10067000B84FD238A496B67DFC76E26B749CF10438
:100680009D455970716420875B8665CF2DE602A871
:10069000601BAD25B0AEF6B9461C696140340F7ED3
:1006A000475523A351DD3AAF5CC3CEF9C5BA26EA5C
:1006B000532C6E0D28850984DFD3F4CD8141524D32
:1006C000DC6AC837C16CFAABE124087BBD0C4AB1C7
:1006D00088788B9563E36DE8CBE9FED5003B391D47
:1006E000EFF20EB75866E4D077A6F87275EB0A4BB6
:1006F0004431B450ED8F1A1F99DB338D119F148351
:100700000901BD6B0901306B316B0901326B336B31
:100710000901346B356B0901366B376B0901386998
:1007200013EE00F0010EF86E04018C0E366F4A0EC7
:10073000376F4A0E386F3F0E396F00C528F001C57C
:1007400029F0E2EC6CF027C000F028C001F029C0CD
:1007500002F02AC003F02C6A2D6A7A0E2E6E440E27
:100760002F6E00C027F001C028F002C029F003C09E
:100770002AF08EEC6DF027C00AF428C00BF429C0D3
:100780000CF42AC00DF40401006B100E0401005D8E
:1007900001E3FAD0DC0E2C6E680E2D6E800E2E6EEC
:1007A0003D0E2F6E0AC427F00BC428F00CC429F0AC
:1007B0000DC42AF0F7EC6CF027C004F028C005F057
:1007C00029C006F02AC007F004C02CF005C02DF0A7
:1007D00006C02EF007C02FF036C427F037C428F02B
:1007E00038C429F039C42AF0E1EC6DF027C000F0DC
:1007F00028C001F029C002F02AC003F00401005112
:10080000040DF3CFE9FFF4CFEAFF800EE926040ED2
:10081000EA2200C0EEFF01C0EEFF02C0EEFF03C0FF
:10082000EEFF020EF76E04010051002500250025A1
:10083000800FF66E0900F5CF43F40900F5CF42F4BE
:100840000900F5CF45F40800F5CF44F4800FF66EAB
:10085000F72A0900F5CF4BF40900F5CF4AF4090057
:10086000F5CF4DF40800F5CF4CF404010051040D10
:10087000F3CFE9FFF4CFEAFF800EE926040EEA2267
:10088000EECF08F0EECF09F0EECF0AF0EFCF0BF08D
:1008900042C42CF043C42DF044C42EF045C42FF0C4
:1008A00008C027F009C028F00AC029F00BC02AF0C0
:1008B000F7EC6CF027C004F028C005F029C006F062
:1008C0002AC007F04AC42CF04BC42DF04CC42EF0C3
:1008D0004DC42FF004C027F005C028F006C029F051
:1008E00007C02AF0E1EC6DF027C000F028C001F04D
:1008F00029C002F02AC003F004010051040DF3CF17
:10090000E9FFF4CFEAFF6B0EE926050EEA2200C0EC
:10091000EEFF01C0EEFF02C0EEFF03C0EEFF0401D8
:100920000051040DF3CFE9FFF4CFEAFF6B0EE92687
:10093000050EEA22EECF00F0EECF01F0EECF02F08E
:10094000EFCF03F02C6A2D6A2E6A2F6A00C027F0C1
:1009500001C028F002C029F003C02AF0D2EC6EF0EA
:10096000010A0FE104010051040DF3CFE9FFF4CFB8
:10097000EAFF6B0EE926050EEA22EE6AEE6AEE6ADF
:10098000EE6A0401002B01D70401100E006F200E47
:100990000401005D12E204010051040DF3CFE9FFF0
:1009A000F4CFEAFF800EE926040EEA22EE6AEE6A30
:1009B000EE6AEE6A0401002BEAD744ECA4F00501CC
:1009C000236B0501226B0501316B0501326B0501BB
:1009D000666B120013EE00F004018C0E366F4A0EA7
:1009E000376F4A0E386F3F0E396F00C528F001C5CA
:1009F00029F0E2EC6CF027C000F028C001F029C01B
:100A000002F02AC003F02C6A2D6A7A0E2E6E440E74
:100A10002F6E00C027F001C028F002C029F003C0EB
:100A20002AF08EEC6DF027C00AF428C00BF429C020
:100A30000CF42AC00DF402C528F003C529F0E2EC3D
:100A40006CF027C000F028C001F029C002F02AC0D5
:100A500003F02C6A2D6A7A0E2E6E440E2F6E00C0A3
:100A600027F001C028F002C029F003C02AF08EEC64
:100A70006DF027C00EF428C00FF429C010F42AC06E
:100A800011F4DC0E2C6E680E2D6E800E2E6E3D0E57
:100A90002F6E0AC427F00BC428F00CC429F00DC433
:100AA0002AF0F7EC6CF027C000F028C001F029C054
:100AB00002F02AC003F000C02CF001C02DF002C0EB
:100AC0002EF003C02FF036C427F037C428F038C406
:100AD00029F039C42AF0E1EC6DF027C026F428C0D3
:100AE00027F429C028F42AC029F404012A6B2B6BAF
:100AF0002C6B2D6B0EC432F40FC433F410C434F4D9
:100B000011C435F413C529F0D1EC6CF027C000F006
:100B100028C001F029C002F02AC003F02C6A2D6A17
:100B2000C80E2E6E420E2F6E00C027F001C028F0B6
:100B300002C029F003C02AF08EEC6DF027C07BF9CB
:100B400028C07CF929C07DF92AC07EF912C529F098
:100B5000D1EC6CF027C000F028C001F029C002F0F1
:100B60002AC003F02C6A2D6AC80E2E6E420E2F6E1C
:100B700000C027F001C028F002C029F003C02AF00D
:100B80008EEC6DF027C077F928C078F929C079F983
:100B90002AC07AF9EDEC93F044ECA4F00501236B44
:100BA0000501226B0501316BF1ECA4F0120050D865
:100BB0000901BD5105E1010EBD6F00EC60F002D0EE
:100BC000F3EC64F01EEC8CF0F1ECA4F00501235181
:100BD000030A27E0020A1DE0010A12E0C4EC9AF0C1
:100BE00044ECA4F0E3EC69F00301010E066FCBECDA
:100BF00090F0050123510F0824E2020E236F23D049
:100C0000C4EC9AF07EEC98F016EC63F005012369D1
:100C10001BD0030E235D01E117D0236B21EC8EF076
:100C200013D044ECA4F0E3EC69F0C2EC69F00201EB
:100C3000C76B926BC4EC9AF0FCEC64F00501236B7B
:100C400003D021EC8EF000D016EC9AF0F7EF64F0B0
:100C500000C528F001C529F0E2EC6CF027C000F0D7
:100C600028C001F029C002F02AC003F02C6A2D6AC6
:100C70007A0E2E6E440E2F6E00C027F001C028F0B1
:100C800002C029F003C02AF08EEC6DF027C00AF4F0
:100C900028C00BF429C00CF42AC00DF402C528F0BA
:100CA00003C529F0E2EC6CF027C000F028C001F089
:100CB00029C002F02AC003F02C6A2D6A7A0E2E6E2B
:100CC000440E2F6E00C027F001C028F002C029F0AA
:100CD00003C02AF08EEC6DF027C00EF428C00FF48C
:100CE00029C010F42AC011F410C529F0D1EC6CF021
:100CF00027C000F028C001F029C002F02AC003F08C
:100D00002C6A2D6AC80E2E6E420E2F6E00C027F080
:100D100001C028F002C029F003C02AF08EEC6DF06B
:100D200027C036F428C037F429C038F42AC039F473
:100D300011C529F0D1EC6CF027C000F028C001F0FB
:100D400029C002F02AC003F02C6A2D6AC80E2E6E4C
:100D5000420E2F6E00C027F001C028F002C029F01B
:100D600003C02AF08EEC6DF027C03AF428C03BF4A3
:100D700029C03CF42AC03DF41CC529F0D1EC6CF02C
:100D800027C000F028C001F029C002F02AC003F0FB
:100D90002C6A2D6AC80E2E6E420E2F6E00C027F0F0
:100DA00001C028F002C029F003C02AF08EEC6DF0DB
:100DB00027C05FF928C060F929C061F92AC062F92B
:100DC0001DC529F0D1EC6CF027C000F028C001F05F
:100DD00029C002F02AC003F02C6A2D6AC80E2E6EBC
:100DE000420E2F6E00C027F001C028F002C029F08B
:100DF00003C02AF08EEC6DF027C063F928C064F9B7
:100E000029C065F92AC066F908C529F0D1EC6CF053
:100E100027C000F028C001F029C002F02AC003F06A
:100E20002C6A2D6AC80E2E6E420E2F6E00C027F05F
:100E300001C028F002C029F003C02AF08EEC6DF04A
:100E400027C0D2F928C0D3F929C0D4F92AC0D5F9CE
:100E500009C529F0D1EC6CF027C000F028C001F0E2
:100E600029C002F02AC003F02C6A2D6AC80E2E6E2B
:100E7000420E2F6E00C027F001C028F002C029F0FA
:100E800003C02AF08EEC6DF027C0E2F928C0E3F928
:100E900029C0E4F92AC0E5F90AC529F0D1EC6CF0C3
:100EA00027C000F028C001F029C002F02AC003F0DA
:100EB0002C6A2D6AC80E2E6E420E2F6E00C027F0CF
:100EC00001C028F002C029F003C02AF08EEC6DF0BA
:100ED00027C0D6F928C0D7F929C0D8F92AC0D9F92E
:100EE0000BC529F0D1EC6CF027C000F028C001F050
:100EF00029C002F02AC003F02C6A2D6AC80E2E6E9B
:100F0000420E2F6E00C027F001C028F002C029F069
:100F100003C02AF08EEC6DF027C0E6F928C0E7F98F
:100F200029C0E8F92AC0E9F90CC529F0D1EC6CF028
:100F300027C000F028C001F029C002F02AC003F049
:100F40002C6A2D6AC80E2E6E420E2F6E00C027F03E
:100F500001C028F002C029F003C02AF08EEC6DF029
:100F600027C0DAF928C0DBF929C0DCF92AC0DDF98D
:100F70000DC529F0D1EC6CF027C000F028C001F0BD
:100F800029C002F02AC003F02C6A2D6AC80E2E6E0A
:100F9000420E2F6E00C027F001C028F002C029F0D9
:100FA00003C02AF08EEC6DF027C0EAF928C0EBF9F7
:100FB00029C0ECF92AC0EDF90EC529F0D1EC6CF08E
:100FC00027C000F028C001F029C002F02AC003F0B9
:100FD0002C6A2D6AC80E2E6E420E2F6E00C027F0AE
:100FE00001C028F002C029F003C02AF08EEC6DF099
:100FF00027C0DEF928C0DFF929C0E0F92AC0E1F9ED
:101000000FC529F0D1EC6CF027C000F028C001F02A
:1010100029C002F02AC003F02C6A2D6AC80E2E6E79
:10102000420E2F6E00C027F001C028F002C029F048
:1010300003C02AF08EEC6DF027C0EEF928C0EFF95E
:1010400029C0F0F92AC0F1F917C529F0D1EC6CF0EC
:1010500027C000F028C001F029C002F02AC003F028
:101060002C6A2D6AC80E2E6E420E2F6E00C027F01D
:1010700001C028F002C029F003C02AF08EEC6DF008
:1010800027C07FF928C080F929C081F92AC082F9D8
:1010900005010251005D0401046F0501035101596E
:1010A0000401056F960E0427000E052309016F6BDE
:1010B000706B716B726BC26BC36BC46BC56BC66BB1
:1010C000C76BC86BC96BCA6BCB6BCC6BCD6BCE6B74
:1010D000CF6BD06BD16B05011B5166E01B51640DCA
:1010E000F3CF06F4F4CF07F404010451065D055173
:1010F00007595AE21BC529F0D1EC6CF027C004F067
:1011000028C005F029C006F02AC007F0850E2C6E15
:10111000EB0E2D6E1F0E2E6E410E2F6E04C027F0AB
:1011200005C028F006C029F007C02AF08EEC6DF04B
:1011300027C000F028C001F029C002F02AC003F047
:101140000EC42CF00FC42DF010C42EF011C42FF0DB
:1011500000C027F001C028F002C029F003C02AF027
:10116000F8EC6CF027C06FF928C070F929C071F94C
:101170002AC072F97FC92CF080C92DF081C92EF0E8
:1011800082C92FF06FC927F070C928F071C929F002
:1011900072C92AF0F8EC6CF027C06FF928C070F91A
:1011A00029C071F92AC072F90501675166E06751DB
:1011B000640DF3CF06F4F4CF07F404010451065D87
:1011C000055107595AE267C529F0D1EC6CF027C0E8
:1011D00004F028C005F029C006F02AC007F0850EEB
:1011E0002C6EEB0E2D6E1F0E2E6E410E2F6E04C058
:1011F00027F005C028F006C029F007C02AF08EECC1
:101200006DF027C000F028C001F029C002F02AC00C
:1012100003F00EC42CF00FC42DF010C42EF011C436
:101220002FF000C027F001C028F002C029F003C051
:101230002AF0F8EC6CF027C0C2F928C0C3F929C025
:10124000C4F92AC0C5F97FC92CF080C92DF081C925
:101250002EF082C92FF0C2C927F0C3C928F0C4C933
:1012600029F0C5C92AF0F8EC6CF027C0C2F928C0F3
:10127000C3F929C0C4F92AC0C5F90501685166E05F
:101280006851640DF3CF06F4F4CF07F40401045160
:10129000065D055107595AE268C529F0D1EC6CF09A
:1012A00027C004F028C005F029C006F02AC007F0C6
:1012B000850E2C6EEB0E2D6E1F0E2E6E410E2F6EB8
:1012C00004C027F005C028F006C029F007C02AF0A6
:1012D0008EEC6DF027C000F028C001F029C002F0AC
:1012E0002AC003F00EC42CF00FC42DF010C42EF051
:1012F00011C42FF000C027F001C028F002C029F06F
:1013000003C02AF0F8EC6CF027C0C6F928C0C7F972
:1013100029C0C8F92AC0C9F97FC92CF080C92DF0AD
:1013200081C92EF082C92FF0C6C927F0C7C928F09D
:10133000C8C929F0C9C92AF0F8EC6CF027C0C6F971
:1013400028C0C7F929C0C8F92AC0C9F905016951DF
:1013500066E06951640DF3CF06F4F4CF07F404019D
:101360000451065D055107595AE269C529F0D1ECCF
:101370006CF027C004F028C005F029C006F02AC090
:1013800007F0850E2C6EEB0E2D6E1F0E2E6E410E8D
:101390002F6E04C027F005C028F006C029F007C052
:1013A0002AF08EEC6DF027C000F028C001F029C0B3
:1013B00002F02AC003F00EC42CF00FC42DF010C4AC
:1013C0002EF011C42FF000C027F001C028F002C099
:1013D00029F003C02AF0F8EC6CF027C0CAF928C045
:1013E000CBF929C0CCF92AC0CDF97FC92CF080C92E
:1013F0002DF081C92EF082C92FF0CAC927F0CBC9C0
:1014000028F0CCC929F0CDC92AF0F8EC6CF027C03F
:10141000CAF928C0CBF929C0CCF92AC0CDF90501F9
:101420006A5166E06A51640DF3CF06F4F4CF07F415
:1014300004010451065D055107595AE26AC529F0B5
:10144000D1EC6CF027C004F028C005F029C006F0EC
:101450002AC007F0850E2C6EEB0E2D6E1F0E2E6E21
:10146000410E2F6E04C027F005C028F006C029F0F9
:1014700007C02AF08EEC6DF027C000F028C001F004
:1014800029C002F02AC003F00EC42CF00FC42DF0C6
:1014900010C42EF011C42FF000C027F001C028F0B6
:1014A00002C029F003C02AF0F8EC6CF027C0CEF996
:1014B00028C0CFF929C0D0F92AC0D1F97FC92CF0B2
:1014C00080C92DF081C92EF082C92FF0CEC927F036
:1014D000CFC928F0D0C929F0D1C92AF0F8EC6CF0B6
:1014E00027C0CEF928C0CFF929C0D0F92AC0D1F938
:1014F00018C529F0D1EC6CF027C000F028C001F02D
:1015000029C002F02AC003F02C6A2D6AC80E2E6E84
:10151000420E2F6E00C027F001C028F002C029F053
:1015200003C02AF08EEC6DF027C0F3F528C0F4F567
:1015300029C0F5F52AC0F6F519C529F0D1EC6CF0F3
:1015400027C004F028C005F029C006F02AC007F023
:10155000660E2C6EE60E2D6EC70E2E6E420E2F6E90
:1015600004C027F005C028F006C029F007C02AF003
:101570008EEC6DF027C000F028C001F029C002F009
:101580002AC003F00EC42CF00FC42DF010C42EF0AE
:1015900011C42FF000C027F001C028F002C029F0CC
:1015A00003C02AF0F8EC6CF027C0F7F528C0F8F576
:1015B00029C0F9F52AC0FAF57FC92CF080C92DF0B1
:1015C00081C92EF082C92FF0F7C527F0F8C528F0A1
:1015D000F9C529F0FAC52AF0F8EC6CF027C0F7F548
:1015E00028C0F8F529C0F9F52AC0FAF51AC529F07E
:1015F000D1EC6CF027C000F028C001F029C002F047
:101600002AC003F02C6A2D6AC80E2E6E420E2F6E71
:1016100000C027F001C028F002C029F003C02AF062
:101620008EEC6DF027C0FBF528C0FCF529C0FDF558
:101630002AC0FEF513C529F0D1EC6CF027C000F0EC
:1016400028C001F029C002F02AC003F02C6A2D6ADC
:10165000C80E2E6E420E2F6E00C027F001C028F07B
:1016600002C029F003C02AF08EEC6DF027C07BF990
:1016700028C07CF929C07DF92AC07EF912C529F05D
:10168000D1EC6CF027C000F028C001F029C002F0B6
:101690002AC003F02C6A2D6AC80E2E6E420E2F6EE1
:1016A00000C027F001C028F002C029F003C02AF0D2
:1016B0008EEC6DF027C077F928C078F929C079F948
:1016C0002AC07AF915C529F0D1EC6CF027C000F0DA
:1016D00028C001F029C002F02AC003F02C6A2D6A4C
:1016E000C80E2E6E420E2F6E00C027F001C028F0EB
:1016F00002C029F003C02AF08EEC6DF027C097F2EB
:1017000028C098F229C099F22AC09AF214C529F08B
:10171000D1EC6CF027C000F028C001F029C002F025
:101720002AC003F02C6A2D6AC80E2E6E420E2F6E50
:1017300000C027F001C028F002C029F003C02AF041
:101740008EEC6DF027C09BF228C09CF229C09DF260
:101750002AC09EF297C22CF098C22DF099C22EF0AA
:101760009AC22FF09BC227F09CC228F09DC229F09C
:101770009EC22AF0F7EC6CF027C09FF228C0A0F2BE
:1017800029C0A1F22AC0A2F20EC42CF00FC42DF081
:1017900010C42EF011C42FF00AC427F00BC428F097
:1017A0000CC429F00DC42AF0F7EC6CF027C000F04F
:1017B00028C001F029C002F02AC003F0F00E2C6E00
:1017C000850E2D6E990E2E6E3E0E2F6E00C027F0E8
:1017D00001C028F002C029F003C02AF08EEC6DF0A1
:1017E00027C016F428C017F429C018F42AC019F429
:1017F00016C427F017C428F018C429F019C42AF019
:1018000093EC6EF028C004F429C005F40401000E26
:10181000045D000E055902E2046B056BFF0ED880D3
:101820000455000E055502E20469056B04C44FF22D
:1018300005011E510201C36FC46B1200010E0201AB
:101840009025906F000E9121916F0501185109E1CB
:101850000AC4EBF50BC4ECF50CC4EDF50DC4EEF5C4
:101860004ED0F3C52CF0F4C52DF0F5C52EF0F6C51D
:101870002FF00AC427F00BC428F00CC429F00DC4C3
:101880002AF0F7EC6CF027C000F028C001F029C066
:1018900002F02AC003F03AC42CF03BC42DF03CC443
:1018A0002EF03DC42FF036C427F037C428F038C4DA
:1018B00029F039C42AF0F8EC6CF027C004F028C0F5
:1018C00005F029C006F02AC007F004C02CF005C0BE
:1018D0002DF006C02EF007C02FF000C027F001C089
:1018E00028F002C029F003C02AF08EEC6DF027C06A
:1018F000EBF528C0ECF529C0EDF52AC0EEF50AC4D9
:101900002CF00BC42DF00CC42EF00DC42FF0EBC541
:1019100027F0ECC528F0EDC529F0EEC52AF0C9EC9A
:101920006EF0010A08E10AC4EBF50BC4ECF50CC437
:10193000EDF50DC4EEF5DC0E2C6E680E2D6E800EEE
:101940002E6E3D0E2F6EEBC527F0ECC528F0EDC5D1
:1019500029F0EEC52AF0C9EC6EF0010A01E097D03B
:10196000DC0E2C6E680E2D6E800E2E6E3D0E2F6ED0
:10197000EBC527F0ECC528F0EDC529F0EEC52AF03F
:10198000F7EC6CF027C000F028C001F029C002F08D
:101990002AC003F000C02CF001C02DF002C02EF0D0
:1019A00003C02FF036C427F037C428F038C429F01C
:1019B00039C42AF0E1EC6DF027C026F428C027F4E2
:1019C00029C028F42AC029F4DC0E2C6E680E2D6E76
:1019D000800E2E6E3D0E2F6EEBC527F0ECC528F065
:1019E000EDC529F0EEC52AF0F7EC6CF027C000F049
:1019F00028C001F029C002F02AC003F000C02CF07A
:101A000001C02DF002C02EF003C02FF03AC427F021
:101A10003BC428F03CC429F03DC42AF0E1EC6DF051
:101A200027C02AF428C02BF429C02CF42AC02DF496
:101A30000AC42CF00BC42DF00CC42EF00DC42FF0F2
:101A4000EBC527F0ECC528F0EDC529F0EEC52AF06E
:101A50008EEC6DF027C000F028C001F029C002F024
:101A60002AC003F02C6A2D6AC80E2E6E420E2F6E0D
:101A700000C027F001C028F002C029F003C02AF0FE
:101A8000E1EC6DF06CEC6EF029C064F50BD0040154
:101A9000266B276B286B296B2A6B2B6B2C6B2D6BA2
:101AA0000501646B0EC432F40FC433F410C434F473
:101AB00011C435F402014C5103E1EDEC93F002D076
:101AC000ECECADF005016351040DF3CFE9FFF4CF69
:101AD000EAFF6B0EE926050EEA22EECF00F0EECF0C
:101AE00001F0EECF02F0EFCF03F02C6A2D6A7A0EF0
:101AF0002E6E440E2F6E00C027F001C028F002C0E9
:101B000029F003C02AF0E1EC6DF093EC6EF028C0F0
:101B100044F229C045F205016351040DF3CFE9FFFA
:101B2000F4CFEAFF800EE926040EEA22EECF04F09D
:101B3000EECF05F0EECF06F0EFCF07F0100E6325E5
:101B4000040DF3CFE9FFF4CFEAFF800EE926040E7F
:101B5000EA22EECF08F0EECF09F0EECF0AF0EFCF99
:101B60000BF008C02CF009C02DF00AC02EF00BC0FD
:101B70002FF004C027F005C028F006C029F007C0E8
:101B80002AF0F8EC6CF027C000F028C001F029C062
:101B900002F02AC003F02C6A2D6A7A0E2E6E440ED3
:101BA0002F6E00C027F001C028F002C029F003C04A
:101BB0002AF0E1EC6DF093EC6EF028C046F229C0FB
:101BC00047F205011F051BE19BC22CF09CC22DF0C2
:101BD0009DC22EF09EC22FF012C427F013C428F02D
:101BE00014C429F015C42AF0E1EC6DF027C012F4FA
:101BF00028C013F429C014F42AC015F408D032C444
:101C000012F433C413F434C414F435C415F412C4F8
:101C10002CF013C42DF014C42EF015C42FF072C490
:101C200027F073C428F074C429F075C42AF0C9ECF5
:101C30006EF0010A05E10501235102E1226B2369DF
:101C400012000401086B096BFCEC64F00201000E49
:101C5000D880BF55000EC05501E388D236C467F95D
:101C600037C468F938C469F939C46AF93AC46BF9F8
:101C70003BC46CF93CC46DF93DC46EF905011851C3
:101C800001E00DD122C4EFF523C4F0F524C4F1F531
:101C900025C4F2F52C6A2D6A2E6A2F6A6FC927F0C7
:101CA00070C928F071C929F072C92AF0C2EC6EF02F
:101CB000010A24E06FC92CF070C92DF071C92EF013
:101CC00072C92FF022C427F023C428F024C429F0BD
:101CD00025C42AF0D2EC6EF0010A10E15FC967F961
:101CE00060C968F961C969F962C96AF963C96BF9C0
:101CF00064C96CF965C96DF966C96EF92C6A2D6AFB
:101D00002E6A2F6AC2C927F0C3C928F0C4C929F0B6
:101D1000C5C92AF0C2EC6EF0010A24E0C2C92CF059
:101D2000C3C92DF0C4C92EF0C5C92FF022C427F0B5
:101D300023C428F024C429F025C42AF0D2EC6EF084
:101D4000010A10E1D2C967F9D3C968F9D4C969F9A0
:101D5000D5C96AF9E2C96BF9E3C96CF9E4C96DF94F
:101D6000E5C96EF92C6A2D6A2E6A2F6AC6C927F05A
:101D7000C7C928F0C8C929F0C9C92AF0C2EC6EF059
:101D8000010A24E0C6C92CF0C7C92DF0C8C92EF03D
:101D9000C9C92FF022C427F023C428F024C429F095
:101DA00025C42AF0D2EC6EF0010A10E1D6C967F919
:101DB000D7C968F9D8C969F9D9C96AF9E6C96BF907
:101DC000E7C96CF9E8C96DF9E9C96EF92C6A2D6AA1
:101DD0002E6A2F6ACAC927F0CBC928F0CCC929F0CE
:101DE000CDC92AF0C2EC6EF0010A24E0CAC92CF079
:101DF000CBC92DF0CCC92EF0CDC92FF022C427F0CD
:101E000023C428F024C429F025C42AF0D2EC6EF0B3
:101E1000010A10E1DAC967F9DBC968F9DCC969F9B7
:101E2000DDC96AF9EAC96BF9EBC96CF9ECC96DF95E
:101E3000EDC96EF92C6A2D6A2E6A2F6ACEC927F079
:101E4000CFC928F0D0C929F0D1C92AF0C2EC6EF070
:101E5000010A24E0CEC92CF0CFC92DF0D0C92EF054
:101E6000D1C92FF022C427F023C428F024C429F0BC
:101E700025C42AF0D2EC6EF0010A10E1DEC967F940
:101E8000DFC968F9E0C969F9E1C96AF9EEC96BF916
:101E9000EFC96CF9F0C96DF9F1C96EF9B1D0F7C5A8
:101EA0002CF0F8C52DF0F9C52EF0FAC52FF022C49C
:101EB00027F023C428F024C429F025C42AF0C9EC53
:101EC0006EF0010A4FE1F3C52CF0F4C52DF0F5C515
:101ED0002EF0F6C52FF022C427F023C428F024C426
:101EE00029F025C42AF0F7EC6CF027C000F028C0D8
:101EF00001F029C002F02AC003F03AC42CF03BC420
:101F00002DF03CC42EF03DC42FF036C427F037C46A
:101F100028F038C429F039C42AF0F8EC6CF027C056
:101F200004F028C005F029C006F02AC007F004C05C
:101F30002CF005C02DF006C02EF007C02FF000C019
:101F400027F001C028F002C029F003C02AF08EEC6F
:101F50006DF027C0EFF528C0F0F529C0F1F52AC0D3
:101F6000F2F54ED0FBC52CF0FCC52DF0FDC52EF0D2
:101F7000FEC52FF022C427F023C428F024C429F082
:101F800025C42AF0F7EC6CF027C000F028C001F05F
:101F900029C002F02AC003F03AC42CF03BC42DF053
:101FA0003CC42EF03DC42FF036C427F037C428F0CF
:101FB00038C429F039C42AF0F8EC6CF027C004F0DA
:101FC00028C005F029C006F02AC007F004C02CF094
:101FD00005C02DF006C02EF007C02FF000C027F07E
:101FE00001C028F002C029F003C02AF08EEC6DF089
:101FF00027C0EFF528C0F0F529C0F1F52AC0F2F5A9
:1020000022C42CF023C42DF024C42EF025C42FF0BC
:10201000EFC527F0F0C528F0F1C529F0F2C52AF088
:10202000C9EC6EF0010A08E122C4EFF523C4F0F513
:1020300024C4F1F525C4F2F5DC0E2C6E680E2D6E6D
:10204000800E2E6E3D0E2F6EEFC527F0F0C528F0E6
:10205000F1C529F0F2C52AF0C9EC6EF0010A69E178
:10206000DC0E2C6E680E2D6E800E2E6E3D0E2F6EC9
:10207000EFC527F0F0C528F0F1C529F0F2C52AF028
:10208000F7EC6CF027C000F028C001F029C002F086
:102090002AC003F000C02CF001C02DF002C02EF0C9
:1020A00003C02FF067C927F068C928F069C929F073
:1020B0006AC92AF0E1EC6DF027C026F428C027F4A5
:1020C00029C028F42AC029F4DC0E2C6E680E2D6E6F
:1020D000800E2E6E3D0E2F6EEFC527F0F0C528F056
:1020E000F1C529F0F2C52AF0F7EC6CF027C000F03A
:1020F00028C001F029C002F02AC003F000C02CF073
:1021000001C02DF002C02EF003C02FF06BC927F0E4
:102110006CC928F06DC929F06EC92AF0E1EC6DF0A8
:1021200027C02AF428C02BF429C02CF42AC02DF48F
:1021300009D00401266B276B286B296B2A6B2B6B4C
:102140002C6B2D6B01EC9CF0F5EC69F00201010E9B
:10215000C16F53ECA4F005012329236F100E235DFA
:1021600004E2010E0401086F096B02D00501236B24
:102170000401010E081901E1095101E162D50501CF
:1021800023510F0803E2010E236F04D0C2EC69F063
:102190000501236B1200C4EC9AF00501236B0AC4FD
:1021A00022F40BC423F40CC424F40DC425F402015E
:1021B000010E926F0401086B096B2C6A2D6A800E68
:1021C0002E6E3F0E2F6E22C427F023C428F024C4A5
:1021D00029F025C42AF0F7EC6CF027C022F428C0BF
:1021E00023F429C024F42AC025F405011F0509E1C0
:1021F000B7C293F2B8C294F2B9C295F2BAC296F2DB
:1022000008D076C493F277C494F278C495F279C476
:1022100096F293C22CF094C22DF095C22EF096C285
:102220002FF022C427F023C428F024C429F025C4A9
:102230002AF0C9EC6EF0010A01E0C7D20EC42CF0FE
:102240000FC42DF010C42EF011C42FF022C427F0BB
:1022500023C428F024C429F025C42AF0C9EC6EF068
:10226000010A01E0B2D20201926B0301066B2C6AF3
:102270002D6A2E6A3F0E2F6E22C427F023C428F049
:1022800024C429F025C42AF0F8EC6CF027C022F40D
:1022900028C023F429C024F42AC025F436C467F9E1
:1022A00037C468F938C469F939C46AF93AC46BF9B2
:1022B0003BC46CF93CC46DF93DC46EF9050118517D
:1022C00001E00DD122C4EFF523C4F0F524C4F1F5EB
:1022D00025C4F2F52C6A2D6A2E6A2F6A6FC927F081
:1022E00070C928F071C929F072C92AF0C2EC6EF0E9
:1022F000010A24E06FC92CF070C92DF071C92EF0CD
:1023000072C92FF022C427F023C428F024C429F076
:1023100025C42AF0D2EC6EF0010A10E15FC967F91A
:1023200060C968F961C969F962C96AF963C96BF979
:1023300064C96CF965C96DF966C96EF92C6A2D6AB4
:102340002E6A2F6AC2C927F0C3C928F0C4C929F070
:10235000C5C92AF0C2EC6EF0010A24E0C2C92CF013
:10236000C3C92DF0C4C92EF0C5C92FF022C427F06F
:1023700023C428F024C429F025C42AF0D2EC6EF03E
:10238000010A10E1D2C967F9D3C968F9D4C969F95A
:10239000D5C96AF9E2C96BF9E3C96CF9E4C96DF909
:1023A000E5C96EF92C6A2D6A2E6A2F6AC6C927F014
:1023B000C7C928F0C8C929F0C9C92AF0C2EC6EF013
:1023C000010A24E0C6C92CF0C7C92DF0C8C92EF0F7
:1023D000C9C92FF022C427F023C428F024C429F04F
:1023E00025C42AF0D2EC6EF0010A10E1D6C967F9D3
:1023F000D7C968F9D8C969F9D9C96AF9E6C96BF9C1
:10240000E7C96CF9E8C96DF9E9C96EF92C6A2D6A5A
:102410002E6A2F6ACAC927F0CBC928F0CCC929F087
:10242000CDC92AF0C2EC6EF0010A24E0CAC92CF032
:10243000CBC92DF0CCC92EF0CDC92FF022C427F086
:1024400023C428F024C429F025C42AF0D2EC6EF06D
:10245000010A10E1DAC967F9DBC968F9DCC969F971
:10246000DDC96AF9EAC96BF9EBC96CF9ECC96DF918
:10247000EDC96EF92C6A2D6A2E6A2F6ACEC927F033
:10248000CFC928F0D0C929F0D1C92AF0C2EC6EF02A
:10249000010A24E0CEC92CF0CFC92DF0D0C92EF00E
:1024A000D1C92FF022C427F023C428F024C429F076
:1024B00025C42AF0D2EC6EF0010A10E1DEC967F9FA
:1024C000DFC968F9E0C969F9E1C96AF9EEC96BF9D0
:1024D000EFC96CF9F0C96DF9F1C96EF9CDD0F7C546
:1024E0002CF0F8C52DF0F9C52EF0FAC52FF022C456
:1024F00027F023C428F024C429F025C42AF0C9EC0D
:102500006EF0010A4FE1F3C52CF0F4C52DF0F5C5CE
:102510002EF0F6C52FF022C427F023C428F024C4DF
:1025200029F025C42AF0F7EC6CF027C000F028C091
:1025300001F029C002F02AC003F03AC42CF03BC4D9
:102540002DF03CC42EF03DC42FF036C427F037C424
:1025500028F038C429F039C42AF0F8EC6CF027C010
:1025600004F028C005F029C006F02AC007F004C016
:102570002CF005C02DF006C02EF007C02FF000C0D3
:1025800027F001C028F002C029F003C02AF08EEC29
:102590006DF027C0EFF528C0F0F529C0F1F52AC08D
:1025A000F2F54ED0FBC52CF0FCC52DF0FDC52EF08C
:1025B000FEC52FF022C427F023C428F024C429F03C
:1025C00025C42AF0F7EC6CF027C000F028C001F019
:1025D00029C002F02AC003F03AC42CF03BC42DF00D
:1025E0003CC42EF03DC42FF036C427F037C428F089
:1025F00038C429F039C42AF0F8EC6CF027C004F094
:1026000028C005F029C006F02AC007F004C02CF04D
:1026100005C02DF006C02EF007C02FF000C027F037
:1026200001C028F002C029F003C02AF08EEC6DF042
:1026300027C0EFF528C0F0F529C0F1F52AC0F2F562
:1026400022C42CF023C42DF024C42EF025C42FF076
:10265000EFC527F0F0C528F0F1C529F0F2C52AF042
:10266000C9EC6EF0010A08E122C4EFF523C4F0F5CD
:1026700024C4F1F525C4F2F52C6A2D6A2E6A3F0EAA
:102680002F6E22C427F023C428F024C429F025C4C7
:102690002AF0F7EC6CF027C022F428C023F429C0FC
:1026A00024F42AC025F4DC0E2C6E680E2D6E800EEC
:1026B0002E6E3D0E2F6EEFC527F0F0C528F0F1C548
:1026C00029F0F2C52AF0C9EC6EF0010A69E1DC0ECE
:1026D0002C6E680E2D6E800E2E6E3D0E2F6EEFC589
:1026E00027F0F0C528F0F1C529F0F2C52AF0F7EC83
:1026F0006CF027C000F028C001F029C002F02AC009
:1027000003F000C02CF001C02DF002C02EF003C079
:102710002FF067C927F068C928F069C929F06AC98C
:102720002AF0E1EC6DF027C026F428C027F429C078
:1027300028F42AC029F4DC0E2C6E680E2D6E800E53
:102740002E6E3D0E2F6EEFC527F0F0C528F0F1C5B7
:1027500029F0F2C52AF0F7EC6CF027C000F028C091
:1027600001F029C002F02AC003F000C02CF001C023
:102770002DF002C02EF003C02FF06BC927F06CC9FA
:1027800028F06DC929F06EC92AF0E1EC6DF027C080
:102790002AF428C02BF429C02CF42AC02DF409D027
:1027A0000401266B276B286B296B2A6B2B6B2C6B18
:1027B0002D6B01EC9CF005012329236F100E235D86
:1027C00004E2010E0401086F096B0401010E0819EF
:1027D00001E1095101E1EED4120013EE00F0010E07
:1027E000F86E050163690401726B736B746B756B32
:1027F0000401006B100E0401005D02E37DEF98F010
:10280000020EF76E04010051002500250025F66E2A
:102810000900F5CF5BF40900F5CF5AF40900F5CFB4
:102820005DF40800F5CF5CF4400FF66E0900F5CFBB
:102830005FF40900F5CF5EF40900F5CF61F40800FC
:10284000F5CF60F4400FF66E0900F5CF43F40900B0
:10285000F5CF42F40900F5CF45F40800F5CF44F474
:10286000400FF66E0900F5CF47F40900F5CF46F4A6
:102870000900F5CF49F40800F5CF48F4400FF66E93
:10288000F72A0900F5CF4BF40900F5CF4AF4090007
:10289000F5CF4DF40800F5CF4CF4400FF66E09006B
:1028A000F5CF4FF40900F5CF4EF40900F5CF51F400
:1028B0000800F5CF50F4D40E2C6E400E2D6E180E7D
:1028C0002E6E380E2F6E5AC427F05BC428F05CC4FD
:1028D00029F05DC42AF0D2EC6EF0010A01E1DED0ED
:1028E000450E2C6E120E2D6EBD0E2E6E3B0E2F6EF3
:1028F0005AC427F05BC428F05CC429F05DC42AF0F8
:10290000C9EC6EF0010A01E1C9D04B0E2C6E890EA4
:102910002D6EC90E2E6E380E2F6E5EC427F05FC46A
:1029200028F060C429F061C42AF0D2EC6EF0010AEC
:1029300001E1B4D09A0E2C6E990E2D6E190E2E6EEA
:102940003E0E2F6E5EC427F05FC428F060C429F0ED
:1029500061C42AF0C9EC6EF0010A01E19FD0440E77
:102960002C6E8B0E2D6E6C0E2E6E3E0E2F6E42C494
:1029700027F043C428F044C429F045C42AF0D2EC1F
:102980006EF0010A01E18AD05C0E2C6E8F0E2D6E66
:10299000A20E2E6E3F0E2F6E42C427F043C428F0C5
:1029A00044C429F045C42AF0C9EC6EF0010A76E06F
:1029B000250E2C6E060E2D6E010E2E6E3F0E2F6E06
:1029C0004AC427F04BC428F04CC429F04DC42AF067
:1029D000D2EC6EF0010A62E0C70E2C6E4B0E2D6E2B
:1029E000770E2E6E3F0E2F6E4AC427F04BC428F090
:1029F0004CC429F04DC42AF0C9EC6EF0010A4EE037
:102A00005C0E2C6E8F0E2D6E020E2E6E3F0E2F6EF4
:102A100046C427F047C428F048C429F049C42AF026
:102A2000D2EC6EF0010A3AE02C6A2D6AE00E2E6EAE
:102A30003F0E2F6E46C427F047C428F048C429F043
:102A400049C42AF0C9EC6EF0010A28E0750E2C6E1C
:102A5000930E2D6ED80E2E6E3E0E2F6E4EC427F0A6
:102A60004FC428F050C429F051C42AF0D2EC6EF0C3
:102A7000010A14E0DF0E2C6E4F0E2D6E6D0E2E6EC1
:102A80003F0E2F6E4EC427F04FC428F050C429F0DB
:102A900051C42AF0C9EC6EF0010A02E10901358B3C
:102AA00004010051040DF3CFE9FFF4CFEAFF800EDB
:102AB000E926040EEA22EECF04F0EECF05F0EECFC9
:102AC00006F0EFCF07F004C02CF005C02DF006C0D3
:102AD0002EF007C02FF026C427F027C428F028C402
:102AE00029F029C42AF0F7EC6CF027C000F028C0C8
:102AF00001F029C002F02AC003F05AC42CF05BC4D4
:102B00002DF05CC42EF05DC42FF000C027F001C092
:102B100028F002C029F003C02AF0E1EC6DF027C0D4
:102B20002EF428C02FF429C030F42AC031F41CEC54
:102B30006AF004010051040DF3CFE9FFF4CFEAFF7E
:102B4000800EE926040EEA22EECF04F0EECF05F067
:102B5000EECF06F0EFCF07F02EC42CF02FC42DF0EF
:102B600030C42EF031C42FF004C027F005C028F087
:102B700006C029F007C02AF0F8EC6CF027C000F07E
:102B800028C001F029C002F02AC003F0040100515E
:102B9000040DF3CFE9FFF4CFEAFF800EE926040E1F
:102BA000EA2200C0EEFF01C0EEFF02C0EEFF03C04C
:102BB000EEFF100E04010025040DF3CFE9FFF4CF62
:102BC000EAFF800EE926040EEA22EECF04F0EECFF3
:102BD00005F0EECF06F0EFCF07F004C02CF005C0F3
:102BE0002DF006C02EF007C02FF02AC427F02BC40A
:102BF00028F02CC429F02DC42AF0F7EC6CF027C083
:102C000000F028C001F029C002F02AC003F05EC421
:102C10002CF05FC42DF060C42EF061C42FF000C012
:102C200027F001C028F002C029F003C02AF0E1EC2F
:102C30006DF027C02EF428C02FF429C030F42AC02C
:102C400031F41CEC6AF0100E04010025040DF3CFE2
:102C5000E9FFF4CFEAFF800EE926040EEA22EECF68
:102C600004F0EECF05F0EECF06F0EFCF07F02EC464
:102C70002CF02FC42DF030C42EF031C42FF004C03E
:102C800027F005C028F006C029F007C02AF0F8ECAC
:102C90006CF027C000F028C001F029C002F02AC063
:102CA00003F0100E04010025040DF3CFE9FFF4CF6B
:102CB000EAFF800EE926040EEA2200C0EEFF01C002
:102CC000EEFF02C0EEFF03C0EEFF04010051040D51
:102CD000F3CFE9FFF4CFEAFF800EE926040EEA22E3
:102CE000EECF00F0EECF01F0EECF02F0EFCF03F029
:102CF000100E04010025040DF3CFE9FFF4CFEAFF25
:102D0000800EE926040EEA22EECF04F0EECF05F0A5
:102D1000EECF06F0EFCF07F004C02CF005C02DF089
:102D200006C02EF007C02FF000C027F001C028F029
:102D300002C029F003C02AF0F8EC6CF027C02EF492
:102D400028C02FF429C030F42AC031F40401005106
:102D5000040DF3CFE9FFF4CFEAFF800EE926040E5D
:102D6000EA22EECF08F0EECF09F0EECF0AF0EFCF77
:102D70000BF008C02CF009C02DF00AC02EF00BC0DB
:102D80002FF042C427F043C428F044C429F045C4BE
:102D90002AF0E1EC6DF027C004F028C005F029C04E
:102DA00006F02AC007F0100E04010025040DF3CF31
:102DB000E9FFF4CFEAFF800EE926040EEA22EECF07
:102DC00010F0EECF11F0EECF12F0EFCF13F010C0F5
:102DD0002CF011C02DF012C02EF013C02FF046C4FD
:102DE00027F047C428F048C429F049C42AF0E1EC90
:102DF0006DF027C00CF028C00DF029C00EF02AC0DD
:102E00000FF00CC02CF00DC02DF00EC02EF00FC036
:102E10002FF004C027F005C028F006C029F007C035
:102E20002AF0F8EC6CF027C000F028C001F029C0AF
:102E300002F02AC003F02EC42CF02FC42DF030C4B1
:102E40002EF031C42FF000C027F001C028F002C0DE
:102E500029F003C02AF08EEC6DF027C042F428C0A0
:102E600043F429C044F42AC045F404010051040D80
:102E7000F3CFE9FFF4CFEAFF800EE926040EEA2241
:102E8000EECF08F0EECF09F0EECF0AF0EFCF0BF067
:102E900008C02CF009C02DF00AC02EF00BC02FF096
:102EA0004AC427F04BC428F04CC429F04DC42AF082
:102EB000E1EC6DF027C004F028C005F029C006F051
:102EC0002AC007F0100E04010025040DF3CFE9FF1E
:102ED000F4CFEAFF800EE926040EEA22EECF10F0CE
:102EE000EECF11F0EECF12F0EFCF13F010C02CF0B8
:102EF00011C02DF012C02EF013C02FF04EC427F0D9
:102F00004FC428F050C429F051C42AF0E1EC6DF010
:102F100027C00CF028C00DF029C00EF02AC00FF019
:102F20000CC02CF00DC02DF00EC02EF00FC02FF0F5
:102F300004C027F005C028F006C029F007C02AF019
:102F4000F8EC6CF027C000F028C001F029C002F0B6
:102F50002AC003F02EC42CF02FC42DF030C42EF064
:102F600031C42FF000C027F001C028F002C029F0C2
:102F700003C02AF08EEC6DF027C04AF428C04BF451
:102F800029C04CF42AC04DF442C42CF043C42DF0A7
:102F900044C42EF045C42FF02EC427F02FC428F0CF
:102FA00030C429F031C42AF0F7EC6CF027C004F0EB
:102FB00028C005F029C006F02AC007F04AC42CF04A
:102FC0004BC42DF04CC42EF04DC42FF004C027F09C
:102FD00005C028F006C029F007C02AF0E1EC6DF02A
:102FE00027C000F028C001F029C002F02AC003F079
:102FF00004010051040DF3CFE9FFF4CFEAFF6B0E9B
:10300000E926050EEA2200C0EEFF01C0EEFF02C075
:10301000EEFF03C0EEFF04010051040DF3CFE9FF02
:10302000F4CFEAFF6B0EE926050EEA22EECF00F0A0
:10303000EECF01F0EECF02F0EFCF03F02C6A2D6A55
:103040002E6A2F6A00C027F001C028F002C029F0C4
:1030500003C02AF0D2EC6EF0010A0FE10401005126
:10306000040DF3CFE9FFF4CFEAFF6B0EE926050E5E
:10307000EA22EE6AEE6AEE6AEE6A04010051040D7D
:10308000F3CFE9FFF4CFEAFF6B0EE926050EEA2243
:10309000EECF00F0EECF01F0EECF02F0EFCF03F075
:1030A00072C42CF073C42DF074C42EF075C42FF0CC
:1030B00000C027F001C028F002C029F003C02AF0A8
:1030C000C9EC6EF0010A15E104010051040DF3CFC3
:1030D000E9FFF4CFEAFF6B0EE926050EEA22EECFF8
:1030E00072F4EECF73F4EECF74F4EFCF75F400C446
:1030F00063F50401002BFAEF93F012000501226B37
:10310000010E0401046F056BEDD822ECA0F00A0E4D
:1031100005012225226F010E04010425046F000E13
:103120000521056F05011F0535E1B3C22CF0B4C2BE
:103130002DF0B5C22EF0B6C22FF09BC227F09CC274
:1031400028F09DC229F09EC22AF0E1EC6DF027C064
:1031500000F028C001F029C002F02AC003F0AFC27D
:103160002CF0B0C22DF0B1C22EF0B2C22FF000C0D0
:1031700027F001C028F002C029F003C02AF0F8ECC3
:103180006CF027C012F428C013F429C014F42AC02C
:1031900015F408D076C412F477C413F478C414F488
:1031A00079C415F432C42CF033C42DF034C42EF09D
:1031B00035C42FF012C427F013C428F014C429F02A
:1031C00015C42AF0C9EC6EF0010A03E10401046998
:1031D000056B0401110E045D000E055995E3FF0E09
:1031E000041901E1055105E1CFD80A0E0501225D60
:1031F000226F010E0401046F056B3C0E0501225D78
:1032000070E2FFDA05012229226F010E0401042574
:10321000046F000E0521056F05011F0535E1B3C2DE
:103220002CF0B4C22DF0B5C22EF0B6C22FF09BC266
:1032300027F09CC228F09DC229F09EC22AF0E1EC42
:103240006DF027C000F028C001F029C002F02AC0AC
:1032500003F0AFC22CF0B0C22DF0B1C22EF0B2C25A
:103260002FF000C027F001C028F002C029F003C0F1
:103270002AF0F8EC6CF027C012F428C013F429C02F
:1032800014F42AC015F408D076C412F477C413F4E9
:1032900078C414F479C415F432C42CF033C42DF07E
:1032A00034C42EF035C42FF012C427F013C428F014
:1032B00014C429F015C42AF0C9EC6EF0010A03E128
:1032C00004010469056B04010A0E045D000E055932
:1032D00098E3FF0E041901E1055103E10501220500
:1032E000226F12000401016B100E015D4CE20151CE
:1032F000040DF3CFE9FFF4CFEAFF000EE926060E36
:10330000EA22EECF00F0EECF01F0EECF02F0EFCFE9
:1033100003F00151040DF3CFE9FFF4CFEAFF800E73
:10332000E926060EEA2200C0EEFF01C0EEFF02C051
:10333000EEFF03C0EEFF100E0125040DF3CFE9FFF1
:10334000F4CFEAFF000EE926060EEA22EECF00F0E7
:10335000EECF01F0EECF02F0EFCF03F0100E01251B
:10336000040DF3CFE9FFF4CFEAFF800EE926060E45
:10337000EA2200C0EEFF01C0EEFF02C0EEFF03C074
:10338000EEFF012BB1D712000401016B100E015D9D
:103390004CE20151040DF3CFE9FFF4CFEAFF800EB8
:1033A000E926060EEA22EECF00F0EECF01F0EECFD6
:1033B00002F0EFCF03F00151040DF3CFE9FFF4CF9A
:1033C000EAFF000EE926060EEA2200C0EEFF01C069
:1033D000EEFF02C0EEFF03C0EEFF100E0125040D4C
:1033E000F3CFE9FFF4CFEAFF800EE926060EEA22CA
:1033F000EECF00F0EECF01F0EECF02F0EFCF03F012
:10340000100E0125040DF3CFE9FFF4CFEAFF000E03
:10341000E926060EEA2200C0EEFF01C0EEFF02C060
:10342000EEFF03C0EEFF012BB1D712000EC42CF04B
:103430000FC42DF010C42EF011C42FF00AC427F0D1
:103440000BC428F00CC429F00DC42AF0C9EC6EF0AE
:10345000010A01E096D005012351010A49E0030A5F
:1034600045E00EC42CF00FC42DF010C42EF011C492
:103470002FF00AC427F00BC428F00CC429F00DC4A7
:103480002AF0F7EC6CF027C000F028C001F029C04A
